:020000040800F2
:203000007829002001310008DF1901087DC50008DD180108354B00089D5B010800000000E3
:203020000000000000000000000000003F350108C56D000800000000411D0108A144010884
:203040001B3100081B3100081B3100081B3100081B3100081B3100081B3100081B310008D0
:20306000CD7300081B3100081B310008855B00081B3100081B3100081B3100081B31000828
:203080001B3100081B310008C54200081B31000865540108394B00081B3100081B3100082F
:2030A0001B310008CD4501081B3100081B3100081B3100081B3100081B3100081B310008A9
:2030C0001B3100081B3100081B3100081B3100081B3100081B3100081B31000879530108CF
:2030E000C17300081B3100081B310008DFF80CD001F098F800480047A1420008782900207D
:203100000648804706480047FEE7FEE7FEE7FEE7FEE7FEE7FEE7FEE7FEE7FEE77545010850
:20312000ED3000082DE9FF1F002000210022002300240025002600275FF000085FF000096B
:203140005FF0000A5FF0000B5FF0000C002001210222032304240525062607275FF00808CA
:203160005FF009095FF00A0A5FF00B0B5FF00C0C00281DD101291BD1022A19D1032B17D167
:20318000042C15D1052D13D1062E11D1072F0FD1B8F1080F0CD1B9F1090F09D1BAF10A0FDA
:2031A00006D1BBF10B0F03D1BCF10C0F00D101E004F0E4BBBDE8FF1F7047000073B40020D0
:2031C00000210124002501262046A04226D1A94224D12846A84221D1A9421FD14FEA440498
:2031E00006F10106202EEFDD5FF0FF305FF0FF317FF000445FF0FF3501262046A0420DD137
:20320000A9420BD12846A84208D1A94206D14FEA740406F10106202EEFDD01E004F0AEBBED
:2032200073BC7047E7B40021002000220125002601272946A94230D1B0422ED1B2422CD1F9
:203240003146B14229D1B04227D1B24225D14FEA450507F10107202FEBDD5FF0FF315FF0CE
:20326000FF305FF0FF327FF000455FF0FF3601272946A94211D1B0420FD1B2420DD13146E8
:20328000B1420AD1B04208D1B24206D14FEA750507F10107202FEBDD01E004F06FBBE7BC5E
:2032A00070472DE9CE01002200210023012600275FF001083246B24233D1B94231D1BB42FC
:2032C0002FD13A46BA422CD1B9422AD1BB4228D14FEA460608F10108B8F1200FEADD5FF014
:2032E000FF325FF0FF315FF0FF337FF000465FF0FF375FF001083246B24212D1B94210D1E0
:20330000BB420ED13A46BA420BD1B94209D1BB4207D14FEA760608F10108B8F1200FEADD79
:2033200001E004F02BBBBDE8CE0170472DE99C0300230022002401275FF000085FF00109B1
:203340003B46BB4233D1424531D144452FD1434643452CD142452AD1444528D14FEA470740
:2033600009F10109B9F1200FEADD5FF0FF335FF0FF325FF0FF347FF000475FF0FF385FF09B
:2033800001093B46BB4212D1424510D144450ED1434643450BD1424509D1444507D14FEA0A
:2033A000770709F10109B9F1200FEADD01E004F0E5BABDE89C0370472DE9381C00240023CB
:2033C00000255FF0010A5FF0000B5FF0010C5446544533D15B4531D15D452FD15C465C45FA
:2033E0002CD15B452AD15D4528D14FEA4A0A0CF1010CBCF1200FEADD5FF0FF345FF0FF335D
:203400005FF0FF357FF0004A5FF0FF3B5FF0010C5446544512D15B4510D15D450ED15C46D1
:203420005C450BD15B4509D15D4507D14FEA7A0A0CF1010CBCF1200FEADD01E004F09EBA84
:20344000BDE8381C70472DE9701C0025002400265FF0010A5FF0000B5FF0010C5546554566
:2034600033D15C4531D15E452FD15D465D452CD15C452AD15E4528D14FEA4A0A0CF1010CF1
:20348000BCF1200FEADD5FF0FF355FF0FF345FF0FF367FF0004A5FF0FF3B5FF0010C5546C7
:2034A000554512D15C4510D15E450ED15D465D450BD15C4509D15E4507D14FEA7A0A0CF1BA
:2034C000010CBCF1200FEADD01E004F057BABDE8701C70472DE9E01C0026002500275FF09B
:2034E000010A5FF0000B5FF0010C5646564533D15D4531D15F452FD15E465E452CD15D45A2
:203500002AD15F4528D14FEA4A0A0CF1010CBCF1200FEADD5FF0FF365FF0FF355FF0FF374D
:203520007FF0004A5FF0FF3B5FF0010C5646564512D15D4510D15F450ED15E465E450BD1AA
:203540005D4509D15F4507D14FEA7A0A0CF1010CBCF1200FEADD01E004F010BABDE8E01CC9
:2035600070472DE9C01D002700265FF000085FF0010A5FF0000B5FF0010C5746574533D1B0
:203580005E4531D1D8452FD15F465F452CD15E452AD1D84528D14FEA4A0A0CF1010CBCF12B
:2035A000200FEADD5FF0FF375FF0FF365FF0FF387FF0004A5FF0FF3B5FF0010C57465745AF
:2035C00012D15E4510D1D8450ED15F465F450BD15E4509D1D84507D14FEA7A0A0CF1010C2A
:2035E000BCF1200FEADD01E004F0C8B9BDE8C01D70472DE9801F5FF0000800275FF000090E
:203600005FF0010A5FF0000B5FF0010CD046D04533D15F4531D1D9452FD1D846D8452CD16F
:203620005F452AD1D94528D14FEA4A0A0CF1010CBCF1200FEADD5FF0FF385FF0FF375FF040
:20364000FF397FF0004A5FF0FF3B5FF0010CD046D04512D15F4510D1D9450ED1D846D845C9
:203660000BD15F4509D1D94507D14FEA7A0A0CF1010CBCF1200FEADD01E004F07FB9BDE8DE
:20368000801F70472DE970075FF000095FF000085FF0000A012400250126A146A14530D100
:2036A000A8452ED1AA452CD1A946A94529D1A84527D1AA4525D14FEA440406F10106202EC4
:2036C000EBDD5FF0FF395FF0FF385FF0FF3A7FF000445FF0FF350126A146A14511D1A84594
:2036E0000FD1AA450DD1A946A9450AD1A84508D1AA4506D14FEA740406F10106202EEBDD14
:2037000001E004F03BB9BDE8700770472DE9700E5FF0000A5FF000095FF0000B0124002524
:203720000126A246A24530D1A9452ED1AB452CD1AA46AA4529D1A94527D1AB4525D14FEADA
:20374000440406F10106202EEBDD5FF0FF3A5FF0FF395FF0FF3B7FF000445FF0FF35012618
:20376000A246A24511D1A9450FD1AB450DD1AA46AA450AD1A94508D1AB4506D14FEA740403
:2037800006F10106202EEBDD01E004F0F7B8BDE8700E70472DE9701C5FF0000B5FF0000A62
:2037A0005FF0000C012400250126A346A34530D1AA452ED1AC452CD1AB46AB4529D1AA45C5
:2037C00027D1AC4525D14FEA440406F10106202EEBDD5FF0FF3B5FF0FF3A5FF0FF3C7FF06B
:2037E00000445FF0FF350126A346A34511D1AA450FD1AC450DD1AB46AB450AD1AA4508D106
:20380000AC4506D14FEA740406F10106202EEBDD01E004F0B3B8BDE8701C70472DE9701855
:203820005FF0000C5FF0000B012400250126A446A44526D1AB4524D1AC46AC4521D1AB45EE
:203840001FD14FEA440406F10106202EEFDD5FF0FF3C5FF0FF3B7FF000445FF0FF3501266F
:20386000A446A4450DD1AB450BD1AC46AC4508D1AB4506D14FEA740406F10106202EEFDD7F
:2038800001E004F07BB8BDE8701870472DE9F0030024002546594E51445105F10405182DD3
:2038A000F8DB04255FF0000801245FF0010944514659B4425FD105F10407C659B0455AD19D
:2038C0002F1FC659B04556D140F805804659B04551D105F10407C659B0454CD12F1FC6594D
:2038E000B04548D14FEA440409F10109B9F1200FDDDD05F10405142DD6DB5FF0FF3400250A
:20390000445105F10405182DFADB04255FF0FF387FF000445FF0010944514659B4422AD119
:2039200005F10407C659B04525D12F1FC659B04521D140F805804659B0451CD105F10407E9
:20394000C659B04517D12F1FC659B04513D14FEA740409F10109B9F1200FDDDD05F10405DE
:20396000142DD5DB00254E59465105F10405182DF9DB012000E00020BDE8F00370472DE955
:20398000F00300240025445105F104058D42FADB00255FF0000801245FF001094451465985
:2039A000B44268D1002D03D02F1FC659B04562D105F104078F4202DAC659B0455BD140F81D
:2039C00005804659B04556D1002D03D02F1FC659B04550D105F104078F4202DAC659B04562
:2039E00049D14FEA440409F10109B9F1200FD5DD05F104058D42CEDB5FF0FF3400254451EA
:203A000005F104058D42FADB00255FF0FF387FF000445FF0010944514659B4422BD1002DF9
:203A200003D02F1FC659B04525D105F104078F4202DAC659B0451ED140F805804659B04559
:203A400019D1002D03D02F1FC659B04513D105F104078F4202DAC659B0450CD14FEA7404E6
:203A600009F10109B9F1200FD5DD05F104058D42CDDB012000E00020BDE8F0037047202A87
:203A800004DB203A21FA02F00021704721FA02F3D040C2F12002914008431946704740EAB7
:203AA00001039B0703D009E008C9121F08C0042AFAD203E011F8013B00F8013B521EF9D249
:203AC0007047D2B201E000F8012B491EFBD270470022F6E710B513460A4604461946FFF7AF
:203AE000F0FF204610BD10B5044604E00B7800F8013B03B1491C521EF8D2204610BD421C16
:203B000010F8011B0029FBD1801A704730B505460020034600E05B1C934205D2EC5CC85C33
:203B2000201A01D1002CF6D130BD2DE9F0410546002090460E46044600E0641C44450BD2AD
:203B4000285D00F083FA0746305D00F07FFA381A02D1295D0029F0D1BDE8F081F0B480EA77
:203B60000102D40F4200B2EB410F02D20246084611464A0042D0C30DDDB2C1F3C752AD1A20
:203B8000202D35DAC1F3160141F4000204B15242C5F1200602FA06F12A411044B3EBD05F23
:203BA00023D0C4B1012DA0EBC35009DCF0BC4FF0004202EAC352DBB200F5000000F055BA3D
:203BC000400000F1807000EBC350A0F1807040EAD170490009E0490841EAC071A0EBC3505D
:203BE00000F50000400800EBC350F0BC00F034BA6142012202EB4101001BF6E7F0BC7047B0
:203C000081F00041AAE780F00040A7E780EA010210B502F00043400022D04A001FD0010E42
:203C200001EB1261C0F35600C2F3560240F4000042F40002A0FB022000047F39140400D042
:203C4000401C50EA124001D44000491EC2B20C0604EBD010401C4008802A02D003E0002088
:203C600010BD20F00100002900DA0020184310BD2DE9FE4F804681EA0300C00F0C460090D3
:203C800021F0004123F00045B8EB0200A94105D24046214690461C460B46024623F0004003
:203CA000104347D0270DC7F30A00C3F30A510290401A019040286BDAC3F3130040F4801BCF
:203CC0000098924620B10023D2EB030A63EB0B0B01985946C0F14002504600F096F90646C6
:203CE0000D4650465946019A00F09EF910EB08006141002487EA115284EAE7731A4340D048
:203D0000009A62B3019A012A4FEA075215DC001B61EB02014FF0004202EA0752CDE9004283
:203D2000001C41F5801132462B4600F0DBF903B0BDE8F08F40462146F9E7001B61EB0201E5
:203D4000001C41F5801300185B412018A2F5001747EB030140EAD570B6196D4111E06D085C
:203D60004FEA360645EAC0754FEA0752001B61EB0201001C41F5801149084FEA30000019B8
:203D8000514132462B4603B0BDE8F04F00F09BB90098012240000023D0EB020263EBE0734F
:203DA000009821464FEAE074B8EB000061EB0401E9E783F000435BE781F0004158E72DE9B4
:203DC000F04D81EA030404F0004B21F0004514464FF0000A23F0004150EA050220D054EA39
:203DE00001021DD0C5F30A570246C5F31303C1F31300C1F30A5640F4801543F48013A7EBA4
:203E00000608101BD64608F2FD3873EB050002D308F1010801E092185B41B8F1000F03DA28
:203E200000200146BDE8F08D00204FF48011064684460EE0171B73EB050705D3121B63EB12
:203E4000050306434CEA010C49084FEA300092185B4150EA0107EDD152EA030012D082EA41
:203E6000040083EA0501084305D0101BAB4106D20122002306E000224FF0004302E06FF0AB
:203E8000010253101AEB06004CEB085110EB0A0041EB0B01BDE8F04D00F015B99623002269
:203EA000114600F0E2B80EB5C10F80EAE0700844CA07002140F233438DE80E000A460B46CA
:203EC00000F010F903B000BD0EB540F2334102910021CDE900110A460B4600F003F903B055
:203EE00000BD00F0004220F00040C10DC0F3160040F400007F2901DA00207047962903DCC0
:203F0000C1F19601C84001E096398840002AF4D04042704720F00040C10DC0F3160040F496
:203F200000007F2901DA00207047962903DCC1F19601C840704796398840704770B5C1F35A
:203F40000A5201F000450024C1F3130140F2FF3341F480119A4201DA002070BD40F233430D
:203F60009A42A2F2334203DC5242FFF788FD00E090402C43F1D0404270BDC1F30A5210B50A
:203F8000C1F3130140F2FF3341F480119A4201DA002010BD40F233439A42A2F2334203DC1F
:203FA0005242FFF76CFD10BD904010BD00F0004230F000400AD0C10D01F56071C0F31600DA
:203FC00042EA0151C20840071143704700200146704701F0004330B421F0004150EA010282
:203FE00006D00A0DA2F56072C1F31301002A02DC30BC00207047440F44EAC104C100E018D9
:2040000030BC00EBC25000F027B8202A04DB203A00FA02F1002070479140C2F1200320FAE0
:2040200003F3194390407047202A06DBCB17203A41FA02F043EAE07306E041FA02F3D0406D
:20404000C2F120029140084319467047A0F14101192900D8203070470029A8BF7047401CC2
:20406000490008BF20F00100704710B4B0FA80FC00FA0CF050EA010404BF10BC704749B109
:20408000CCF1200421FA04F411FA0CF118BF012121430843A3EB0C01CB1D4FEA00614FEA26
:2040A000102042BF002010BC704700EBC35010440029A4BF10BC7047401C490008BF20F04F
:2040C000010010BC704710B5141E73F1000408DA401C41F1000192185B411A4301D120F007
:2040E000010010BD2DE9F04D92469B4611B1B1FA81F202E0B0FA80F220329046FFF785FF66
:2041000004460F4640EA0A0041EA0B0153465A46084313D0114653EA010019D0C8F14002B5
:204120005046FFF7ACFC05460E46504659464246FFF76BFF084305D0012004E02046394685
:20414000BDE8F08D0020054346EAE0762C4337430A986305E40AA0EB08000022FD0A44EA84
:2041600047540A3002D500200146E9E7010510196941DDE9084500196941BDE8F04DA2E742
:204180002DE9F04D00231A461B1A8A4103DB00200146BDE8F08DC1F30A52C1F3130141F4D5
:2041A00080154FF0000BD10702D100186D41521E0027044640F2FF11384601EB620A3E4632
:2041C0008046024600204FF48011FFF758FCC2197141BB1846EB0100B4EB030C75EB000CE7
:2041E00004D3E41A65EB000517460E46241908F101006D4180463428E3DDF91946EB0600D4
:20420000091BA84103D24FF0FF32134601E0002213461BEB070046EB0A51BDE8F04DFFF726
:2042200052BF0000064C074D06E0E06840F0010394E8070098471034AC42F6D3FEF75AFFBA
:20424000087E0108287E010870B58C1810F8015B15F0070301D110F8013B2A1106D110F8B4
:20426000012B03E010F8016B01F8016B5B1EF9D12B0705D40023521E0DD401F8013BFAE77E
:2042800010F8013BCB1A921C03E013F8015B01F8015B521EF9D5A142D8D3002070BD00008F
:2042A00010B572B606480079AA2801D00FF048F800200349087162B612F076F910BD00002D
:2042C0000030024010B5024804F0E4FD10BD0000A41D002070B5044600252068806800F0E6
:2042E0000100F0B12068806820F001002168886006F08AFA05460EE006F086FA401B02287C
:2043000009D9A06A40F01000A062E06A40F00100E062012070BD2068806800F001000028DB
:20432000EAD10020F6E770B505466C6AA06A00F05000E0B9A06A40F40070A062206880687C
:2043400000F46020B0F5602F0DD1E06858B9A06A20F48070A062A06A00F4805018B9A06AC5
:2043600040F00100A062204604F0C0FB03E0206A016B2846884770BD70B505466C6AA06A62
:2043800040F04000A062E06A40F00400E062204604F07FFD70BD70B50446656A284604F048
:2043A00077FD70BD38B504460025002000902068806800F0010080BB2068806840F0010013
:2043C00021688860164800681649B0FBF1F0009002E00098401E009000980028F9D106F043
:2043E00013FA054613E006F00FFA401B02280ED9A06A40F01000A062E06A40F00100E062FE
:2044000000BF002084F8240000BF012038BD2068806800F001000028E5D00020F6E700000D
:204420000000002040420F0070B505460E4606F0EBF922490968401A02283DD3002418E0A1
:204440001F4850F824001F4931F81410C0EB81201B4951F8241001EBE010194941F824000C
:20446000084650F82400C0F38F2025F81400601CC4B2092CE4DB002418E0134850F8240026
:20448000124931F81410C0EB81200F4951F8241001EBE0100C4941F82400084650F824000B
:2044A000C0F38F2026F81400601CC4B2032CE4DB06F0AAF90149086070BD00006805002083
:2044C000181E0020501D00203C1E00201405002010B5154803F0CEFF144803F0CBFF1248F1
:2044E00004F08EFE114804F08BFE104804F0D2F909220F490C4804F01BFF0B48006A006845
:20450000006820F004000849096A09680860094807F0BDF90C21074807F030FC0C2105486B
:2045200007F0D6F810BD0000741D0020A41D0020501D0020901C0020014600226648814224
:204540000DD1664848604A68824201D000207047634848604A68824201D00020F7E76148C8
:2045600081420DD1604848604A68824201D00020EDE75E4848604A68824201D00020E6E78D
:2045800040F2555048614A69824201D00020DEE740F6AA2048614A69824201D00020D6E7A0
:2045A00040F2555088618A69824201D00020CEE740F6AA2088618A69824201D00020C6E7A0
:2045C00040F25550C861CA69824201D00020BEE740F6AA20C861CA69824201D00020B6E7A0
:2045E00040F2555008620A6A824201D00020AEE740F6AA2008620A6A824201D00020A6E79C
:2046000040F2555048624A6A824201D000209EE740F6AA2048624A6A824201D0002096E79B
:2046200040F2555088628A6A824201D000208EE740F6AA2088628A6A824201D0002086E79B
:204640002B48C862CA6A824201D000207FE72948C862CA6A824201D0002078E726480863B2
:204660000A6B824201D0002071E7244808630A6B824201D000206AE71F4848634A6B8242DB
:2046800001D0002063E71D4848634A6B824201D000205CE71A4888638A6B824201D000202B
:2046A00055E7184888638A6B824201D000204EE700204860C860086148618861C861086216
:2046C00040F6FF70486200208862C86208634863886301203BE700000024014055554500BF
:2046E000AAAA8A000028014055554000AAAA800055555500AAAAAA0055555515AAAAAA2A7C
:2047000055551500AAAA2A0088B001460022086800904868019088680290CB6803930B69BB
:2047200004934B690593552008600A68552A02D0002008B07047AA2008600A68AA2A01D01E
:204740000020F6E745F2555048604A68824201D00020EEE74AF6AA20486048684AF6AA232D
:2047600000EA03021846824201D00020E1E745F2555088608A68824201D00020D9E742F60C
:20478000AA2088608A68824201D00020D1E745F25553CB60CA681846824201D00020C8E70A
:2047A00042F6AA23CB60CA681846824201D00020BFE745F255530B610A691846824201D02D
:2047C0000020B6E742F6AA230B610A691846824201D00020ADE745F255534B614A691846F5
:2047E000824201D00020A4E742F6AA234B614A691846824201D000209BE7009808600198E7
:20480000486002988860039BCB60049B0B61059B4B6101208DE70246002004E0002322F830
:204820001030431C98B28842F8DB70472DE9F04704460E46924699466527844800780128A0
:204840007AD105F0E1FF40F6C411884202D20020BDE8F0877E480088401C7D490880608A71
:204860007C49096808447B49086079480088012801DC1920ECE776480088032801DC32208F
:20488000E6E773480088052801DC4B20E0E770480088072801DC6420DAE700206B490870EF
:2048A000B9F1180F0AD16B480068C0F3CF0000EB80004000072190FBF1F011E0B9F1300F96
:2048C0000AD164480068C0F3CF0000EB800040000D2190FBF1F003E05E480068C0F3CF00AF
:2048E00080B25D490880002523E0781EA84205DC4FF00008C4F804800020A9E7B01C30F8A4
:2049000015005549098888420EDC30886843642190FBF1F03188A1EB0008C4F80480781B2B
:20492000401EC0B294E707E04FF00008681C80B20546BD42D9DB86E0484880F800A00078C4
:2049400047490870607C00287AD143F698216069B0FBF1F081B2434802780078401C414B21
:20496000187004F11C0020F81210184600780C2827DBB9F1180F0BD10C2104F11C0003F07A
:20498000C3FC00EB80004000072190FBF1F013E0B9F1300F0BD10C2104F11C0003F0B4FC80
:2049A00000EB800040000D2190FBF1F004E00C2104F11C0003F0A8FC27490880002029496F
:2049C0000870002524E0781EA84207DC4FF00008C4F804800020224908701BE0B01C30F85A
:2049E00015001D49098888420EDC30886843642190FBF1F03188A1EB0008C4F80480781B83
:204A0000401E1749087005E04FF00008681C85B2BD42D8DB00BF1248007810490978884292
:204A20000ADD0F4801780D4800781430814203DA0A4800780A4908700020606101206074A3
:204A40000748007804E700BF02E700008A03002086030020900300208C0300208903002098
:204A6000880300208B03002030B51E2A04DB0CDB64280ADA0A2908DA9C891C809C89DC8122
:204A80009C895C8000245C6030BD40F6EB244C43B4EB002F01D2040202E040F6EB244C4317
:204AA000950405EB85056D00B5FBF4F41C801C88B4F5FA7F02DA4FF4FA7407E01C88B4F5BB
:204AC000FA5F02DD4FF4FA5400E01C881C801D885C68C4EB85245D6805EB64145C605C687F
:204AE000C4F38F245C805C88DC8100BFCCE7000038B504460B48012300220A2100900A48E0
:204B000007F036FF0948012300220A210090084807F02EFF0348007804490978084020703A
:204B200038BD00003E040020F01B00203F040020041C002000BFFEE710B5024804F058FD54
:204B400010BD0000A822002000B58BB0002006900790012008904CF2200001900020029007
:204B60004DF2E01003904FF6FF700490002005900120099001A9244804F09AFC20B14FF408
:204B8000A77122A011F0A6FA0120069000200790012008904FF460400190002002904CF20F
:204BA000E01003904FF6FF700490002005900120099001A9144804F07BFC20B140F26311D3
:204BC00012A011F087FA0220069000200790012008904FF240500190002002904FF6C070F0
:204BE00003904FF6FF70049001200590099001A9054804F05DFC20B14FF4BC7103A011F062
:204C000069FA0BB000BD0000A82200202E2E5C436F72655C5372635C63616E2E63000000EB
:204C20002DE9F04104460D46002700260DB9666B00E0A66B206800F5D87000EB051000688E
:204C400000F00400B060B06858B9206800F5D87000EB0510006840F2FF7101EA505030603D
:204C60000AE0206800F5D87000EB051000686FF0604101EAD0007060206800F5D87000EBE2
:204C80000510006800F00200F060206800F5D87000EB0510406800F00F0030613562206839
:204CA00000F5D87000EB05104068C0F30720F061206800F5D87000EB05108068307520680A
:204CC00000F5D87000EB05108068010A7175206800F5D87000EB05108068010CB175206856
:204CE00000F5D87000EB05108068000EF075206800F5D87000EB0510C0683076206800F50C
:204D0000D87000EB0510C068010A7176206800F5D87000EB0510C068010CB176206800F593
:204D2000D87000EB0510C068000EF0764DB920202168C8602068406920F00A00216848611B
:204D400008E02020216808612068406920F050002168486194F83C70222F01D0322F05D1E5
:204D60002068406920F40F4021684861EDB994F83C00422804D0622806D072280CD107E003
:204D8000122084F83C000BE0322084F83C0007E0522084F83C0003E0012084F83C0000BFA8
:204DA00000BF204604F0ACFE1CE094F83C00522804D0622806D072280CD107E0122084F8B2
:204DC0003C000BE0222084F83C0007E0422084F83C0003E0012084F83C0000BF00BF204611
:204DE00004F056FE0020BDE8F08100002DE9F34F83B0044660790B287EDB0021204611F073
:204E0000B3FA00906449009808700121204611F0ABFA8246604981F801A0009855286CD18D
:204E2000BAF1AA0FFBD12088000A88702078C8700221204611F098FA064657490E71112E02
:204E400003D0162E01D00C2E7ED10321204611F08BFA8046504880F805800521204611F0E9
:204E600083FA83460421204611F07EFA0BEB00201FFA80F94FEA19204749887181F8079035
:204E80000521204611F070FA0546A8EB0500022872D1617908F10900814217DA207C012876
:204EA00004D105F0B1FCE0600020207405F0ACFCE168411A0498814205D96179204611F0C8
:204EC0000FFA0120207405B0BDE8F08F0120207400270EE0B81DC1B2204611F045FA2F490B
:204EE000C8550846C15D07F108002B4A1154781C87B2AF42EEDB01E04CE047E0A81DC1B25C
:204F0000204611F031FA4FEA006BE81DC1B2204611F02AFA0BEB004B05F10800C1B2204640
:204F200011F022FA0BEB002B05F10900C1B2204611F01AFA0BEB0001019105F10801164860
:204F400000F038F9029000E01BE0DDE90110081A0CD12088114B4A46314600F09BFE08F160
:204F60000900C1B2204611F0BBF9ACE70121204611F0B6F90EE0FFE70121204611F0B0F9C9
:204F800008E00121204611F0ABF903E00121204611F0A6F900BF96E73F0D0020400C0020DD
:204FA00030B50A4600211CE00F4B5B6B14335B5CC57884686355C3785B1CDBB2C370847832
:204FC000A34201DB0023C37043795B1CDBB243718478A34203DD83784371012383714B1C57
:204FE000D9B29142E0DB30BDA82200202DE9F047824688461446002C5FDD2046E11704EBCF
:205000005171C910A4EBC1018FB237B90827E11704EB5171C1F3CF0907E02046E11704EBDB
:205020005171C910491C1FFA81F92548006BC0F800A000202249096BC8602149096B8860C0
:2050400000261CE008201E49096B086100250AE0082000FB065018F800101948006B14300A
:205060004155681C85B2082DF2DB0A21144804F0B7FD012801D10CF021FA701C86B2A9F13E
:205080000100B042DEDC0E48006B076100250AE0082000FB065018F800100948006B143092
:2050A0004155681C85B2BD42F2DB0A21044804F097FD012801D10CF001FABDE8F0870000C6
:2050C000A822002010B504462068406920F001002168486194F83C00122805D1206840695A
:2050E00020F40F402168486194F83C00422804D0522806D072280CD107E0222084F83C006D
:205100000BE0322084F83C0007E0622084F83C0003E0012084F83C0000BF00BF204604F0E5
:20512000B7FE002010BD000010B5014600224C69CB69552008600A68552A01D0002010BD2A
:20514000A82008600A6802F0A802A82A01D00020F5E70A4848614A69824201D00020EEE73A
:20516000074848614A69824201D00020E7E74C61CB614FF4004008600120E0E755050100FA
:205180002A8A020030B503460C460021002200BF09E0985C80EA1120C0B2054D35F810005E
:2051A00080EA0121521CA242F3D388B230BD00000C740108F0B502460B460025681E002191
:2051C0000FE0565C7040002407E0060E064F57F8265000026840661CB4B2042CF5DB4E1C49
:2051E000B1B29942EDDBF0BD0C76010800B585B000BF1848806940F00400164988610846B5
:20520000806900F00400009000BF00BF00BF0846806940F0080088610846806900F008005D
:20522000009000BF00BF08200190002002900120039001A9084805F047F94FF400400190FE
:20524000002002900120039001A9044805F03CF905B000BD00100240000C0140000801406E
:205260002DE9F84F04460D4616461F4600F0FAF8009000F0F7F8804600F0F4F88146009821
:20528000404504D1C84502D16A4880F800906A48007830B9674800786649487001206649A9
:2052A00008706448007863494978884238D0614840786049097801F00301604A515C884272
:2052C00009D1002060705E4908805E4908806068401C606024E0574840785649097801F056
:2052E0000301594A515C88420DD155480088401C5349088008460088042811DB012060702E
:20530000002008800CE04F480088401C4D490880084600880A2803DD0120607000200880DF
:205320004FF0020A4348007800F001004149497801F0010188422DD005F066FA43490968D7
:20534000401A4FF47A71B1FBF0F04149088005F05BFA3E49086017B94FF0010A00E0B246FC
:20536000607858B93B480078401C3A49087008460078504504DB0120A07001E00020A07076
:2053800035490888012111F02FFB208105F03CFA32490860324800682D490988C0EB8120CE
:2053A0002F49096801EB20202D49086008460068C0F3872020704FF0640B2548008814287B
:2053C00002DA4FF496700DE021480088282801DD642007E01E48008800EB80004FF4FA712A
:2053E000A1EB40001FFA80FB0BFB05F0642190FBF1F085B205F008FA18490968401AA8421D
:2054000011D90020A070022060700020207010490880134908600F4908700F490888002152
:2054200011F0E2FA20810348007802494870BDE8F88F0000C8030020CA030020DC7D0108C2
:20544000CC030020CE030020E07D0108D0030020D8030020DA03002022050020DC030020D5
:20546000D403002070B54FF40041084805F0BAF905462C460821064805F0B4F9064644EA44
:205480004600C4B204F0030070BD000000080140000C014000BF084A1268526A91B201EB20
:2054A000810292004FF47A7392FBF3F202800022014B1B685A627047D01C002010B54FF43B
:2054C000FA710948FFF792FC4FF4FA710748FFF78DFC4FF4FA710648FFF788FC4FF4FA71EC
:2054E0000448FFF783FC10BD90050020A4050020B8050020CC050020F0B58DB007460E464F
:20550000154618A103C9CDE90B0118A103C9CDE9070109AB002231460BA810F08FFF05AB68
:205520000022314607A810F089FF002405E009A8005D01A90855601CC4B2082CF7DB002461
:2055400007E005A8015D01AA04F108001154601CC4B2082CF5DB294601A801F03AFC0DB05A
:20556000F0BD000039FF6C063454333029270957FFFFFFFF30B502460B460021002400BFBB
:205580000EE0481C84B207E0505C155DA84201D1002030BD601C84B29C42F5DB481C81B2BE
:2055A0009942EEDB0120F4E731B581B0BDF80400ADF80000BDF9040044F6E61500FB05F1F6
:2055C000C913BDF9060000FB05F2D2130C4613466042C01AC01A00B2ADF8020000983CBD71
:2055E00070B504460AB9084670BD081B800290FBF2F086B2934202DD0D462846F4E706FB63
:2056000003F004EBA02085B22846EDE710B510223A493B480CF0D0FF044624B910223749CE
:205620003848FEF73CFA10223449354814300CF0C3FF04462CB91022304932481030FEF708
:205640002EFA20222D492E4828300CF0B5FF044624B9202229492C48FEF721FA10222749EB
:2056600027484C300CF0A8FF044624B9102223492648FEF714FA10222049214860300CF0D6
:205680009BFF044624B910221C492148FEF707FA10221A491A4874300CF08EFF044624B908
:2056A000102216491B48FEF7FAF908221349144888300CF081FF04462CB917480F490A68A0
:2056C000026049684160CC220C490D4894300CF073FF044624B9CC2208491048FEF7DFF9C1
:2056E000202206490E480CF067FF044624B9202202490C48FEF7D3F910BD0000F0150020A6
:2057000008FC01081C090020400B0020600B0020700B0020800B0020B0040020B40900204A
:205720006CFD01089001002010B50446594B0C220421204602F030FE401C28B9554B0C22AF
:205740000421204602F028FE534B20221221204602F022FE401C28B94F4B20221221204669
:2057600002F01AFE4C4800784C4908704C4B04223421204602F010FE401C28B9484B042298
:205780003421204602F008FE464B10223A21204602F002FE401C28B9424B10223A21204623
:2057A00002F0FAFD404B30224C21204602F0F4FD401C28B93C4B30224C21204602F0ECFDA9
:2057C00039480068401C384908600B4630224C2120460EF072FA401C28B9334B30224C2141
:2057E00020460EF06AFA314B1022EC21204602F0D3FD401C28B92D4B1022EC21204602F0B2
:20580000CBFD2B4B18227E21204602F0C5FD401C28B9274B18227E21204602F0BDFD254B4D
:2058200008229821204602F0B7FD401C28B9214B08229821204602F0AFFD1F4B1022A2218A
:20584000204602F0A9FD401C28B91B4B1022A221204602F0A1FD194B1022D621204602F0D7
:205860009BFD401C28B9154B1022D621204602F093FD134B2022B421204602F08DFD401C2F
:2058800028B90F4B2022B421204602F085FD002010BD0000C40B0020B00A0020B90100204C
:2058A000BA010020F00A0020000B0020300B002062150020BF010020300C0020200C00204E
:2058C000D00A00201CB52A492A4801F02DFD10222949284808300EF08DF91022264910314B
:2058E00024481C300EF086F920222449214830300EF080F9102222491E4854300EF07AF98C
:20590000102220491B4868300EF074F910221E4918487C300EF06EF908221C4915489030D0
:205920000EF068F9CC221A4912489C300EF062F92022184918480EF05DF918480078000603
:205940001649497800EB01401449897800EB01201249C9780844009004211048FFF72AFC80
:20596000019002226946034801F0B0FE1CBD0000FFFF010800FC01081C090020400B002044
:20598000600B0020700B0020800B0020B0040020B4090020900100206CFD0108E47D0108F8
:2059A00038B50546002410F047FB10F01FFB284601F066FB284601F01FFB1F480088009077
:2059C0009DF800200021284601F024FC401C28B99DF800200021284601F01CFC9DF8012032
:2059E0000121284601F016FC401C28B99DF801200121284601F00EFC02216846FFF7C2FB12
:205A0000044622120221284601F004FC401C20B922120221284601F0FDFBE2B2032128467D
:205A200001F0F8FB401C20B9E2B20321284601F0F1FB002038BD0000E87D010810B5094AAF
:205A40000949A2F10C00FFF757FD064B0C22042106480EF032F90648006820F400100449C9
:205A6000086010BDC40B0020BF0100202C0400208C01002070B50546002639480078C8B915
:205A8000002404E03748C0880644601C84B20A2CF8DB0A20B6FBF0F03349088004F0B4FECD
:205AA0003249086004F0B0FE3149086001202C4908704FE004F0A8FE2D490968401AB0F5C2
:205AC000FA7F03D904F0A0FE284908602868C0F3804000283ED104F097FE24490968401A0B
:205AE000B0F5FA6F36D9002404E01E48C0880644601C84B20A2CF8DB0A20B6FBF0F01A49B0
:205B0000088008460088B0F57A7F05DB0846008840F6B831884219DD286820F4802000F5BB
:205B2000802028600720134948800F4800888880084601F0CDFC00200F4908700F484089F3
:205B4000401C0E49488102200D49087004F05CFE0649086004F058FE0549086070BD0000A7
:205B600040000020501D0020380500204400002048000020880700209D030020300B002045
:205B8000BE01002010B5024804F004FA10BD0000D41D00203FB50446002520680090606804
:205BA0000190A0680290E06803900020206045F2555020602568854202D0002004B030BDFC
:205BC0000020206042F6AA2020602568854201D00020F3E70020206045F255506060052023
:205BE0000DF09EFC656845F25550854201D00020E4E74AF6AA20606005200DF091FC65689C
:205C00004AF6AA20854201D00020D7E74FF05530A060A568B5F1553F01D00020CEE74FF014
:205C2000AA30A060A568B5F1AA3F01D00020C5E74FF05530E060E568B5F1553F01D00020D5
:205C4000BCE74FF0AA30E060E568B5F1AA3F01D00020B3E7019860600298A0600398E06013
:205C6000009820600120A9E730B590F840500124AC40C56B6C60046863604468102C04D165
:205C80000468A2600468E16003E00468A1600468E26030BD2DE9F84F0746884615461C46C9
:205CA00005F0FF0A40F23171781A8F4273D00CDCA7F25160002801F04280CF280ED0D02892
:205CC0000DD0DF2841F0548064E00F287ED010287DD01F287CD02028F4D1A4E300BF41F274
:205CE0000C61681A8D4236D00BDCA5F58050A0F1100070B1B0F53E7F23D0B0F5806F45D1CE
:205D000023E0B0F5807F2CD0A0F5C850F93878BB2FE052462146FE48FDF7C1FEFC48407ACA
:205D2000FC49C8730020FC49887604F06DFDFA49C8610020F949087004F066FDF74948609D
:205D400025E001200CF01CF921E052462146F448FDF7A5FE1BE052462146F248FDF79FFE74
:205D600015E052462146EF480C30FDF798FE0EE00CE052462146ECA0FDF7C8FE28B9EC48FE
:205D8000007820F00100EA49087000E000BF00BFECE300E000BFB5F5545F7DD025DC43F223
:205DA0000511A5EB01008D427AD014DCA5F58050A0F10800B0B3B0F5017F38D0B0F5417F3B
:205DC0003BD0A0F5F850FA38002802E023E223E228E372D138E0A0F20310002871D0F82801
:205DE0007FD0B0F5007FF4D1AAE0B5F5824F67D00DDCA5F55850A0F1050000286FD0A0F275
:205E0000FB2000286CD0B0F5E16FE2D140E1A5F58440083800287DD0F8287CD0B0F5067F91
:205E2000D7D1CDE1FFE701200CF0AAF8F1E152462146C048FDF733FEEBE152462146BD4899
:205E40000C30FDF72CFEE4E1BB48007801280DD052462146B948FDF722FEB8480078C04313
:205E6000B7490870B5484078C0434870B3480078A8494873B148407888730B464FF4815208
:205E80000C214FF4E2600DF0B7FF0020AD49087004F0BAFCAB4901E095E001E04860B8E1F9
:205EA00052462146A0A0FDF731FE28B9A048007820F002009E490870ABE1A9E101E010E0E7
:205EC000F4E052462146A048FDF7E9FD9FA345F203320C2140F213700DF08EFF99E17BE03E
:205EE000AEE09B4B202212219A4802F055FA9848007B20709648407860709548007900F0FF
:205F00007F00A0709248C07EE070934B2022B421904801E0D1E0E3E002F03EFA012020718C
:205F20000F2060718C48007CA0710020E071234645F208420C2140F213700DF05DFF68E121
:205F4000207840B28249C876084690F91B000A2801DD0A20C8767E4890F91B0010F10A0FC0
:205F600002DAF6207A49C8766078794948700B462022122177480DF0A0FE207940B2764972
:205F80000874084690F91000002802DD0020087408E0714890F9100010F1140F02DAEC20B5
:205FA0006D4908746C4B2022B4216A480DF085FE01F0AEFE65A345F203320C2140F21370BC
:205FC0000DF01AFF25E1654B41F210520C214FF4E2600DF011FF1CE15246214660A0FDF7B1
:205FE00095FD60BB00205D498860C86009225E495EA0FDF78BFD80B158480068B0F57A7FFB
:2060000003D20020554908604860092257A15648FDF769FD002058490870504B1022D621C5
:206020004C480DF04AFE49A345F203320C2140F213700DF0E1FE0020364908834883E8E0B4
:206040004E48007818BB10224D494E480CF0B4FA10224B4910314B4814300CF0ADFA0C21A9
:206060004948FFF7A7F806464548C66203464FF492520C214FF4E2600DF0BEFE434B4FF44D
:20608000B9520C214FF4E2600DF0B6FE00BFC0E0524621463E48FDF702FD2CA345F2033280
:2060A0000C2140F213700DF0A7FEB2E0394A3A493A48007802F072F8ABE052462146364866
:2060C000FDF7EDFC00202C49087001F021FE1FA345F203320C2140F213700DF08DFE98E0B6
:2060E0001B4B202212211B4802F056F918480E30016821604168616000892081164B202262
:20610000B421144802F048F913481230016847E07C090020DC08002014030020EC01002001
:20612000A40900208C0900205245414459000000B0010020800A0020D8000020DA000020FB
:20614000DC000020DC010020B101002041434B00B00A00202C040020D00A0020200C002035
:20616000434C454152000000600B0020434C4541525F4F444F000000250400200202002018
:206180001C09002008FC0108B80B00205C090020A804002088040020B0040020B90400201C
:2061A000C4F80A104168C4F80E1000896082234645F220620C2140F213700DF01DFE28E0F7
:2061C000F648216801606168416021890181F448D4F80A100160D4F80E104160618A018186
:2061E000EE4B0E3B20221221EE480DF066FDEC4B123B2022B421EB480DF05FFDAFF2B40393
:2062000045F203320C2140F213700DF0F5FD00E000BF00BFBCE500BFB5F5445F5ED010DC1C
:20622000A5F58050A0F58670C8B1B0F5807F1CD0B0F57F7F20D0A0F5F050F43800286FD164
:2062400022E0A5F548500838F0B3FD2869D0B0F5FC7F67D0A0F2FD200028F0D1A7E05246BB
:206260002146D148FDF71BFCDAE052462146CE480C30FDF714FCD3E00020CC49087004F030
:20628000C3FACA494860CBE0C948007828BB1022C849C9480CF090F91022C6491031C64806
:2062A00014300CF089F90C21C448FEF783FF0646C048C66203464FF492520C214FF4E260CE
:2062C0000DF09AFDBE4B00E02DE04FF4B9520C214FF4E2600DF090FD00BFA1E0AF4B0E3B27
:2062E00020221221AF4802F057F8AC480E38007B2070AA480E3840786070A8480E3800793D
:2063000000F07F00A070A5480E38C07EE070234647F208320C2140F214700DF06DFD7FE0B8
:206320007DE02DE03AE0207840B29C490E39C876084690F91B000A2801DD0A20C87697489C
:206340000E3890F91B0010F10A0F03DAF62093490E39C876607891490E3948700B462022A1
:20636000122190480DF0A9FC01F0D2FCAFF2242347F203420C2140F214700DF03DFD4FE002
:2063800052462146AFF26020FDF7C0FB28B98D48007820F004008B49087041E08A4B41F277
:2063A00010520C214FF4E2600DF026FD38E052462146AFF25420FDF7A9FB78BB00208249C7
:2063C0008860C86009228149AFF26020FDF79EFB88B17D480068B0F57A7F03D200207A494E
:2063E000086048600922AFF27C217848FDF77BFB002077490870744B1022D62169480DF00C
:206400005CFCAFF2B82347F203420C2140F214700DF0F2FC00206F490883488300BF00BFB0
:2064200000BFB5E400BF42F22041681A8D4272D04DDCB5F5D05F6FD028DCB5F5A85F6CD0EB
:2064400015DCB5F5905F69D008DCB5F5805F79D0A5F588500838002875D1C5E0B5F5985F5D
:2064600072D0A5F5A05010380028F5D112E1A5F5B0501038002868D0F02867D0B0F5007F72
:2064800072D0A0F2F1200028E6D157E1B5F5F85F6BD00DDCB5F5D95F69D0B5F5E05F67D0A0
:2064A000A5F5E8501038002872D0F028D4D1B3E1B5F5005F6DD0B5F5045F6BD0A5F5085087
:2064C0001038002867D0B0F5807FC5D1F3E1B0F51D6F61D023DCB0F59C6F5ED00CDCE528D3
:2064E0007CD0A0F2E510002879D0A0F20310002876D0FA28B0D165E2A0F2E150002870D030
:20650000A0F2011000286DD0FF286CD0A0F206200028A1D104E3E1E12CE1CDE07FE041F2C9
:20652000E942811A904276D011DCB0F51E6F73D0B0F52E6F71D0B0F53E6F6FD0B0F5506FA3
:206540008AD187E315E0F6E395E0C4E0D5E0A1F2C31100297ED044297DD0B1F59A7F7BD038
:20656000B1F5157F90D1D4E3D6E066E1E6E310E12EE1194B082298210A4801F00DFF164B0C
:206580004AF208420C2140F215700DF035FCD4E32DE161E172E17AE1F4E27BE2BE0A002093
:2065A000E20A00202C040020980A0020E4010020020200201C09002008FC0108B80B00205F
:2065C0005C090020B0010020200C0020600B002025040020DC080020BF01002090E1AAE165
:2065E000D4E160E278E297E252462146FE48FDF756FAFD4B08229821FC480DF05EFBAFF2E2
:20660000B4434AF603120C214FF4E2600DF0F4FBFFF714FA91E332E3FBE203E30BE3F44816
:20662000007838BB1022F349F3480BF0C5FF1022F0491031F04814300BF0BEFF0C21EF4843
:20664000FEF7B8FD0646EB48C66203464FF492520C2102E028E339E34DE34FF4E2600DF091
:20666000CBFBE74B4FF4B9520C214FF4E2600DF0C3FB00BF61E31022E249DF484C300BF069
:206680009BFFE04B4AF210620C2140F215700DF0B3FB52E352462146DA48FDF700FA002094
:2066A000D9490870AFF25C534AF603120C214FF4E2600DF0A1FB40E31022D449CE48603038
:2066C0000BF07AFFD14B4AF210720C2140F215700DF092FB31E352462146CC48FDF7DFF90B
:2066E0000020C9490870AFF29C534AF603120C214FF4E2600DF080FB1FE31022C449BE489A
:2067000074300BF059FFC24B4AF610020C2140F215700DF071FB10E352462146BC48FDF7EC
:20672000BEF90020B8490870AFF2E0534AF603120C214FF4E2600DF05FFBFEE22078B54961
:20674000087008460078C043B3490870B148007878B1B248006820F48060B04908600846E5
:20676000006820F4805008600846006820F400600860E2E2AA4B202212219C4801F00CFEC6
:20678000A74B4AF220020C2140F215700DF034FBD3E252462146A248FDF781F9A04800782D
:2067A000A04908709E4B2022122190480DF085FA9B49487B0EF054FF01F0AAFAAFF27463C1
:2067C0004AF603120C2140F215700DF015FBB4E2954B10223A21854801F0DEFD924B4AF2BE
:2067E00010120C2140F215700DF006FBA5E2524621468D48FDF753F98B4B10223A217B48D4
:206800000DF05BFAAFF2BC634AF603120C2140F215700DF0F1FA90E2844B4AF230220C2149
:2068200040F215700DF0E8FA814B4AF610420C2140F215700DF0E0FA7FE220227D496E488A
:2068400028300BF0B9FE7B4B4AF220520C2140F215700DF0D1FA70E2234618227E216348CF
:2068600001F09AFD7448C08AE082734B4AF218320C2140F215700DF0BFFA5EE26F4B41F21D
:2068800001420C214FF4E2600DF0B6FA55E2524621465848FDF703F900205B490870AFF2B3
:2068A00054734AF603120C214FF4E2600DF0A4FAFFF7C4F841E2524621464E481030FDF7D1
:2068C000EEF8002050490870AFF280734AF603120C214FF4E2600DF08FFA2EE25246214671
:2068E0005448FDF7DCF8002047490870AFF2A4734AF603120C214FF4E2600DF07DFA1CE2DB
:20690000524621464EA0FDF701F998B9AFF2C4734AF603120C2140F215700DF06DFA0020B6
:206920000BF02EFB642003F089FC01200FF0AAFC04F08CF801E252462146AFF2DC70FDF736
:20694000E5F810BBFF2304220021284800F026FBFF2350224C21254800F020FB3A4926483B
:20696000083800F0E1FC3949394800F0DDFCAFF624034AF603120C2140F215700DF03CFA06
:2069800001200FF07FFC04F061F8D6E15246214630A0FDF7BBF8A0B90FF04EFB134800F0F6
:2069A0006FFBFEF78FFFAFF65C034AF603120C2140F215700DF020FA01200FF063FC04F023
:2069C00045F8BAE1524621462548FDF768F824480078C0432349087021484078C043487078
:2069E00000202149087041E0BF0100202C040020020200201C09002008FC0108B80B0020EB
:206A00005C090020600B002025040020700B0020800B0020D8000020D90000208C01002039
:206A2000B00A0020B9010020F00A0020000B0020300B0020400B002062150020B00100202F
:206A40005245534554000000FFFF0108FFF3010800F001085245434F564552590000000049
:206A6000DA000020DC000020DC01002003F0CCFEC1494860C1480078C1494873BF484078AF
:206A800088730B464FF481520C214FF4E2600DF0B3F952E1BB4B4AF604220C2140F21570B6
:206AA0000DF0AAF949E152462146B648801CFCF7F6FFB44B04223421B3480DF0FEF8AFF67E
:206AC00074134AF603120C214FF4E2600DF094F95520AC49C87030E1AA48C078552803D071
:206AE000A848C078AA2816D1AA20A649C87052462146A448FCF7D3FFA24B04223421A248C2
:206B00000DF0DBF8AFF6BC134AF603120C214FF4E2600DF071F910E120789C4908700CE1F0
:206B200000BF20790006617900EB0140A17900EB0120E179084421780906627801EB024174
:206B4000A27801EB0221E2781144401A461C20780006627800EB0240A27800EB0220E2787B
:206B60008118324604F10800FCF799FF4AF60830304482B223460C2140F215700DF03CF9DD
:206B800000BFDAE000BF20780006617800EB0140A17800EB0120E1784618207900066179C5
:206BA00000EB0140A17900EB0120E17900EB010BABEB060000F10109B6F1005F0FD94A461D
:206BC00004F108013046FCF76AFFAFF680234AF603120C2140F215700DF00EF917E06C48B5
:206BE000864214D906F2FF31304600F09DFB09F0FF0204F1080130460CF0FCFFAFF6B423D9
:206C00004AF603120C2140F215700DF0F5F800BF00BF604B41F210520C214FF4E2600DF0E4
:206C2000EBF88AE05C4B41F208620C214FF4E2600DF0E2F881E0594B2022B421524801F093
:206C4000ABFB564B4AF620520C2140F215700DF0D3F872E0524621465048FCF720FF4F4BFA
:206C60002022B42148480DF028F8AFF620334AF603120C2140F215700DF0BEF85DE0524697
:206C8000214647A0FCF742FF68B90FF0AFF93E4800F0B2F9AFF64C334AF603120C2140F2B1
:206CA00015700DF0A9F848E0524621463F48FCF7F6FE00203E490870AFF670334AF6031260
:206CC0000C2140F215700DF097F836E0524621463048FCF7E4FE2F4B1022D6212A480CF0D1
:206CE000ECFFAFF698334AF603120C2140F215700DF082F821E020222E492F480BF05CFC05
:206D00002C4B4BF620320C2140F215700DF074F813E0524621462748FCF7C1FE002024497C
:206D20000870AFF6D8334AF603120C214FF4E2600DF062F801E0FFE700BF00BF19E0A5F5F5
:206D40001450053820B1A0F5F840063828B900E000BF02201949087000E000BF00BF2B466B
:206D6000424640F25161164800940DF091F800E000BF00BFBDE8F88FDC010020DA000020AE
:206D8000DC080020BA0100202C040020D301002000300008200C0020F4010020D00A00203D
:206DA0004C4F4720434C454152000000B409002025040020900100206CFD01085D000020A4
:206DC000F0050020704700BF0100A0F10100FBD1704710B50246002016E0135C041D145DEE
:206DE00063400B54031DD35C00F10804145D6340041D0B55231DD35C0834145D634000F100
:206E000008040B55431CD8B20428E6DB10BD000010B503F0F9FC14490968401AB0F5FA7F70
:206E200021D303F0F1FC104908601048007858B90FA343F20902112140F212700CF0DCFF2D
:206E400001200A4908700EE00848007801280AD107A345F20902112140F213700CF0CCFFF2
:206E600000200249087010BDD0000020D400002048414E445348414B450000001FB54FF4E0
:206E80006040009011200190022003906946194803F01AFB4FF4E06000901120019002203C
:206EA00003906946144803F00FFB00224FF48071114803F0A3FC00224FF400710E4803F0D7
:206EC0009DFC00224FF480610B4803F097FC00224FF40051074803F091FC00224FF480414F
:206EE000044803F08BFC00224FF40041014803F085FC1FBD000C01400008014010B5002111
:206F00000D4804F05BFF04210B4804F057FF0821094804F053FF0021074804F0EFFB0421D9
:206F2000054804F0EBFB0821034804F0E7FB0C21014804F023FF10BD901C0020F8B50446C4
:206F4000002000906A460021204600F00DF90DF101020121204600F007F902216846FEF715
:206F600011F906466A460221204600F0FDF80DF101020321204600F0F7F89DF801009DF808
:206F8000001000EB012085B2A81B03D12046FEF7CBFBF8BD2046FEF703FDFAE72DE9F047A8
:206FA00080460C4616461F46301B00F0FF09002507E06019C1B23A46404600F02BF9681C1F
:206FC000C5B24D45F5DBBDE8F08700001FB50446022000900120019003906946054803F0B8
:206FE00073FA01220221034803F008FC204605F0F1FA1FBD000C014010B504461C4B302265
:207000004C2120460CF059FE401C28B9184B30224C2120460CF051FE164B1022EC21204634
:207020000CF04BFE401C28B9124B1022EC2120460CF043FE104B1022D62120460CF03DFE6E
:20704000401C28B90C4B1022D62120460CF035FE0A4B1022A22120460CF02FFE401C28B9C8
:20706000064B1022A22120460CF027FE10BD0000000B0020300B0020200C0020300C002048
:2070800010B50446314B0C22042120460CF015FE401C28B92D4B0C22042120460CF00DFE28
:2070A0002B4B0822982120460CF007FE401C28B9274B0822982120460CF0FFFD254B20226E
:2070C000122120460CF0F9FD401C28B9214B2022122120460CF0F1FD1F4B2022B4212046D0
:2070E0000CF0EBFD401C28B91B4B2022B42120460CF0E3FD194B10223A2120460CF0DDFD83
:20710000401C28B9154B10223A2120460CF0D5FD134B0422342120460CF0CFFD401C28B9CD
:207120000F4B0422342120460CF0C7FD0D4B18227E2120460CF0C1FD401C28B9094B182238
:207140007E2120460CF0B9FD10BD0000C40B0020BF010020B00A0020D00A0020F00A0020EE
:20716000BA010020621500202DE9F04106460F4615460024304605F0A0FAA021304605F005
:20718000E1FA00BF00BF601C84B240F6B830844203DD4FF0FF30BDE8F081304605F0FAF93E
:2071A0000028F0D13946304605F0CCFA002400BF601C84B240F6B830844202DD4FF0FF3070
:2071C000E9E7304605F0E6F90028F1D1304605F074FAA121304605F0B5FA002400BF601C97
:2071E00084B240F6B830844202DD4FF0FF30D2E7304605F0CFF90028F1D12946304605F078
:2072000006FA304605F036FA304605F076FA0020C1E700002DE9F04106460F4615460024C9
:2072200000220221294803F0E9FA304605F045FAA021304605F086FA00BF00BF601C84B23C
:2072400040F6B830844203DD4FF0FF30BDE8F081304605F09FF90028F0D13946304605F010
:2072600071FA002400BF601C84B240F6B830844202DD4FF0FF30E9E7304605F08BF90028F6
:20728000F1D12946304605F05DFA002400BF601C84B240F6B830844202DD4FF0FF30D5E779
:2072A000304605F077F90028F1D1304605F025FA0A2002F0C3FF01220221044803F09EFA84
:2072C000034803F0CFFA0020C0E70000000C0140F0070020F8B50E480468001D0568200E55
:2072E0008DF80000200C8DF80100200A8DF80200E0B28DF8030004216846FDF75BFF06461F
:20730000701B02D1FEF782F901E0FEF7DBFAF8BD00FC010810B50446207818B9FEF7D2FA01
:207320000120207010BD000038B504460D4600200C49086008468460281B401C800AC860E5
:2073400003F04AF800BF34200749C86000BF6946044802F087FF02F0DDFF642002F06EFF8A
:2073600038BD0000E01500200020024010B504220E490F480BF020F90446A4B904220B49D3
:207380000CA0FCF7C3FB70B928220849084808300BF012F9044634B9282204490748FCF72E
:2073A0007EFB002010BD0120FCE70000F015002000E80108464C414700000000900B002078
:2073C00010B54FF4805003F071F810BD10B5042003F06CF810BD00001FB54FF46040009058
:2073E0000220019003906946064803F06DF84FF4E06000900220019003906946024803F0AD
:2074000063F81FBD000C01400008014010B50021104804F0B3FC04210E4804F0AFFC08217B
:207420000C4804F0ABFC0C210A4804F0A7FC0021084804F04DF90421064804F049F90821CA
:20744000044804F045F90C21024804F041F90AF023FE10BD901C00202DE9F04107460C466F
:20746000207860BB384600F057F846B2701C48B11448402101FB06054022394628460CF010
:20748000EFFB1AE00F49491E0F48FFF74DFFF0220C4940310C4800F019F90C490948FFF7E6
:2074A00043FFF0220849074800F010F9074D3F3D4022394628460CF0D3FB01202070BDE8A0
:2074C000F081000000F0010800EC0108FFF3010810B504460B480068A0600B484068E0604D
:2074E00020220A4904F11000FCF7D9FA0848016821634068606307480168A1634068E063DD
:2075000010BD00008C010020000B0020DC080020F4010020DE00002010B50246002116E08B
:207520000F4C04EB811003884FF6FF7083420CD111B90120108006E04020C0EB8110084C3E
:20754000035B581C1080084610BD481C41B21029E6DB04480388581C10804FF0FF30F3E73A
:2075600000F00108C0F301080021074AD1610749096941F00401054A11611146096941F0FF
:20758000400111617047000020070020002002400021074AD1610749096941F00201054AEF
:2075A000116111464861096941F040011161704720070020002002400022054BDA61054AA7
:2075C000126942F00102034B1A61018070470000200700200020024000201E49C96801F0A8
:2075E000100139B11C49C96941F002011A4AD16140F010001749C96801F0040139B116491F
:20760000C96941F00101144AD16140F004001149C96901F0010169B10F49C96941F00401E8
:207620000D4AD16100BF0B49C96921F00101094AD16100BF00BF40F20111884206D1054933
:20764000C96921F00101034AD16101E00149C86000BF7047002002402007002070B5044685
:2076600003F0D2F8054609E0601C38B124B103F0CBF8401BA04201D9032070BD1248C06840
:2076800000F001000028EFD10F48C06800F0200020B100BF20200C49C86000BF0A48C068FC
:2076A00000F0100048B90848C06900F0010020B90548C06800F0040018B1FFF78DFF0120B1
:2076C000DBE70020D9E70000002002402DE9F04104460E461746002502F07EFE00BF0FE023
:2076E00056F825C0624600232146022002F01CFE08B9241D03E002F00DFEBDE8F0816D1C76
:20770000BD4202D203488442EAD902F003FE00BFF3E70000FBFF010802200549087000202B
:207720000449088048800449088048807047000030000020280000202C0000200120014909
:2077400008707047300000202DE9FF4705460E4617464FF0000A0CF09FF903900398FDF753
:2077600023FF029039B202980AF0A4FA0090714800990160B0F900006F490968C1EB8020D7
:207780006D49096801EBA0206B49086008460068801200B2694908806648B0F902006849BC
:2077A0000968C1EB80206649096801EBA0206449086008460068801200B262490880624854
:2077C000007C002849D161480078042845D16048408840F6EC01884210DA5E4805605E4890
:2077E000006810F1040F05DA5B480068001D5A49086042E00020584908603EE0544840882E
:2078000040F6BE11884221DA51484088A0F6EC0000EB800040F21A41081A50490860084652
:207820000068854201DA284601E04C4800684949086049480068801E4749086008460068B4
:2078400010F5D27F19DA4648086016E00020414908604348404908600FE03E4805603E4805
:20786000006810F1040F05DA3B480068001D3A49086002E00020384908603A4A2F48B0F92B
:2078800000103448008800B20AF0D4F9044636480068C0EB44203449096801EBE0003249E7
:2078A000086032484088B7214843C0F3CF1947F698107043B9F57A7F02DA4FF47A7100E0F7
:2078C000494690FBF1FA284800680AEB602447F69810844200DD00E02046044620B22449FB
:2078E0000880244A1748B0F900101B48008800B20AF0A0F9804620480068C0EB48201E493A
:20790000096801EBE0001C49086008460068401200B21749488008460AF084FE14480068ED
:2079200000900AF0A5FE019001980BF009FEBDE8FF870000280000200C000020200000200F
:207940001000002022000020C8070020DE000020501D0020040000200800002024000020AB
:207960005CFEFFFF4406002018000020F00A00202C000020680600201C00002004F030FFBA
:2079800009F0E4FD09F084FE62B60020124981F83C0009F093FD72B609F05AFE0AF084FBCF
:2079A000FFF76CFA00200D4908600846006820F4005000F5005008600DE0084B41F204123D
:2079C0000C214FF4E2600CF017FAC8200BF098FD034802F047FFF0E7A82200208C0100207F
:2079E000F007002070B505460E46049CAC4208DAFF2E01D100210DE0281B7043C0F58061A3
:207A000008E0944202DA4FF4806103E0A01A5843C0F58061002901DC002000E0084601463F
:207A200088B270BD87B0014600220868009048680190C86803903D4881423AD04FF0553025
:207A400008600A68B2F1553F02D0002007B070474FF0AA3008600A68B2F1AA3F01D0002045
:207A6000F4E74FF0553048604A68B2F1553F01D00020EBE74FF0AA3048604A68B2F1AA3F14
:207A800001D00020E2E745F25550C860CA6890B245F25553984201D00020D7E74AF6AA2042
:207AA000C860CA6890B24AF6AA23984235D00020CCE700986FF30B0000F2555008600A68F5
:207AC000C2F30B0040F25553984201D00020BDE700986FF30B0000F6AA2008600A68C2F349
:207AE0000B0040F6AA23984201D00020AEE7039820F00700C01DC860CA6802F00700072807
:207B000001D00020A2E7039820F00700C860CA6802F0070008B1002098E7009808600198F5
:207B200048600398C860012090E70000001401402DE9F04104460E4615462948007801289B
:207B400012D1284801780078401C264A1070264820F8116010460078322810DB0020204902
:207B60000870114608700AE032221F49304609F01BFF643087B22088B84200DD00BF2888D4
:207B8000C0F3C03050BB208840F2DC51884203DC02F03AFE1549086002F036FE13490968A4
:207BA000401A42F21071884218D9286820F4004000F50040286001200D494880208888806B
:207BC0000846FFF785FC00200A4908700A488088401C09498880022008490870BDE8F081E4
:207BE00077040020780400202C1C00207C040020880700209D030020300B0020BE0100209D
:207C0000B1F5967F03DA0122044B1A7002E00022024B1A7001F164020280704776040020CA
:207C200010B502460020B2F5FA7F01DC01200EE0B2F5E16F01DB084609E040F2145393FBDA
:207C4000F1F4A2F5FA7393FBF4F35B1CD8B210BD10B50446207800284DD12749087002F031
:207C6000D3FD25494860608840F2AA71884236D120792249087060794870A0798870E079A1
:207C8000C870617A207A01EB00201C4988801C48807EEE2811D10846808820B94FF6FF7081
:207CA0001849886009E0154880884EF6602191FBF0F0144988600020C870A07A0F498871F4
:207CC000E07AC87108468079C0F3401018B100200D4908700DE001200B49087009E0608865
:207CE00040F2AB71884204D1084861680160A16841600120207010BDA0040020DC0700202E
:207D0000B00A0020EC030020B90400208404002010B500BF2A480078052803DA05202849E7
:207D2000087006E026480078182802DD18202449087023480078401E43F2C82191FBF0F0F8
:207D400084B218211F48FCF766FD00200BE000FB04F10A2291FBF2F101F5FA71194A22F883
:207D60001010411CC8B216490978491E8142EEDC4FF4E16112480078401E124A22F81010ED
:207D800000BF00BF1048807900EB4000C0000A2190FBF1F00D4908700B48C07948700A482E
:207DA000007B0949C97E084464380849487104484078887002488078C87000BF10BD0000BB
:207DC000B0040020BA040020B00A00208C04002010B502F019FD40F6B831884206D9C148C9
:207DE0000078F02802D1C049C87710BDBF48FFF72FFFBF48007858B902F006FDBC494968A5
:207E0000401A40F6B831884202D90120B8490870B4480078202823D040285CD080285BD094
:207E2000F02875D1AF480078AF49C87700BF02F0EBFCB0490968401AC82809D90120AE49F8
:207E40000870084600F086F902F0DEFCA949086000BFA748007810B92020A24908703DE117
:207E6000A048007800F0E0009F49C87700BFA3480078052800DB16E002F0C6FCA04909687D
:207E8000401AC8280ED99F4A9F49A048007800F085F902F0B9FC9A49086098480078401C6C
:207EA0009649087000BF00BF9948007890B198480078032803D140208A4908700AE094488B
:207EC0000078042803D092480078082802D180208449087002E100BF8D480078082805D1FC
:207EE0008549087000204880888054E088480078032829D140207B49087003207E490870AD
:207F000083484078012804DA82480088488017E0E3E07F4840787C490978884208DD7A48CD
:207F20000078401E7B4931F810007349488007E077484078401E774931F810006E494880B6
:207F400000206D49888026E071480078042822D18020644908700420674908706C48407870
:207F600069494978884204DA67484078624988800EE06748407864498978884204DD624874
:207F800080785D49888003E0614840785A49888000205949488056480078012803D1F0209F
:207FA0005149C87725E04F480078402812D1564A1178594A5278642302FB03F0FFF730FE58
:207FC00000F01F004749097801F0E00108444649C8770EE04348007880280AD14148007820
:207FE00000F0E0004C49497801F01F0108443E49C87700BF02F008FC48490968401AB0F582
:208000007A7F39D94248007808280FD144480078052807DA384800F09DF841480078401CCF
:208020003F49087000203F49087021E03D480078012808DA3C4800F07DF83A480078401CD8
:208040003849087011E03748007805280DDA2A4800F080F833480078401C324908700846C1
:208060000078052801DB0020087000202C49087002F0CAFB2949086000BF00BF022402F0B3
:20808000C3FB2A490968401AB0F57A7F23D91F480078012809D100BF1A4A1B49204600F08B
:2080A0007DF800202249087011E01848007870B900241F480078052809DA124A1249204626
:2080C00000F06CF81A480078401C1949087002F09BFB1649086000BF00E000BF00BF00BF11
:2080E00083E60000B8040020DC08002094040020A0040020EC040020E6070020F404002086
:20810000F004002088040020B0040020B9040020A8040020BA040020DC070020F804002025
:20812000FD040020FC0400208C04002000050020040500201CB5044600200090019020681C
:208140000090606801900822694640F2AC70FCF74DFF1CBD1CB50446002000900190207803
:208160008DF80000608800128DF80100A0788DF80200A08800128DF8030020798DF8040077
:2081800000208DF805008DF806008DF807000822694640F2AD70FCF729FF1CBD7FB5064682
:2081A0000C461546002000900190029003908DF800602088ADF80100A0788DF80300287839
:2081C0008DF804006B4645F210520C2140F213700BF012FE7FBD000038B5044601234FF405
:2081E0007A720A210248009404F0C2FB38BD0000181C002030B503460024002204E033F80D
:2082000012502C44551CAAB28A42F8DBB4FBF1F5A8B230BD70B505462C480078012811D1DD
:2082200000202A49087002F0EFFAB0F5E16F05D902F0EAFAC8302649088003E04FF4FA6040
:208240002349088002F0E0FA2149098888423BD920480078012837D11F48007858B11F4825
:208260000088C82807DC40F2C27085420CDD40F63E00854208DA00201949C8720A2219A1D0
:208280001B48FBF730FC1CE001201549C872002415E0184830F81400A8420EDB0A2216A13D
:2082A0001348FBF720FC1748015D1148203880F8271000200749087070BD601CC4B2092CFC
:2082C000E7DB00200349087000BFF5E7820400208004002002020020D4010020D001002009
:2082E000C80700205144303037482E20333600003C090020EA7D010854544B5A3031394167
:2083000033360000FC7D010810B502460B460020002107E032F81140844201DD32F8110092
:208320004C1CA1B29942F5DB10BD10B502460B464FF6FF70002107E032F81140844201DAD4
:2083400032F811004C1CA1B29942F5DB10BD00000246002108E0064830F81100904201DC28
:2083600008467047481CC1B2C829F4DB0020F8E7048001080246002108E0064830F81100FD
:20838000904201DC08467047481CC1B2BF29F4DB0020F8E7948101082DE9F84F82460D4606
:2083A00014461F4600260EE01C488219A819C1B25046FEF7D9FE401C18B94FF0FF30BDE815
:2083C000F88F701CC6B2A642EEDB21461348FCF7D9FE81462819C1B26A465046FEF7C4FE5D
:2083E0002819401CC1B20DF101025046FEF7BCFE9DF801009DF8001000EB01201FFA80F84F
:20840000B8EB090006D1224604493846FBF747FB0020D4E74FF0FF30D1E70000F01A002047
:208420002DE9FC5F804689464FF0000A002549464046FFF7DFFE8346002407E038F81400C8
:20844000ABEB000505FB05AA601C84B24C45F5DB5046FBF728FD06460F46304639460EF07E
:208460009DFACDE90001FBF769FD05462846BDE8FC9F0000F8B5044600260020009000BFD1
:2084800094F82400012801D10220F8BD012084F8240000BF2046FBF71DFF0646002E62D1B9
:2084A000A06A20F4885040F00200A062022002F0EFFA30490968B1FBF0F04000009002E06D
:2084C0000098401E009000980028F9D12046FBF769FF2068806840F008002168886002F0C1
:2084E00093F9054611E002F08FF9401B0A280CD9A06A20F0020040F01000A06200BF00208B
:2085000084F8240000BF0120BFE72068806800F008000028E7D12068806840F004002168C0
:20852000886002F071F9054611E002F06DF9401B0A280CD9A06A20F0020040F01000A06293
:2085400000BF002084F8240000BF01209DE72068806800F004000028E7D1A06A20F00200D8
:2085600040F00100A06200BF002084F8240000BF30468AE70000002038B50246002300200B
:208580000090906800B100BF00BF92F82400012801D1022038BD012082F8240000BF9068EE
:2085A00090B94868012809D11068806B6FF315000C6840EAC4301468A06338E0906A40F092
:2085C00020009062012332E00C694868A0421ED84C680869001BC0F1030000EB80041F20B4
:2085E000A04040F440141068806BA0434D680C69641BC4F1030404EB84050C68AC400D8AF9
:208600006D1E44EA055420431468A0630FE04C680869001BC0F1030000EB80041F20A040F5
:2086200040F440141068806BA0431468A0631068806800F0010040B91068806847F2010405
:20864000A043CC6920431468A060886901280FD1C869B0F5E04F06D11068406840F4806019
:208660001468606004E0906A40F0200090620123486901280DD1886930B91068406840F494
:2086800080501468606004E0906A40F020009062012308680A2812D31068C0680C780A3C99
:2086A00004EB44050724AC40A0430D780A3D05EB45058C68AC4020431468E0600FE010681C
:2086C00000690C7804EB44050724AC40A0430D7805EB45058C68AC4020431468206108680C
:2086E000102802D00868112805D11068806840F400001468A0604868012806D002280DD02B
:20870000032814D004281BD11BE0106840696FF30B00CC682043146860611BE01068806979
:208720006FF30B00CC6820431468A06112E01068C0696FF30B00CC6820431468E06109E07B
:2087400000BF1068006A6FF30B00CC6820431468206200BF00BF0868102802D008681128D5
:2087600027D1174C1068A0421ED11068806800F40000F0B91068806840F400001468A06048
:208780000868102815D10F4800680F4CB0FBF4F000EB80004000009002E00098401E0090FF
:2087A00000980028F9D104E0906A40F020009062012300BF002082F8240000BF1846E9E682
:2087C000002401400000002040420F0010B504460121204600F044F84FF6FF7101EA001010
:2087E0001A4948800221204600F03AF84FF6FF7101EA0010154988800321204600F030F8EB
:208800004FF6FF7101EA001010490880104800880988401A00B20F4908800D4840880B49F9
:208820004988401A00B20B4948800948808807498988401A00B2074988800749054809F08B
:2088400081FA01200549087010BD000014050020260500202C050020320500202005002078
:208860000246002001290FD0022909D0032904D0042908D11368986C09E01368586C06E0F0
:208880001368186C03E000BF1368D86B00BF00BF7047000070B50446002500BF94F8240041
:2088A000012801D1022070BD012084F8240000BF2046FBF777FD0546002D5BD1A06A42F240
:2088C0000101884340F48050A0622E492068884208D12D48006800F4702008B9012002E0FE
:2088E000002000E0012020B1A06A20F48010A06203E0A06A40F48010A062A06A00F4807035
:2089000008B90020E06200BF002084F8240000BF401F216808602068406840F0800021683D
:2089200048602068406800F4806010BB2068806800F4E040B0F5E04F15D1124920688842D5
:2089400008D11148006800F4702008B9012002E0002000E0012030B12068806840F402107D
:20896000216888600BE02068806840F400402168886004E000BF002084F8240000BF2846B6
:2089800091E70000002801400424014038B5024600230020009000BF92F82400012801D11D
:2089A000022038BD012082F8240000BF4868072812D21068406B0C79641E04EB84051F247A
:2089C000AC40A0430D796D1E05EB85050C68AC4020431468606327E048680D2812D21068F3
:2089E000006B0C79E41F04EB84051F24AC40A0430D79ED1F05EB85050C68AC4020431468AF
:208A0000206311E01068C06A0C790D3C04EB84051F24AC40A0430D790D3D05EB85050C682A
:208A2000AC4020431468E06208680A2812D31068C0680C780A3C04EB44050724AC40A04306
:208A40000D780A3D05EB45058C68AC4020431468E0600FE0106800690C7804EB440507245A
:208A6000AC40A0430D7805EB45058C68AC402043146820610868102802D00868112827D10D
:208A8000174C1068A0421ED11068806800F40000F0B91068806840F400001468A0600868AD
:208AA000102815D10F4800680F4CB0FBF4F000EB80004000009002E00098401E00900098B4
:208AC0000028F9D104E0906A40F020009062012300BF002082F8240000BF184661E700007E
:208AE000002401400000002040420F0070B50646CD480068401CCC49086008460068B0F53E
:208B0000967F01D900200860C8480078012805D14120C74948758875C87599E0C548C07A2F
:208B2000012808D1C4480078012804D10020C249087008F089FBC1480088C149096808443A
:208B4000BF490860BD488088BE4909680844BD490860BA48C089BC4909680844BA490860EE
:208B6000BA480088401CB94908800846008840F6B83188426CDBAF48C07A012822D1B0483A
:208B80000068B0FBF1F085B22846FFF7F3FBA8494875AC48006840F6B831B0FBF1F085B26C
:208BA0002846FFF7E7FBA2498875A748006840F6B831B0FBF1F085B22846FFF7DBFB9C492F
:208BC000C8753CE09E48006840F6B831B0FBF1F085B22846FFF7BCFB95494875994800680D
:208BE00040F6B831B0FBF1F085B22846FFF7B0FB8F4988759648007801280ED10846407D46
:208C0000944908709048006840F6B831B0FBF1F09149088000208E4908708B48006840F6D2
:208C2000B831B0FBF1F08C490988081A00EB400080018849097801EBA0207D49C87500206A
:208C4000824908807E4908607E4908607E4908607A48408881490968C1EB80207F490968EA
:208C600001EB60207D49086008460068801244F2CE714843C0F38F206D49C8800846C0881C
:208C80000989C91101EBC10202EB011108446849C8807348007803280BD10846C088A0F510
:208CA000F850A43840F27A514843C0F38F206049C8806C48407C01281FD101F0A5FDB0F5F4
:208CC000FA6F1AD35A48C0880A2190FBF1F06549488208464069498A08446249486108468D
:208CE0008069401C88610846806943F69821884203D300205B49886148744E48C07A01281B
:208D000015D14E48C08858490988401A49F6192148438412002C01DC002006E049F61920E2
:208D2000844201DB401E00E02046044613E04348C0884D490988401A4CF250314843C4123C
:208D4000002C01DC002005E04CF25030844200DB00E02046044645480068C0EB8420434946
:208D6000096801EB60204149086008460068C0F38F202F4908813E48C078AA2811D02F4823
:208D800000893C49C98A401A642148433849897890FBF1F4002C01DC002000E0204604465D
:208DA00007E0344AD18A254A1089314A0BF0C4FF044631490C8031480078D8B91F48808970
:208DC0002F490988441A002C01DC002000E0204604462C480068C0EB84202A49096801EB78
:208DE00020202849086008460068C0F38F202249488002E000202049488010484089224950
:208E00000968C1EB80202049096801EB60201E49086008460068C0F38F201C49088007492B
:208E2000488809F06FF870BD3C05002002020020DC080020C807002064050020501D002047
:208E4000500500204C050020540500204805002058050020590500205A0500204005002067
:208E6000FC010020340300203805002044050020BA01002062150020220500207604002065
:208E8000740400205C05002060050020000200207047704710B504462068406800F0200055
:208EA00020282FD12068006800F00200022829D1A06A00F0100018B9A06A40F40070A062D9
:208EC0002068806800F46020B0F5602F13D1E06888B92068406820F0200021684860A06A72
:208EE00020F48070A062A06A00F4805018B9A06A40F00100A0622046FFF7F8FD6FF01200CE
:208F0000216808602068406800F0800080283BD12068006800F00400042835D1A06A00F0FC
:208F2000100018B9A06A40F40050A0622068806800F4E040B0F5E04F0DD02068406800F467
:208F40008060D0B92068806800F46020B0F5602F13D1E06888B92068406820F080002168DA
:208F60004860A06A20F48050A062A06A00F4807018B9A06A40F00100A0622046FFF726FCDF
:208F80006FF00C00216808602068406800F0400040280FD12068006800F0010050B1A06AE1
:208FA00040F48030A062204600F0A8F86FF001002168086010BD00002DE9F04104460027FF
:208FC00000250026A84614B90120BDE8F081A06810B1606900B100BFA06A30B90020E062FD
:208FE00084F82400204600F08BF82046FBF772F90746A06A00F01000002873D1002F71D101
:20900000A06A20F4885040F00200A062E16960680843E16840EA41000643A068B0F5807F20
:2090200002D0A068012802D14FF4807000E0002005436069012811D1E06838B9A069401E6B
:209040004FF4006141EA4030054307E0A06A40F02000A062E06A40F00100E0622068406859
:2090600020F469402843216848602068806821490840304321688860A068B0F5807F02D013
:20908000A068012802D14FF4807000E00020B0F5807F03D1208A401E4FEA00582068C06AD6
:2090A00020F4700040EA08002168C8622068806811490840B04208D10020E062A06A20F0EE
:2090C000020040F00100A06211E0A06A20F0020040F01000A062E06A40F00100E062012727
:2090E00005E0FFE7A06A40F01000A062012738466BE70000FDF7E1FFFE0E1FFF70470000AC
:2091000010B586B004463249206888423CD100BF3048806940F400702E49886108468069D5
:2091200000F40070019000BF00BF1F2002900320039002A9284801F0C7F9A02002900320F4
:20914000039002A9254801F0BFF9254825490860002048600021234881608021C160490038
:20916000016189004161202181610021C16100F0DFFF20B140F217111BA00CF0ABFF00BFE3
:2091800018482062446221E01C49206888421DD100BF1048806940F480600E4988610846FF
:2091A000806900F48060019000BF00BF0E2002900320039002A9094801F086F90122114687
:2091C000122001F0F0FB122001F0E0FB06B010BD00240140001002400010014000080140AF
:2091E00008000240D41D00202E2E5C436F72655C5372635C6164632E6300000000280140D1
:2092000070B50446002500BF94F82400012801D1022070BD012084F8240000BF2046FBF729
:20922000C1F80546002D77D1A06A40F20121884340F48070A0623C492068884208D13B4833
:20924000006800F4702008B9012002E0002000E0012078B1A06A20F48010A0622068406834
:2092600000F4806000B3A06A20F4005040F48050A06219E0A06A40F48010A0622B49091F8E
:209280002068884203D028492068884204D12748006800F4806000E0002028B1A06A20F46F
:2092A000005040F48050A062A06A00F4805020B1E06A20F00600E06201E00020E06200BF15
:2092C000002084F8240000BFC01E216808602068806800F46020B0F5602F16D1124920685E
:2092E000884208D11148006800F4702008B9012002E0002000E0012038B12068806840F414
:20930000A000216888600CE006E02068806840F480102168886004E000BF002084F8240062
:2093200000BF284675E7000000280140042401402DE9F04104460D46164600275749206843
:20934000884203D056492068884205D15348001D006800F4702000E0002000287ED100BFCF
:2093600094F82400012802D10220BDE8F081012084F8240000BF2046FBF714F80746002FA9
:209380006DD1A06A40F60161884340F48070A06243492068884209D14048001D006800F443
:2093A000702008B9012002E0002000E0012078B1A06A20F48010A0622068406800F480605B
:2093C00000B3A06A20F4005040F48050A06219E0A06A40F48010A06230492068884203D0FF
:2093E0002F492068884205D12C48001D006800F4806000E0002028B1A06A20F4005040F485
:209400008050A062A06A00F4805020B1E06A20F00600E06201E00020E06200BF002084F89B
:20942000240000BF1F48216A88621F48216AC8621E48216A08636FF002002168086020681B
:20944000806840F4807021688860226802F14C0133462A46206A00F0A3FE01E01AE014E0F2
:209460002068806800F46020B0F5602F06D12068806840F4A000216888600CE020688068EC
:2094800040F480102168886005E000BF002084F8240000E00127384667E7000000240140FA
:2094A0000028014027430008974300087943000830B5024600230C7D012000FA04F31068C8
:2094C000D0F8000220F47C5001254C6A45EA042420431468C4F800021068D0F81C029843D9
:2094E0001468C4F81C02C869E8B91068D0F80C0298431468C4F80C02888880B28C8940EA54
:209500000444106800F510704D6940F83540088880B20C8940EA0444106800F510704D6947
:2095200000EBC5004460C86901281DD11068D0F80C0218431468C4F80C02888880B20C88CA
:2095400040EA0444106800F510704D6940F83540888980B20C8940EA0444106800F5107012
:209560004D6900EBC5004460886938B91068D0F8040298431468C4F8040206E01068D0F87A
:20958000040218431468C4F80402086938B91068D0F8140298431468C4F8140206E01068ED
:2095A000D0F8140218431468C4F81402086A012806D11068D0F81C0218431468C4F81C02A3
:2095C0001068D0F8000220F001001468C4F80002002030BD0168496941F002010268516186
:2095E0000168496941F0100102685161704700002DE9F0410446002500260027A8462068C2
:20960000C068C0F3001520684069C0F3C0062DB126B148F4007810202168C8602068006975
:20962000C0F3001520684069C0F380162DB126B148F480681020216808612068406900F0CC
:20964000010000283BD0206880687A490840884201D1012000E00020054620688068764924
:209660000840884201D1012000E0002006462068806872490840884201D1012000E0002069
:2096800007460DB906B9D7B120688068C0F3400520688068C0F340262068806800F0010717
:2096A0000DB906B91FB12046FBF70CFD01E048F40068206880686249084321688860206810
:2096C000C06800F0030520684069C0F3400625B11EB100212046FBF7A3FA2068006900F0A4
:2096E000030520684069C0F3001625B11EB101212046FBF795FA206C40EA080020642068F0
:20970000806900F0010520684069C0F3002620684069C0F3C0372DB126B11FB1206C40F044
:209720000100206420688069C0F3400520684069C0F3402620684069C0F3C0372DB126B161
:209740001FB1206C40F00200206420688069C0F3800520684069C0F3802620684069C0F3E0
:20976000C0372DB126B11FB1206C40F0040020642068806900F0700008B9012000E0002076
:20978000054620684069C0F3C02620684069C0F3C03795BB8EB387B32068806900F0700538
:2097A000402D1BD006DC102D09D0202D0CD0302D24D10EE0502D16D0602D1FD118E0206C8C
:2097C00040F0080020641AE0206C40F01000206415E0206C40F02000206410E0206C40F082
:2097E000400020640BE0206C40F08000206406E0206C40F48070206401E007E000BF00BF9A
:209800002068806920F0700021688861206C78B1042021684860012084F83C0020684069D1
:2098200048F65B718843216848612046FFF7D2FEBDE8F081010000040001000800000110C0
:20984000090501002DE9F041044600270026002514B90120BDE8F08194F83C0028B9002029
:2098600084F83D00204600F0A5F8022084F83C002068006820F0020021680860206800687F
:2098800040F001002168086000F0BEFF06460EE000F0BAFF801B0A2809D9032084F83C008C
:2098A00000BF002084F83D0000BF0320D2E72068406800F001000028EAD02068406800F052
:2098C0000100002867D0A069012802D145F0800501E025F08005E069012802D145F040052F
:2098E00001E025F04005206A012802D145F0200501E025F02005606A012802D145F0100522
:2099000001E025F01005A06A012802D145F0080501E025F00805E06A012802D145F004056D
:2099200001E025F004052068006820F0FC00284321680860D4E90201084321690843616926
:2099400008436168491E08432168C8612068006820F001002168086000F056FF06460EE01E
:2099600000F052FF801B0A2809D9032084F83C0000BF002084F83D0000BF03206AE72068C9
:20998000406800F001000028EAD12068406800F0010000B90127012F06D10020206401207D
:2099A00084F83C00002055E7042084F83C00012050E7000010B586B004462D492068884252
:2099C00054D100BF2B48C06940F000702949C8610846C06900F00070019000BF00BF881549
:2099E000029000200390049002A9234800F06CFD4FF400700290022003900320059002A9C2
:209A00001D4800F061FD00BF1C49486820F4C04040F0E06040F48040486000BF0122114666
:209A2000142000F0C0FF142000F0B0FF01221146152000F0B8FF152000F0A8FF1048206373
:209A4000104860631048A063FBF77EF80F480068406940F002000D49096848610B48006863
:209A6000406940F0100009490968486106B010BD0064004000100240000C0140000001408A
:209A8000481E0020641E0020881E0020A8220020816B896811B9416B096941B9164909685F
:209AA000496941F01001144A126851617047816B0968A1F2AA7111B1012911D100E000BFF9
:209AC000816B096908290AD100210C4A1170816B09885180816B4B6953608969916000E0C0
:209AE00000BF00BF04490968496941F01001024A1268516100BFD9E7A8220020940400209D
:209B000010B50446606B806810B9606B006940B92E480068406940F002002C490968486145
:209B200010BD606B006840F23172811A904214D009DCA0F2516080B3CF2818D0D02817D0E6
:209B4000DF2837D108E00F291CD010291BD01F2924D020292ED122E000BF606B00881C49C9
:209B60000880606B017C1A48FBF71AFA23E000BF606B008817490880606B017C1548FBF719
:209B80000FFA18E000BF606B008813490880606B017C1148FBF704FA0DE001E000BF00BFF1
:209BA000606B00880D490880606B017C0B48FBF7F7F900E000BF00BF04480068406940F00C
:209BC000020002490968486100BFA9E7A822002090050020A4050020B8050020CC05002099
:209BE0002DE9F04104460E46042500272068806800F08060B0F1806F0DD02068806800F023
:209C00000060B0F1006F06D02068806800F08050B0F1805F7ED100BF94F83D00012802D17B
:209C20000220BDE8F081012084F83D0000BF94F83C00222804D0322806D062280CD107E0EF
:209C4000422084F83C000BE0522084F83C0007E0722084F83C0003E0122084F83C0000BF18
:209C600000BF2068806800F0806008B1002507E02068806800F0006008B1012500E002257A
:209C8000206800F5C07000EB0510006800F00101206800F5C07000EB05100160206B80683C
:209CA00098B9206800F5C07000EB05100068216BC968226B128841EA42510843216801F5D2
:209CC000C07101EB0511086015E0206800F5C07000EB05100068216B8968226B526841EAF0
:209CE000C201226BD26811430143206800F5C07000EB05100160206B007C00F00F00216BA2
:209D00000861206800F5C07000EB0510406820F00F0100E0B1E0206800F5C07000EB051047
:209D20004160206800F5C07000EB05104068216B09690843216801F5C07101EB051148608A
:209D4000206BC07D0106206B807D41EA0041206B407D41EA0020216B097D0843216801F5D1
:209D6000C07101EB05118860206BC07E0106206B807E41EA0041206B407E41EA0021206BE3
:209D8000007E0143206800F5C07000EB0510C160206800F5C07000EB0510006840F00101EC
:209DA000206800F5C07000EB0510016000F02CFD074620E0701CF0B126B100F025FDC01B3E
:209DC000B04218D9032084F83C001DB980202168886009E0012D03D1E8032168886003E0B4
:209DE0004FF400002168886000BF002084F83D0000BF032015E74DB9206880682149084011
:209E0000884201D1012016E0002014E0012D09D1206880681C490840884201D101200AE0AF
:209E2000002008E02068806818490840884201D1012000E000200028BCD094F83C0042285E
:209E400004D0522806D072280CD107E0222084F83C000BE0322084F83C0007E0622084F8AC
:209E60003C0003E0012084F83C0000BF00BF00BF002084F83D0000BFD3E6042084F83C0080
:209E80000120CEE6010000040001000800000110704710B504460CB9012010BD607920B9A3
:209EA00000202071204600F005F8012060710020F3E7000008B5094A016891420DD100BFC9
:209EC0000749496941F04001054A51611146496901F04001009100BF00BF08BD003002408C
:209EE0000010024070B50446002594F82100022803D00420A063012548E02068006820F05D
:209F00000E00216808602068006820F00100216808601F492068884201D1012026E01C4938
:209F200014312068884201D110201FE0184928312068884201D1801518E015493C312068CB
:209F4000884201D1801411E0114950312068884202D14FF4803009E00D49643120688842C7
:209F600002D14FF4801001E04FF08070084908394860012084F8210000BF002084F82000B8
:209F800000BF606B10B12046616B8847284670BD0800024070B50446E06B05682068066873
:209FA00094F84010042088402840002846D006F00400002842D02068006800F0200028B91E
:209FC0002068006820F004002168086057492068884201D1042027E0544914312068884269
:209FE00001D1402020E0514928312068884201D1001519E04D493C312068884202D14FF49F
:20A00000804011E0494950312068884202D14FF4802009E0454964312068884202D14FF400
:20A02000800001E04FF08060404908394860E06A00287AD02046E16A884776E094F84010C0
:20A04000022088402840A0B306F0020088B32068006800F0200040B92068006820F00A0025
:20A0600021680860012084F8210030492068884201D1022028E02D4914312068884201D18B
:20A08000202021E0294928312068884201D140151AE026493C312068884202D14FF40050AD
:20A0A00012E0224950312068884203D14FF400300AE017E01D4964312068884202D14FF4E5
:20A0C000001001E04FF0007018490839486000BF002084F8200000BFA06A30B32046A16AFE
:20A0E000884722E094F84010082088402840E0B106F00800C8B12068006820F00E002168BC
:20A10000086094F8401001208840E16B48600120A06384F8210000BF002084F8200000BF23
:20A12000206B10B12046216B884770BD080002400146002209B901207047184B0868C01AEB
:20A140001423B0FBF3F08000086414480838C863022081F821000868026843F6F070824393
:20A16000D1E901031843CB6818430B6918434B6918438B691843CB69184302430868026065
:20A1800000208862C862086348638863012081F82100002081F8200000BFCDE70800024059
:20A1A0002DE9F04104460D4616461F464FF0000800BF94F82000012802D10220BDE8F08114
:20A1C000012084F8200000BF94F8210001282CD1022084F821000020A0632068006820F04E
:20A1E0000100216808603B46324629462046FBF73BFDE06A30B12068006840F00E00216893
:20A2000008600BE02068006820F00400216808602068006840F00A002168086020680068EB
:20A2200040F001002168086006E000BF002084F8200000BF4FF002084046BFE770B50446F8
:20A2400000F0E2FA06462546681C10B104480078054400BF00F0D8FA801BA842FAD370BD29
:20A26000580000202DE9F04104460E460127002500BF2648007E012802D10220BDE8F08155
:20A2800001202249087600BF2068022813D14CF25030FDF7E3F990BB0120FDF765F94CF2D5
:20A2A0005030FDF7DBF907461948006920F004001749086123E04CF25030FDF7CFF9F0B93C
:20A2C0004FF0FF303060A56812E02846FDF760F94CF25030FDF7C2F907460D48006920F03E
:20A2E00002000B4908610FB1356007E005F58065D4E9021001EB8020A842E6D800BF00BF03
:20A3000000200249087600BF3846B7E720070020002002400348006940F0800001490861B9
:20A3200000207047002002402DE9FE4F05468B4617469846012600240020029000BF244802
:20A34000007E012802D10220BDE8FE8F01202049087600BF4CF25030FDF780F9064686BBB0
:20A36000012D02D10120029006E0022D02D10220029001E00420029000241EE02201B946B2
:20A38000C24648465146F9F77AFB80B20190022000FB04B000900199FDF70EF94CF25030B4
:20A3A000FDF75CF906460B48006920F001000949086106B104E0601CC4B202988442DDDBDB
:20A3C00000BF00BF00200249087600BF3046BBE7200700200020024000200849096901F0C2
:20A3E000800151B10649054A5160064951601146096901F0800101B1012070470020024064
:20A4000023016745AB89EFCD10B50446042C3BD100202149C8700846807840B900F0F4F953
:20A420001D494860601F88600120887011E000F0EBF919494968401A1749886008468068DE
:20A440004B2802D215480068886000F0DDF91249486011488068114908600F4880684B288A
:20A4600018D30F480068401C0D4908600D48007E08B9012001E00B48007E09490968B1FB42
:20A48000F0F00549C86005E0B4F5805F02D101200549087010BD0000EC0300208C050020B2
:20A4A00088050020B00A0020D802002010B5044604480068204020B1024804602046FFF71D
:20A4C000A3FF10BD140401402DE9F84703460024002000258446002700226EE14FF0010803
:20A4E00008FA02F4D1F8008008EA0400A0427DD1DFF8D0A2D1F80480A8EB0A09D0453AD09A
:20A5000014DCB8F1030F50D009DCB8F1000F31D0B8F1010F1CD0B8F1020F49D120E0B8F1B0
:20A52000110F18D0B8F1120F42D11EE0B9F5881F25D006DCB9F5803F20D0B9F5801F37D15A
:20A540001AE0B9F5001F18D0B9F5041F30D117E0D1F80CC02DE0D1F80C8008F1040C28E07B
:20A56000D1F80C8008F1080C23E0D1F80C8008F10C0C1EE000BF00BF00BF00BF00BF00BF98
:20A58000D1F80880B8F1000F02D14FF0040C0BE0D1F80880B8F1010F03D14FF0080C1C61F7
:20A5A00002E04FF0080C5C6103E04FF0000C00E000BF00BFFF2801D8984601E003F104085E
:20A5C0004646FF2802D84FEA820803E0A2F108084FEA88084746D6F800804FF00F0909FAA7
:20A5E00007F928EA09080CFA07F900E088E048EA0908C6F80080D1F8048008F08058B8F1A3
:20A60000805F7DD100BFDFF8C081D8F8188048F00108DFF8B491C9F81880C846D8F81880A2
:20A6200008F00108CDF8008000BF00BF4FEAB9384FEA920958F829504FEA82784FEA187992
:20A640004FF00F0808FA09F825EA0805DFF87C81434502D14FF0000816E0DFF874814345C5
:20A6600002D14FF001080FE0DFF86881434502D14FF0020808E0DFF86081434502D14FF032
:20A68000030801E04FF004084FEA82794FEA197908FA09F848EA0505DFF840814FEA9209D9
:20A6A00048F82950D1F8048008F48038B8F5803F0AD1DFF82C81D8F8008048EA0008DFF8B4
:20A6C0002091C9F8008009E0DFF81481D8F8008028EA0008DFF80891C9F80080D1F80480CB
:20A6E00008F40038B8F5003F10D1DFF8F48008F10408D8F8008048EA0008DFF8E49000E054
:20A700005AE009F10409C9F800800DE0DFF8D08008F10408D8F8008028EA0008DFF8C0900D
:20A7200009F10409C9F80080D1F8048008F48018B8F5801F0ED1DFF8A88008F10808D8F8ED
:20A74000008048EA0008DFF8989009F10809C9F800800DE0DFF8888008F10808D8F80080CF
:20A7600028EA0008DFF8789009F10809C9F80080D1F8048008F40018B8F5001F0ED1DFF8B1
:20A78000608008F10C08D8F8008048EA0008DFF8509009F10C09C9F800800DE0DFF84080B7
:20A7A00008F10C08D8F8008028EA0008DFF8309009F10C09C9F80080521C102AFFF48EAE64
:20A7C000BDE8F887000011100010024000080140000C01400010014000140140080001405D
:20A7E00000040140024693680B400BB1012000E000207047C2684A40C26070470AB1016148
:20A8000001E00B040361704701480068704700005000002070B504460CB9012070BD4CF691
:20A82000CC402168086045F2555021680860D4E9001048602168A0688860FFF7E5FF05463B
:20A8400006E0FFF7E1FF401B302801D90320E5E72068C0680028F4D14AF6AA202168086028
:20A860000020DBE701464AF6AA200A681060002070470000034800680349097808440149D6
:20A8800008607047500000205800002010B50848006840F0100006490860032000F0C2F870
:20A8A000002000F007F800F02BF8002010BD00000020024070B504460E4800784FF47A71BC
:20A8C000B1FBF0F00C490968B1FBF0F5284600F06FFE08B1012070BD102C07D20022214625
:20A8E000501E00F060F80548046001E00120F2E70020F0E758000020000000205400002013
:20A9000008B500BF1F48806940F001001D4988610846806900F00100009000BF00BF032092
:20A9200000F080F8002211466FF00B0000F03BF8002211466FF00A0000F035F80022114631
:20A940006FF0090000F02FF800221146501F00F02AF800221146101F00F025F80022114650
:20A96000901E00F020F800221146501E00F01BF800BF0549486820F0E06040F000704860E2
:20A9800000BF08BD001002400000014000BF00F01F02012191404209920002F1E022C2F851
:20A9A000001100BF70472DE9F05F80460D461646002707F015F8074639462A46334601F065
:20A9C0000700C0F1070ABAF1040F02D94FF0040A01E0C0F1070AD14600F1040ABAF1070F4E
:20A9E00002D24FF0000A01E0A0F1030AD4464FF0010A0AFA09FAAAF1010A0AEA020A0AFAA6
:20AA00000CFA4FF0010B0BFA0CFBABF1010B0BEA030B4AEA0B042146404606F0E9FFBDE87B
:20AA2000F09F000000BF00F00702064B19684FF6FF031940044B0B4343EA0221014B1960AB
:20AA400000BF70470CED00E00000FA0500BF00BF00BF00BF00BFBFF34F8F00BF00BF00BF20
:20AA60000948006800F4E06008490843001D0649086000BF00BF00BFBFF34F8F00BF00BF2E
:20AA800000BF00BF00BFFDE70CED00E00000FA052DE9F04385B006463DA30FCB01AC0FC4B9
:20AAA0003FA0006800904FF00008002500270024A146012E30D0022E58D0102E61D13948A9
:20AAC0004468006800F0807000B301A8C4F38341475C04F4803070B132484068C0F34040EA
:20AAE0001DF8008004F4803040B12F48B0FBF8F000FB07F502E02D4807FB00F529484068C0
:20AB000000F48000B0F5800F01D1A94603E068000321B0FBF1F935E02248046A04F4407033
:20AB2000B0F5807F05D104F0020010B14FF400491BE004F44070B0F5007F07D11948406AAE
:20AB400000F0020010B149F640490EE004F44070B0F5407F07D11348006800F4003010B100
:20AB60004FF2244901E04FF000090BE000F0A0F90C494968C1F38131491C4900B0FBF1F9DB
:20AB800000E000BF00BF484605B0BDE8F083000002030405060708090A0B0C0D0E0F101065
:20ABA000010200000010024000127A0000093D00F8B5044600260025207800F0010000287B
:20ABC0006BD000274348C06900F0805070B900BF4048C06940F080503E49C8610846C069DF
:20ABE00000F08050009000BF00BF01273A48006800F48070B0B93848006840F4807036499D
:20AC00000860FFF701FE064606E0FFF7FDFD801B642801D90320F8BD2F48006800F4807019
:20AC20000028F2D02B48006A00F440752DB3A08800F44070A84220D02648006A20F440757D
:20AC4000012026490860002008602248056205F0010090B1FFF7D8FD064608E0FFF7D4FDA6
:20AC6000801B41F28831884201D90320D3E71948006A00F002000028F0D01648006A20F44B
:20AC800040706168084313490862012F04D10846C06920F08050C86100BF207800F002005C
:20ACA000022807D10B48406820F44040A168084308494860207800F01000102807D10548C1
:20ACC000406820F48000E1680843024948600020A1E700000010024000700040400442423F
:20ACE00070B504460D4600266248006800F00700A8420ED25F48006820F0070028435D4962
:20AD000008600846006800F00700A84201D0012070BD207800F00200022807D15648406843
:20AD200020F0F000A168084353494860207800F0010000285DD06068012806D14E480068D7
:20AD400000F4003090B90120E2E76068022806D14948006800F0007040B90120D8E7464813
:20AD6000006800F0020008B90120D1E74248406820F00300616808433F494860FFF744FD1F
:20AD800006466068012810D108E0FFF73DFD801B41F28831884201D90320B9E73648406869
:20ADA00000F00C000428F0D123E06068022810D108E0FFF729FD801B41F28831884201D9A5
:20ADC0000320A5E72C48406800F00C000828F0D10FE008E0FFF718FD801B41F28831884288
:20ADE00001D9032094E72448406800F00C000028F0D12048006800F00700A8420ED91D48E5
:20AE0000006820F0070028431A4908600846006800F00700A84201D0012079E7207800F00C
:20AE20000400042807D11448406820F4E060E168084311494860207800F00800082808D183
:20AE40000D48406820F46050216940EAC1000A49486000F03DF808494968C1F30311074A81
:20AE6000515CC840064908600020FFF723FD00204EE700000020024000100240346B01087F
:20AE80000000002001480068704700000000002000B5FFF7F7FF04494968C1F30221034A47
:20AEA000515CC84000BD000000100240446B010800B5FFF7E7FF04494968C1F3C221034AA3
:20AEC000515CC84000BD000000100240446B0108F0B585B00FF26C0C9CE8E01001A8A0E8FE
:20AEE000E0101CA52D68009500210022002300240020194D696801F00C05F5B1042D02D0EB
:20AF0000082D19D101E0154819E001ADC1F38346AC5D01F4803555B10F4D6D68C5F3404589
:20AF20001DF805200D4D6543B5FBF2F302E00C4D04FB05F3184602E000BF084800BF00BF41
:20AF400005B0F0BD02030405060708090A0B0C0D0E0F1010010200000010024000127A0017
:20AF600000093D00F8B504460025207800F00100002878D0F848406800F00C0004280CD08A
:20AF8000F548406800F00C00082811D1F248406800F48030B0F5803F0AD1EF48006800F466
:20AFA000003000285FD0606800285CD10120F8BD00BF6068B0F5803F06D1E748006840F48A
:20AFC0008030E549086028E0606858B9E248006820F48030E04908600846006820F48020F9
:20AFE00008601AE06068B0F5A02F0BD1DA48006840F48020D84908600846006840F4803056
:20B0000008600AE0D448006820F48030D24908600846006820F48020086000BF606888B181
:20B02000FFF7F2FB054606E0FFF7EEFB401B642801D90320BBE7C848006800F400300028D3
:20B04000F2D010E0FFF7E0FB054606E0FFF7DCFB401B642801D90320A9E7BF48006800F498
:20B0600000300028F2D1207800F00200022857D1B948406800F00C0050B1B748406800F09C
:20B080000C00082818D1B448406800F4803098B9B148006800F0020020B12069012801D04B
:20B0A000012084E7AC48006820F0F800616940EAC100A949086033E02069E8B10120A7494B
:20B0C0000860FFF7A1FB054606E0FFF79DFB401B022801D903206AE79F48006800F00200A3
:20B0E0000028F2D09C48006820F0F800616940EAC1009949086013E0002098490860FFF7C1
:20B1000083FB054606E0FFF77FFB401B022801D903204CE79048006800F002000028F2D13E
:20B12000207800F0080008282DD1A069B8B101208B490860FFF768FB054606E0FFF764FBA3
:20B14000401B022801D9032031E78348406A00F002000028F2D0012006F0C2FF13E0002019
:20B160007F490860FFF750FB054606E0FFF74CFB401B022801D9032019E77748406A00F015
:20B1800002000028F2D1207800F00400042873D100267148C06900F0805070B900BF6E4860
:20B1A000C06940F080506C49C8610846C06900F08050009000BF00BF01266A48006800F40E
:20B1C0008070B0B96748006840F4807065490860FFF71AFB054606E0FFF716FB401B64289B
:20B1E00001D90320E3E65F48006800F480700028F2D000BFE068012806D15748006A40F06C
:20B2000001005549086227E0E06858B95248006A20F00100504908620846006A20F00400E1
:20B22000086219E0E06805280BD14B48006A40F00400494908620846006A40F001000862DA
:20B240000AE04548006A20F00100434908620846006A20F00400086200BFE068A0B1FFF782
:20B26000D3FA054609E0FFF7CFFA401B41F28831884202D903209AE622E03748006A00F0A4
:20B2800002000028EFD012E0FFF7BEFA054608E0FFF7BAFA401B41F28831884201D903203A
:20B2A00085E62D48006A00F002000028F0D1012E05D12948C06920F080502749C86100BF92
:20B2C000E069C8B32448406800F00C00082860D0E069022848D1002020490866FFF794FA33
:20B2E000054606E0FFF790FA401B022801D903205DE61948006800F000700028F2D1206A3A
:20B30000B0F5803F07D11448406820F40030A168084311494860D4E9080108430E4949683A
:20B3200021F4741108430C49486001200B490866FFF76AFA054607E02DE0FFF765FA401BFF
:20B34000022801D9032032E60348006800F000700028F2D01FE000000010024000004242DC
:20B36000800442420070004000200C490866FFF74BFA054606E0FFF747FA401B022801D930
:20B38000032014E60648006800F000700028F2D101E001200BE6002009E600000000424209
:20B3A00000100240042808D14FF0E021096941F004014FF0E022116107E04FF0E021096902
:20B3C00021F004014FF0E022116170470EB55A480078012800D10EBD5848407E08B902200A
:20B3E00001E05648407E02465448418801235448F9F736FF5348007830B9534A1188534AAF
:20B400001088534A03F050FD524853490978CDE90010524802784D48006802905048037884
:20B4200048480078029903F071FA4A480078C0434C49087047488079C04388714548B0F937
:20B440000200C04348804348B0F90400C04388804548007838B945488278454801893C4BC1
:20B46000444809F099FB4448007828B940488189374A4248FCF75CFB41494248F8F7D4FF11
:20B48000414805F081FD41480088401C3F49088008460088052801DB002008803C480088A0
:20B4A000401C3B490880084600880A2809DB00200880254B1A88997A5B8898B2354BF9F7CE
:20B4C000D3FA35480088401C3349088008460088322804DB002008803048F9F7DBFF3048C9
:20B4E0000088401C2E49088008460088642809DB00200880124908780A222A4906F054FABD
:20B500001149887228480088401C2749088008460088C82801DB0020088024480088401CF1
:20B520002249088008460088B0F57A7F01DB0020088000BF4FE700005C000020B00A0020D5
:20B54000BC030020D8000020DC080020220500208C010020DE0000203D040020DA000020C3
:20B560003C040020E600002018040020BA010020501D0020781500207604002074040020E2
:20B580001A050020621D0020D00B00205E000020600000200402002062000020D00100203B
:20B5A00064000020D6140020660000206800002070B504462546681EB0F1807F01D30120FA
:20B5C0000FE0681E4FF0E02148610F214FF0FF3006F00EFA00204FF0E02188610720086198
:20B5E000002070BD10B5FFF7F1FE10BD7047704710B50346002200BF93F83C00012801D168
:20B60000022010BD012083F83C0000BF22F0FF00CC6840EA040222F440708C6840EA040245
:20B6200022F480604C6840EA040222F400600C6840EA040222F480500C6940EA040222F475
:20B6400000504C6940EA040222F480408C6940EA040222F400408C6940EA04021868426419
:20B6600000BF002083F83C0000BF00BFC9E7024600BF92F83C00012801D102207047012044
:20B6800082F83C0000BF022082F83D001068406820F0700013685860106840680B6818439B
:20B6A000136858601068806820F0800013689860106880684B68184313689860012082F878
:20B6C0003D0000BF002082F83C0000BF00BFD5E770B504460D4604222946206808F0C6FFC2
:20B6E0002068406C40F40040216848642068006840F0010021680860002070BD70B504469F
:20B700000D4600222946206808F0B0FF00BF2068006A41F21111084050B92068006A891034
:20B72000084028B92068406C20F400402168486400BF00BF2068006A41F21111084050B90D
:20B740002068006A8910084028B92068006820F001002168086000BF002070BD10B5044628
:20B760000CB9012010BD94F83D0028B9002084F83C00204600F00CF8022084F83D00211D21
:20B78000206808F02BFF012084F83D000020E9E710B586B0044632492068884233D100BF60
:20B7A0003048806940F400602E4988610846806900F40060019000BF00BF8814029000204C
:20B7C0000390049002A92848FEF77EFE4FF46040029002200390059002A92348FEF774FE7A
:20B7E0004FF47060029002200390059002A91F48FEF76AFE012211461920FFF7D4F819203D
:20B80000FFF7C4F829E02068B0F1804F25D100BF1448C06940F001001249C8610846C0690F
:20B8200000F00100019000BF00BF00BF0846806940F0040088610846806900F00400019039
:20B8400000BF00BF012002900020039004900220059002A90548FEF737FE06B010BD000014
:20B86000002C014000100240000C0140000801400146022081F83D000868006840F001004B
:20B880000A681060012081F83D000020704701460868C06840F001000A68D060086800688E
:20B8A00040F001000A681060002070472DE9F04104460D46002600BF94F83C00012802D111
:20B8C0000220BDE8F081012084F83C0000BF022084F83D002068866826F0770626F47F46D5
:20B8E00020688660286850283BD00CDC202860D004DC002853D0102865D155E030285DD014
:20B90000402860D141E0602835D070280DD0B0F5805F03D0B0F5005F55D115E02068806885
:20B9200020F00700216888604EE0D5E902136A68206808F0A9FE2068866826F0770646F046
:20B940007706206886603FE0D5E902136A68206808F09AFE2068806840F48040216888604B
:20B9600032E0EA686968206808F06CFF5021206808F096FE28E0EA686968206808F077FF01
:20B980006021206808F08CFE1EE0EA686968206808F058FF4021206808F082FE14E00021AE
:20B9A000206808F07DFE0FE01021206808F078FE0AE02021206808F073FE05E0302120689C
:20B9C00008F06EFE00E000BF00BF012084F83D0000BF002084F83C0000BF00BF71E77047A7
:20B9E00010B5044620680069C0F34000D8B12068C068C0F34000B0B16FF002002168086174
:20BA0000012020772068806900F0030018B12046FFF7E5FF05E0204600F0D6F8204600F0A2
:20BA2000ABF90020207720680069C0F38000D8B12068C068C0F38000B0B16FF004002168CE
:20BA40000861022020772068806900F4407018B12046FFF7C4FF05E0204600F0B5F8204679
:20BA600000F08AF90020207720680069C0F3C000D8B12068C068C0F3C000B0B16FF00800C4
:20BA800021680861042020772068C06900F0030018B12046FFF7A3FF05E0204600F094F8C7
:20BAA000204600F069F90020207720680069C0F30010D8B12068C068C0F30010B0B16FF0A7
:20BAC000100021680861082020772068C06900F4407018B12046FFF782FF05E0204600F06F
:20BAE00073F8204600F048F9002020772068006900F0010058B12068C06800F0010030B120
:20BB00006FF0010021680861204600F095F920680069C0F3C01058B12068C068C0F3C0103F
:20BB200030B16FF08000216808612046FFF75EFD20680069C0F3801058B12068C068C0F3FC
:20BB4000801030B16FF0400021680861204600F077FA20680069C0F3401058B12068C0686F
:20BB6000C0F3401030B16FF02000216808612046FFF73DFD10BD00001FB504460E49206810
:20BB8000884218D140200090022001900320039069460A48FEF798FC00BF0949486820F43A
:20BBA000406040F0E06040F44060486000BF0021044800F00BF81FBD000400400010014069
:20BBC00000000140101D00207047000030B504460D4601222946206808F03AFD0A4920687A
:20BBE000884201D1012000E0002028B12068406C40F40040216848642068006840F00100B1
:20BC000021680860002030BD002C014070B504460D46164600BF94F83C00012801D10220F7
:20BC200070BD012084F83C0000BF022084F83D0036B1042E1BD0082E31D00C2E5ED145E09B
:20BC40002946206808F036FD2068806940F00800216888612068806920F0040021688861B0
:20BC600020688069296908432168886147E02946206808F051FD2068806940F40060216812
:20BC800088612068806920F480602168886120688069296940EA0120216888612FE02946A6
:20BCA000206808F071FD2068C06940F008002168C8612068C06920F004002168C8612068FC
:20BCC000C069296908432168C86118E02946206808F090FD2068C06940F400602168C86141
:20BCE0002068C06920F480602168C8612068C069296940EA01202168C86100E000BF00BF4F
:20BD0000012084F83D0000BF002084F83C0000BF00BF85E710B504460CB9012010BD94F87A
:20BD20003D0028B9002084F83C00204600F00CF8022084F83D00211D206808F04FFC0120AE
:20BD400084F83D000020E9E708B5094A016891420DD100BF0749C96941F00201054AD1611A
:20BD60001146C96901F00201009100BF00BF08BD00040040001002407047000030B50446F6
:20BD80000D4601222946206808F062FC0A492068884201D1012000E0002028B12068406C3B
:20BDA00040F40040216848642068006840F0010021680860002030BD002C014030B504461F
:20BDC0000D4600222946206808F042FC19492068884201D1012000E0002090B100BF206892
:20BDE000006A41F21111084050B92068006A8910084028B92068406C20F4004021684864C2
:20BE000000BF00BF2068006A41F21111084050B92068006A8910084028B92068006820F058
:20BE200001002168086000BF012084F83D00002030BD0000002C014038B504467048008886
:20BE4000401C6F49088008460088B0F5967F01DB002008806B4840786B4B0090DA7999791C
:20BE600058796A4B1B7800F05BFE69480078401C674908700846007805280ADB65480068C6
:20BE8000806840F0010063490968886000206049087061480068401C5F49086000F04CFA90
:20BEA0005D48C08842F6FF7188420CDA5A480089594989880844584908810846C088898842
:20BEC00008445549C880544A917A108905F008FD524948805249534804F08CFA52480078CF
:20BEE000524909784840FF281AD14F4880794F4989794840FF2813D14B4880884B4989888F
:20BF0000484080B24FF6FF71884209D14648408846494988484080B24FF6FF7188420AD045
:20BF2000FEF772FC42490968401AC82807D902204049087003E0FEF767FC3D4908603D48A7
:20BF40000078012802D0022856D151E03648807901284CD138480078012804D1FBF73CFA11
:20BF600000203549087030480078012811D0022804D003280ED0042837D116E0264B1A896C
:20BF8000264BB3F90210284BB3F90200FBF7DCFB2CE000BF204B1A89204BB3F90210224B19
:20BFA000B3F90400FBF7D0FB20E02448007800F0010050B9184B1A89184BB3F902101A4BAA
:20BFC000B3F90400FBF7C0FB0EE01C48007800F0010048B1104B1A89104BB3F90210124BDC
:20BFE000B3F90200FBF7B0FB00E000BF00BF04E001201149087000E000BF00BF38BD00006E
:20C0000010050020DA000020D00A00203C04002008050020741D0020C8070020DC080020C6
:20C020008C010020D8020020DE000020E60000200C0500203000002009050020B9010020CC
:20C04000704770472DE9F0470446206805682068C668206847694FF00008C14605F00F089E
:20C06000B8F1000F0AD105F0200038B106F0200020B1204609F006F8BDE8F087B8F1000F17
:20C080006DD007F0010018B906F49070002866D005F0010030B106F4807018B1E06B40F03D
:20C0A0000100E06305F0040030B107F0010018B1E06B40F00200E06305F0020030B107F012
:20C0C000010018B1E06B40F00400E06305F0080030B107F0010018B1E06B40F00800E0636F
:20C0E000E06B68B305F0200028B106F0200010B1204608F0C7FF20684069C0F38019E06B29
:20C1000000F0080010B9B9F1000F22D0204608F04AFF2068406900F04000B0B12068406919
:20C1200020F0400021684861606B50B11748616B4863606BFDF7D6FE10B1606B416B884741
:20C140000CE02046FFF77DFF08E02046FFF779FF04E02046FFF775FF0020E0638CE705F0E0
:20C16000800030B106F0800018B1204609F0D0F882E705F0400030B106F0400018B1204614
:20C1800008F021FF78E700BF76E70000554E010810B504460CB9012010BDA06900B100E004
:20C1A00000BF94F8390028B9002084F83800204600F028F8242084F839002068C06820F413
:20C1C00000502168C860204608F0BEFF2068006920F49040216808612068406920F02A0011
:20C1E000216848612068C06840F400502168C8600020E063202084F8390084F83A000020FA
:20C20000CAE7000010B586B004462B49206888424FD100BF2948C06940F480202749C8617C
:20C220000846C06900F48020019000BF00BF0815029002200390012004900320059002A968
:20C240001F48FEF741F94FF400600290002003900120049002A91A48FEF736F900BF194959
:20C26000486820F0300040F0E06040F01000486000BF012211462720FEF795FB2720FEF735
:20C2800085FB11480068C06840F480700E490968C8600D480068406940F001000A490968C6
:20C2A000486109480068C06840F0200006490968C86006B010BD000000480040001002405F
:20C2C0000010014000000140EC2400207047704710B500F011F9054931F8100041F255510F
:20C2E0000844034908810020086010BDCC7D0108C807002000B585B000BF0D48806940F070
:20C3000010000B4988610846806900F01000009000BF00BF4FF46070019000200290012014
:20C32000039001A90348FEF7CFF805B000BD00000010024000100140F8B500F0DDF80646E6
:20C3400000F0DAF8044600F0D7F80546A64203D1AC4201D15E4805705E48007830B95C4885
:20C3600000785B49487001205A4908705848007857494978884210D0FEF746FA564908604E
:20C380005648007828B155480078401C5349087017E001205249887213E0FEF735FA4E49CE
:20C3A0000968401AC8280CD900204D4988724B4908704B498881C8814A490870012048497E
:20C3C00008744748807A10B9002047490870404800783F494978454A515C884245D140487A
:20C3E000006840B13E48006842F6AA21B1FBF0F03B49888002E00120394988803A48007854
:20C40000401C394908700846007802280DDD3448006844F63E11B1FBF0F031498881002050
:20C420003049087001202E4908742F4800780F280CDA274800782E4931F8100041F255517B
:20C440000844274908810020888009E00F20264908701F480078264931F8100020490881F7
:20C4600000201F490860C88026E019484078184909781E4A515C88421ED100201A490870BA
:20C480001749888012480078194931F8100041F255510844124908814FF6FF700860114849
:20C4A0000078401CC0B20F490870052804DD0620087000200A490874054800680D49009030
:20C4C00003F0A4F80248007801494870F8BD0000A0030020A2030020A4030020A30300203F
:20C4E000C8070020A8030020A9030020BC7D0108CC7D01088C01002010B51E48C07AA8B9AF
:20C500004FF400711C48FEF76DF904464FF480711948FEF767F944EA4000C4B28021164891
:20C52000FEF760F944EA8000C4B220E04FF400711148FEF757F908B9012000E0002004460B
:20C540004FF480710C48FEF74DF908B9012000E0002044EA4000C4B280210748FEF742F932
:20C5600008B9012000E0002044EA8000C4B204F0070010BDC80700200010014007E004487A
:20C5800003F06DFE002005F09BFCFAF777FCF6E70001002070B50446204609F05AFEA189DF
:20C5A0000122A068FEF72AF90120FAF70CFCA1882068FEF717F90546A1890022A068FEF7D4
:20C5C0001DF90120FAF7FFFB012D01D1012070BD0020FCE71FB50446A06809F0B7FD20688D
:20C5E00009F0B4FDA089009001200390112001906946A068FDF768FFA088009001200390E4
:20C600001120019069462068FDF75EFF1FBD2DE9F04704460F464FF000084FF08009204693
:20C6200009F017FE00251CE0A1890122A068FEF7E5F83220FAF7C7FBA1882068FEF7D2F82F
:20C640000646012E03D149FA05F040EA0808A1890022A068FEF7D2F83220FAF7B4FB681C90
:20C66000C5B2082DE0DB87F800800120FAF7ABFBBDE8F08710B50446204609F0F2FDA188FA
:20C6800001222068FEF7BAF80120FAF79CFBA1890122A068FEF7B2F83220FAF794FBA189AF
:20C6A0000022A068FEF7AAF8A18800222068FEF7A5F80120FAF787FB10BD10B5044620467E
:20C6C00009F0CFFDA1890122A068FEF797F8A18801222068FEF792F83220FAF774FBA1888E
:20C6E00000222068FEF78AF83220FAF76CFBA1890022A068FEF782F810BD10B5044620466A
:20C7000009F0AFFDA18800222068FEF777F8A1890122A068FEF772F83220FAF754FBA188CE
:20C7200001222068FEF76AF83220FAF74CFBA18800222068FEF762F8A1890022A068FEF702
:20C740005DF810BD2DE9F04104460D46A8468026204609F086FD002736E006EA0800C0B1B7
:20C76000A18801222068FEF749F83220FAF72BFBA1890122A068FEF741F83220FAF723FB62
:20C78000A1890022A068FEF739F83120FAF71BFB17E0A18800222068FEF730F83220FAF79D
:20C7A00012FBA1890122A068FEF728F83220FAF70AFBA1890022A068FEF720F83120FAF717
:20C7C00002FB7610781CC7B2082FC6DBA18801222068FEF713F80120FAF7F5FABDE8F08106
:20C7E00001480249086070470030000808ED00E0012029490978052910D127491031097824
:20C800009B290BD1244914310978522906D1224918310978052901D103203BE01E49097898
:20C8200004291BD11C4910310978C32916D11A4914310978B42911D11749183109780B299F
:20C840000CD116490988802901D1022022E013490988B1F5807F1DD105201BE00E490978F4
:20C8600081B90D491031097810290BD10A4914310978042906D10849183109780A2901D114
:20C88000012007E006490968064A914201D1042000E0002070470000D0FF0FE0E0F7FF1F4D
:20C8A000002004E01004031300B585B000BF2B48806940F01000294988610846806900F083
:20C8C0001000009000BF00BF2548264908604014888008468088019000200290012003904D
:20C8E000086801A9FDF7F0FD00201E4988714872C860C87108721A481B4908604FF48040F7
:20C9000088800846808801900020029001200390086801A9FDF7D8FD0020134988714872B0
:20C92000C860C87108720E48104908604FF40040888008468088019000200290012003902D
:20C94000086801A9FDF7C0FD0020084988714872C860C871087205B000BD00000010024049
:20C9600000100140F01B0020041C0020181C00202DE9F04104460F4616469846069DB8F13B
:20C98000000F04D10121204609F044FC03E00221204609F03FFCE07900F0010020B1012016
:20C9A0006072FDF731FFE060607A01281BD1207A50B9FDF729FFE060FDF726FF2061002099
:20C9C0006072012028700EE0FDF71EFFE168401AB84208D9FDF718FFE0600020607228707A
:20C9E000FDF712FF2061287868B966B1FDF70CFF2169401AB04206D9FDF706FF206100208B
:20CA0000607201202870BDE8F0812DE9F04105460E4617469846B8F1F10F13D100240EE0B5
:20CA2000BC4201D1012300E000231A4605EBC403998855F83400FDF7E1FE601CC4B2B4428B
:20CA4000EEDB0DE0002409E005EBC402918855F834000022FDF7D2FE601CC4B2B442F3DB27
:20CA6000BDE8F08110B586B000BF2A48806940F00400284988610846806900F00400019041
:20CA800000BF00BF00BF0846806940F0080088610846806900F00800019000BF00BF00249F
:20CAA00033E01D4A02EBC40291881B4A52F834000022FDF7A3FE184800EBC40080880290ED
:20CAC0000120039002200590134951F8340002A9FDF7FAFC114A02EBC40291880F4A52F8B3
:20CAE00034000022FDF78AFE0C4800EBC400808802900120039002200590084951F834008E
:20CB000002A9FDF7E1FC601CC4B2032CC9DB06B010BD00000010024040040020580400201F
:20CB20002DE9F0470746894692461C46DDF82080FDF76AFEB0F5FA6F0DD2F0232A460321ED
:20CB40009848FFF762FFF023324603219648FFF75CFFBDE8F087B9F1060F06D0B9F10C0F4A
:20CB600005D0B9F1FF0F06D103E0002505E0012503E0022501E0002500BF00BFBAF1060FF0
:20CB800006D0BAF10C0F05D0BAF1FF0F06D103E0002605E0012603E0022601E0022600BFAC
:20CBA00000BF07F0F000102802D0202807D107E0F1232A4603217B48FFF727FF07E000BF91
:20CBC00043462A4603217748FFF71FFF00BF00BF07F00F00072843D2DFE800F04204436FEE
:20CBE0007AA6AD004CB9F123324603216E48FFF70CFF00206D49088031E0B8F1F10F22D1F1
:20CC00006B48408969490988884206DDF123324603216548FFF7F9FE0FE06548808963490D
:20CC20000988884206DDF023324603215E48FFF7ECFE02E000205D4908805C480088401CC9
:20CC40005A4908800BE0B8F1F00F08D1F023324603215548FFF7D9FE0020544908809DE062
:20CC600000BF04BB51480088B0F5167F06DAF123324603214C48FFF7C8FE0EE04B480088F2
:20CC8000B0F5966F06DAF023324603214648FFF7BCFE02E000204549088044480088401C95
:20CCA0004249088008E04346324603213E48FFF7ACFE00203D49088070E00CB9F12000E0FA
:20CCC000F0200346324603213748FFF79EFE65E004BB36480088B0F5167F06DAF12332469E
:20CCE00003213148FFF791FE0EE030480088B0F5966F06DAF023324603212B48FFF785FEFF
:20CD000002E000202949088028480088401C2749088008E0F023324603212348FFF775FE60
:20CD200000202249088039E0F123324603211E48FFF76BFE32E01F4800881D49098988428F
:20CD400022DB1B48408919490988884206DDF123324603211448FFF758FE0FE0144880895E
:20CD600012490988884206DDF023324603210E48FFF74BFE02E000200C4908800B4800881C
:20CD8000401C0A49088008E0002008490880F023324603210448FFF738FE00BF00BF00BF17
:20CDA000D7E60000400400205804002070040020D00A0020EC0300207CB504460D46094919
:20CDC00003C9CDE90001084803F03CFA01208DF8060003208DF80000009820600198606092
:20CDE0007CBD000054710108000100202DE9FF4F85B080461D464FF00009FE4903C9CDE938
:20CE00000301FD48008800B2FC490880FC48B0F9020064286DDD0846B0F90000002868DD99
:20CE2000F748B0F9020064214843F449B1F90010B0FBF1F000B2F34908800846B0F90040C8
:20CE4000F1480068C0EB0420EF49096801EBA010ED49086008460068001200B2EB49088049
:20CE6000E648B0F90000EA49B1F90010401A052811DDE348B0F90200E649B1F90010401A60
:20CE8000002804DDDF48B0F90000E3490880DC484088E0490880D948B0F90000DC490880F1
:20CEA000DE48007820BBDE48B0F90400192829DDDC480088401CDB49088008460088282805
:20CEC00020DB00200880D1480088D749D74A128821F81200D5480088401CD4490880084614
:20CEE000008832280EDB002008800120CB49087008E0C248B0F90000C5490880C048408811
:20CF0000C4490880CA48408800B2CA4908800798A0F16404B4F5006F02DD4FF4006000E043
:20CF20002046044604FB04F0C11700EB5151CC12C14800780521B1EBD00F1BDBB04AD17BAD
:20CF4000BE4A1279012383EAD21282F0010003F04BF9BA49097901F07F01B94A92F910206B
:20CF60001144B54A127801EBD2010A314843C0F387291AE0A24AD17BB04A1279012383EAA3
:20CF8000D21282F0010003F02FF9AC49097901F07F01AB4A92F910201144A74A127801EBCB
:20CFA000D20115394843C0F3872909F10100604332214843A349C98990FBF1F000B2A2499F
:20CFC000088009EB8900162101EB40008B49B1F90010884202DA00209B49088096480078D3
:20CFE000C0F3800038B18548B0F900003C2802DC0020954908809448B0F90000002803DD4A
:20D000009148B0F9000000E000208F4908800846B0F900008749B1F90010884203DA8A4834
:20D02000B0F9000002E08348B0F90000864908809DF81800C0F34000B0B305F00F0001286A
:20D0400006D002280FD0032818D004282DD120E04FF4FA6201217748B0F9000007F01AFA80
:20D060007A4908602CE040F2DC5201217148B0F9000007F00FFA7549086021E04FF47A723F
:20D0800001216C48B0F9000007F004FA6F49086016E04FF4FA7201216648B0F9000007F0E7
:20D0A000F9F96A4908600BE00BE04FF47A7201216048B0F9000007F0EDF96449086000BF3A
:20D0C00009E04FF4FA7201215A48B0F9000007F0E1F95E4908604FF47A7201215548B0F9D4
:20D0E000000007F0D7F95A4908604D48807968B94348B0F90200642808DD41484088554919
:20D100000880084600880004534908609DF81800C0F34000F0B305F00F00012806D0022839
:20D1200014D0032824D0042842D134E04649B1F9001001EBC1010811474B45490A6843496B
:20D14000096809F0ABF8434908803EE03E49B1F9001001EB410202EBC10108113E4B3C494A
:20D160000A683A49096809F099F83A4908802CE03549B1F9001001EB810202EBC101081139
:20D18000354B33490A683149096809F087F8314908801AE01AE0304B2D4802682B48016892
:20D1A0002948B0F9000009F079F82A4908800CE0294B27480268254801682348B0F90000CD
:20D1C00009F06CF82349088000BF0BE0224B204802681E4801681C48B0F9000009F05EF8EA
:20D1E0001C4908806FF0C7001C49086140F63400486135E03C710108EC030020260100201A
:20D20000DC0800202C010020080100202E0100202A010020280100200C0100201001002053
:20D22000DE00002012010020140800200E010020F00A002030010020B9010020B00A002033
:20D24000D00A0020040200203201002034010020380100203C01002020010020D406002015
:20D260005D48C08901B25D4A5D48B0F9000004F0E1FC5C4908806FF063005849086140F21C
:20D280001A404861584AD17B584A127A012383EAD21002F07BFF5549097A4FF47A725143AC
:20D2A00048434014019050480089C111504A019804F0C0FC4F4908804F4A117B4A4AD088F7
:20D2C0004E4A128801F006FC07464C48078001231A464B480188384601F054FD4849088048
:20D2E000424A517A404A907D01F0E2FB82463F4A527A0F3A91B23C4A507D01F0D9FB8346E8
:20D300000AFB0BF0810A0291029988B201231A463C49098801F036FD3A4908803148B0F92F
:20D3200000003749098848438612364800887043861235480078B0B934480068301A0228B2
:20D3400005DD32480068801C3049086018E02F480068301A10F1030F12DA2C480068C01EB2
:20D360002A4908600CE029480068132805DD2748006810382549086002E000202249087016
:20D380002248006810F1C80F03DA6FF0C7001F4908601348008818B91D4802F060FF02E0C4
:20D3A0001B4802F04FFF194800681249B1F900100844401000B2ADF8100001208DF8120031
:20D3C00004208DF80C000398C8F800000498C8F8040009B0BDE8F08FC8070020D406002017
:20D3E0003C01002046010020DC080020B00A0020B006002048010020F00A00204A010020C7
:20D400004C0100204E0100204401002040010020000100202DE9FF4F87B0824616461F4625
:20D42000FE4903C9CDE90501002004900390BE4203DA07FB07F0C01202E006FB06F0C01283
:20D44000F749488008464088B0F5006F02DD4FF4006001E0F2484088F14948809DF820007E
:20D46000C0F3400000287CD0149803287AD004DC012807D0022876D149E0042874D03328DF
:20D48000F9D1D7E0E748007A002801DC012001E0E448007A0490E348407A0390E0484088B9
:20D4A000E049C9884843C00A04B2DE48C088A04202DADC48C08800E0204604B2D948408969
:20D4C000D949097A48434FF47A714843401400EBC00101EB00104FF6FF7101EA800501231E
:20D4E0000522D2480188284601F04CFCCF490880CC48C0884042CE49086100204861C948E3
:20D50000C0888002404288610020C861DFE0C548007D002801DC012001E0C248007D049022
:20D52000C048407D0390BE484088BE49498A4843C00A04B2BB48408AA04202DAB948408A8A
:20D5400000E0204604B2B748C08AB749097A48434FF47A714843401400EBC00101EB0010C3
:20D5600003E0B5E01DE0ADE063E04FF6FF7101EA800501230522AD480188284601F002FC1B
:20D58000AA490880A748408A4042A949086100204861A448408A8002404288610020C861C5
:20D5A00095E0A04890F82000002801DC012002E09C4890F8200004909A4890F82100039020
:20D5C000974840889749C98B4843C00A04B29548C08BA04202DA9348C08B00E0204604B25D
:20D5E0009048408C9049097A48434FF47A714843401400EBC00101EB00104FF6FF7101EA4B
:20D6000080050123052289480188284601F0BAFB864908808348C08B404285490861002086
:20D6200048618048C08B8002404288610020C8614DE000BF7B4890F82C00002801DC01206F
:20D6400002E0784890F82C000490764890F82D000390734840887349498D4843C00A04B2BA
:20D660007048408DA04202DA6E48408D00E0204604B26C48C08D6C49097A48434FF47A71F6
:20D680004843401400EBC00101EB00104FF6FF7101EA80050123052264480188284601F0FF
:20D6A00071FB624908805F48408D404260490861002048615B48408D80024042886100207D
:20D6C000C86104E0002004900390002400BF4DE09DF82000C0F34000F0BB524890F8380039
:20D6E000002801DC012002E04E4890F8380004904C4890F82D000390494840884949498D9B
:20D700004843C00A04B24748408DA04202DA4548408D00E0204604B24248C08D4249097AA9
:20D7200048434FF47A714843401400EBC00101EB00104FF6FF7101EA8005012305223B48B6
:20D740000188284601F01EFB384908803548408D40423749086100E008E000204861314800
:20D76000408D8002404288610020C861314890F90E00322805DC2F4890F90E0010F1320F0B
:20D7800002DA00202B4988732A4890F90F00322805DC284890F90F0010F1320F02DA002093
:20D7A0002449C873244800780521B1EBD00F6BDB224AD17B1C4A1279012383EAD21282F066
:20D7C000010002F011FD1849097901F07F01194A92F9102011449DF8202001EBD2010831B4
:20D7E00001EB8101134A92F90E2002EB41014843C0F38F2012490880104AD17B0A4A127921
:20D80000012383EAD21282F0010002F0EDFC0649097901F07F01074A14E000004471010800
:20D82000F0000020E40B0020B00A002052010020F8060020D00A0020B9010020DC08002086
:20D840005601002092F9102011449DF8202001EBD2010A3101EB8101BE4A92F90F2002EB55
:20D86000410116314843C0F38F20BB49088008460088BA490988401AC01E4FF4806191FB54
:20D88000F0F0B749088054E0B64AD17BB64A1279012383EAD21282F0010002F0A5FCB2499F
:20D8A000097901F07F01AB4A92F9102011449DF8202001EBD201173901EB8101A54A92F9A4
:20D8C0000E2002EB41014843C0F38F20A3490880A44AD17BA44A1279012383EAD21282F0F0
:20D8E000010002F081FCA049097901F07F01994A92F9102011449DF8202001EBD201153907
:20D9000001EB8101934A92F90F2002EB410116314843C0F38F2090490880084600888F4990
:20D920000988401AC01E4FF4806191FBF0F08C4908808E480078C0F3800078B98C48008823
:20D9400000908748008803B28448028800210846FAF748F86043800A04B20EE08448008810
:20D9600000907F48008803B27C480288FF213C20FAF738F86043800A04B27E488480B0F9D2
:20D980000400002802DC00207A4988807848008872490988884220DD7648B0F9040075490E
:20D9A000B1F90610401A022806DD7248C088401C00B27049C88033E06E48B0F904006D4903
:20D9C000B1F90610401AB0F1FF3F29DA6948C088401E00B26749C88022E000BF6548B0F933
:20D9E00004006449B1F90610401A022807DD6148C1880498084400B25E49C88010E05D483E
:20DA0000B0F904005B49B1F90610401AB0F1FF3F06DA5848C1880398081A00B25549C8809E
:20DA20005448B0F90600062801DA062002E05148B0F906004F49C8804D4800884649098825
:20DA4000884208DD01204B4908700020C8804A4802F005FC02E0484802F0F4FB474A117B8D
:20DA6000404AD088464A128801F034F881464448A0F8009001231A4642480188484601F0EC
:20DA800081F940490880384A517A364A907D01F00FF80290344A527A0F3A91B2314A507D79
:20DAA00001F006F80190DDE9011048434FEA902B1FFA8BF001231A463349098801F062F91F
:20DAC00031490880274AD17B274A127A012383EAD21002F05BFB2D4909884843642190FB2D
:20DAE000F1F0801200B200901E480089C111284A009804F09FF8274908801E48B0F906000E
:20DB00002049098848434FEAA0281F48008808FB00F04FEAA0281F48B0F9000040444FEACF
:20DB20006008B8F1000F01DA002000E0404600B2ADF8160001208DF81A0004208DF814007A
:20DB40000598CAF800000698CAF804000BB0BDE8F08F0000D00A0020580100205601002039
:20DB60005A010020DC080020B00A0020B9010020EC030020F000002000010020F00A002018
:20DB80005C0100205E0100206001002052010020F8060020500100202DE9FF4F8BB08146A0
:20DBA0008A46FE4903C9CDE9090100200890834605900490FA48A0F802A0FA480088C828E2
:20DBC00001DA642002E0F748008880100690F44841880698814204DBFCF716FEF249086028
:20DBE00020E0F248B0F90200C82807DDEF48B0F90200EF4991FBF0F086B201E04FF496668E
:20DC0000B6F5FA7F02DA4FF4FA7000E030460646FCF7FAFDE4490968401AB04202D90120E5
:20DC2000DF490870E14800883C2812DDDD480088C82801DA96200AE0DA480088B0F52F7F2B
:20DC400002DD40F20D2002E0D64800884010079010E0D4480088C82801DA962009E0D14800
:20DC60000088B0F52F7F02DD40F20D2001E0CD4800880790CA4841880798814202DB00203C
:20DC8000C7490870CB484078012802D0C948807810B90120C2490870C148007801283ED107
:20DCA000BF48B0F90610C4484079002801DA032007E0C1484079052801DD032001E0BE48F5
:20DCC0004079401EBD4A105C81420CDC0020B449C880BB4802F0C3FA0120BA49087000203C
:20DCE000B9490880BBE3AE48B0F90610B2484079002801DA032007E0AF484079052801DDCC
:20DD0000032001E0AC484079401EAC4A105C081A00B2A349C880AA4802F094FA9FE3A049AD
:20DD20000E984880A148B0F90200B0F5FA7F23DDA04800780F281FDB08464088C8281BDD34
:20DD40009A48B0F90200642148439A49097890FBF1F09E4908609E4800680968C0EB01306C
:20DD60009B49096801EBA0209949086008460068C0F30F30974908800D9803287DD004DC4B
:20DD8000012807D0022879D15FE0042877D03328F9D192E19048007A002801DC012001E06C
:20DDA0008D48007A08908C4890F809B0DFF8F0C1BCF802308446BCF80220BCF80010BCF8E1
:20DDC00000C04FEA6C00F7F70BFC754949884843800A04B280488088A04202DD7E48808830
:20DDE00000E0204604B27C48C088A04202DA7A48C08800E0204604B2774840896E49097A95
:20DE000048434FF47A714843401400EBC00101EB00104FF6FF7101EA8005012305226F489B
:20DE20000188284600F0AEFF6C4908806A48C08840426B490861002048616748C088800236
:20DE4000404288610020C861A4E16348007D002801DC012001E06048007D08905E4890F86F
:20DE600015B0DFF83CC1BCF802308446BCF80E20BCF80C10BCF80CC002E045E085E1C3E017
:20DE80004FEA6C00F7F7ACFB454949884843800A04B25148008AA04202DD4F48008A00E039
:20DEA000204604B24C48408AA04202DA4A48408A00E0204604B24848C08A3F49097A484362
:20DEC0004FF47A714843401400EBC00101EB00104FF6FF7101EA8005012305223F4801880D
:20DEE000284600F04FFF3D4908803B48408A40423B490861002048613748408A8002404296
:20DF000088610020C86145E1334890F82000002801DC012002E0304890F8200008902E4850
:20DF200090F821B0DFF878C0BCF802308446BCF81A20BCF81810BCF818C04FEA6C00F7F7E0
:20DF40004FFB174949884843800A04B22248808BA04202DD2048808B00E0204604B21E4870
:20DF6000C08BA04202DA1C48C08B00E0204604B21948408C1049097A48434FF47A714843A0
:20DF8000401418490978484385B20123052213480188284600F0F6FE104925E05C710108D4
:20DFA000F0000020BA01002068010020DC08002020550300BC030020B00A00200101002096
:20DFC0000001002071010020720100207C01002080010020FE010020E40B00206E01002000
:20DFE000F8060020EE0000200880F748C08B4042F649086100204861F348C08B8002404266
:20E0000088610020C861C5E0EF4890F82C00002801DC012002E0EC4890F82C000890EA4884
:20E0200090F82DB0DFF8A8C3BCF802308446BCF82620BCF82410BCF824C04FEA6C00F7F77C
:20E04000CFFAE34949884843800A04B2DE48008DA04202DDDC48008D00E0204604B2DA48EC
:20E06000408DA04202DAD848408D00E0204604B2D548C08DD749097A48434FF47A714843DB
:20E080004014D5490978484385B201230522D3480188284600F076FED0490880CA48408D8A
:20E0A0004042CA49086100204861C748408D8002404288610020C8616CE0C34890F8380070
:20E0C000002801DC012002E0BF4890F838000890BD4890F839B0BE484088B0F5FF7F15DA83
:20E0E000DFF8ECC2BCF80230DFF8DCC2BCF80E20BCF80C10BCF80CC04FEA6C00F7F770FA11
:20E10000B34949884843800A04B207E0B04840884043AD49498EB0FBF1F004B2AA48808E2E
:20E12000A04202DDA848808E00E0204604B2A648C08EA04202DAA448C08E00E0204604B2F4
:20E14000A148408FA349097A48434FF47A7148434014A1490978484385B2012305229F48A1
:20E160000188284600F00EFE9C4908809648C08E404296490861002048619348C08E8002D5
:20E18000404288610020C86104E0002008908346002400BF00BF924890F90E00322805DC18
:20E1A0008F4890F90E0010F1320F02DA00208C4988738B4890F90F00322805DC884890F9E4
:20E1C0000F0010F1320F02DA00208549C873854AD17B804A1279012383EAD21282F0010091
:20E1E00002F002F87B49097901F07F017C4A92F91020114401EB8101794A92F90E2002EBCF
:20E2000041014843C0F38F2077490880754AD17B704A1279012383EAD21282F0010001F05E
:20E22000E3FF6C49097901F07F016D4A92F91020114401EB81016A4A92F90F2002EB410182
:20E2400016314843C0F38F20684908800846008865490988401AC01E4FF4806191FBF0F074
:20E26000634908806348008800900846008803B25D48028800210088F9F7B4FB6043800A78
:20E2800004B253488480B0F90400002802DC00204F498880574800885349098801EB8101F4
:20E2A000B0EB410F20DD4A48B0F904004849B1F90610401A022806DD4548C088401C00B29C
:20E2C0004349C880ADE04248B0F904004049B1F90610401AB0F1FF3F05DA3D48C088401E1A
:20E2E00000B23B49C8809CE000BF43480078012858D138484078032805D100203F490880A7
:20E300003D4908708DE033484078012805D14FF4967005901E20049003E0642005900A208A
:20E32000049036480088401C34490880084601880598814230DC2648B0F904002449B1F96D
:20E340000610401A022815DD2C480188049891FBF0F0C0F10A002949098891FBF0F200FB05
:20E36000121078BB1A48C1880898084400B21849C88056E01648B0F904001549B1F90610F7
:20E38000401AB0F1FF3F4CDA1148C088A0EB0B0000B20F49C88044E0002018490880164909
:20E3A00008703EE00A48B0F904000949B1F90610401A022824DD0648C1880898084400B2FC
:20E3C0000349C8802DE00000E40B0020F8060020F0000020B00A0020EE0000206E010020E8
:20E3E000D00A0020DC080020840100208601002088010020EC0300207101002072010020F6
:20E400005248B0F904005149B1F90610401AB0F1FF3F06DA4D48C088A0EB0B0000B24B4989
:20E42000C8804A48B0F90600062801DA062002E04648B0F906004549C8804548008845498C
:20E440000988884208DD0120404908700020C880414801F004FF02E03F4801F0F3FE3F4AA1
:20E46000117B3F4AD0883F4A128800F033FB80463C48A0F8008001231A463B480188404676
:20E4800000F080FC38490880384A517A344A907D00F00EFB0290354A527A0F3A91B2304A53
:20E4A000507D00F005FB0190DDE901104843810A0391039988B201231A462D49098800F03C
:20E4C00061FC2B490880264AD17B284A127A012383EAD21001F05AFE26490988484364215D
:20E4E00090FBF1F0801200B200901D480089C111214A009803F09EFB204908801348B0F998
:20E500000600194909884843871219480088784387121A48B0F9000038444710002F01DAB9
:20E52000002000E0384600B2ADF8260001208DF82A0002208DF824000998C9F800000A9841
:20E54000C9F804000FB0BDE8F08F0000F0000020EC0300208601002000010020F00A002012
:20E56000DC0800207401002076010020B00A0020780100206E010020F80600206C010020BE
:20E580002DE9FF5F82460E468C4903C9CDE90201002700BF0025002E40D1A9468848C07F49
:20E5A00008B9872001E08648C07F8146854840680A21C1EB4911884205D282484068401C29
:20E5C0008049486010E07F4840680A2101EB4911884205D97B484068401E7A49486003E03B
:20E5E0004FEA491077494860774AD17B744A127A012383EAD21001F0C9FD7149097A4FF420
:20E60000FA7251434843401400906F480089C1116E4A009803F00EFB044655E06C48408832
:20E62000400141F2883190FBF1F0C5B2012D01DA012000E0284605466548408840016549A3
:20E6400009784843642190FBF1F00A385D494968884205D95B48406828445A49486026E074
:20E660005B48408840015B4909784843642190FBF1F00A305349496888420DD251484068DC
:20E68000A84205D94F484068401B4E4948600EE000204C4948600AE04D48408840014D4970
:20E6A00009784843642190FBF1F046494860464A1289D111424A127A4FF47A735A43D01153
:20E6C000424A03F0B7FA04463F4AB2F902103D4A5268520910B2404A03F0ACFA074638195B
:20E6E00007B236BB4FF000093548807F08B93C2001E03348807F814633480088A9F10501CA
:20E700008AB2009088B280230021F9F76BF97843800A07B22C480088484506DD00202949DF
:20E7200048602E4801F09BFD02E02C4801F08AFD02E02A4801F086FD254A117B224AD088DD
:20E74000274A128800F0C6F980462548A0F8008001231A4623480188404600F013FB21494E
:20E760000880174A517A184A907D00F0A1F9019001231A461C480188019800F003FB1A4900
:20E7800008801848008878434FEAA02B084600880BFB00F04FEAA02B0FFA8BF0ADF80C0045
:20E7A00001208DF80E008DF808000298CAF800000398CAF80400BDE8FF9F00004C71010852
:20E7C000B00A0020F8000020DC080020B0060020F00A0020D3010020D40600200001002044
:20E7E00062010020640100206601002070B504460D461646FCF708F83C490968401A64289D
:20E8000070D3FCF701F8394908603948006828443749086037480078401C3649087008460A
:20E82000007808280ADB32480068C0F3CF003249088000202F4908702D490860462C0BDA9F
:20E840002D48008841F27071884205DD2B480088401C2A49088002E0002028490880462C3C
:20E8600005DC2548008841F28831884207DA962E05DA23480088401C2149088002E0002045
:20E880001F4908801D480088B0F5967F05DD00201A49088001201B49087019480088642882
:20E8A00004DD0020164908801649087015480078012814D1462C0EDA04F11E001249087076
:20E8C00008460078642801DD642001E00E4800780D49087006E064200B49087002E064206B
:20E8E000094908700848007870BD0000A4000020A8000020AC000020AE000020B000002063
:20E90000B2000020B4000020B50000202DE9FF4385B0074615469846DDE9109408EA090004
:20E9200000F00103BDF81A10554800782A46049001F0E6FB06462078B04223D0514800783F
:20E9400000BB052601204F4908702078042819D14D480068142806DD0426002008700120F3
:20E960004A4908700EE000204949086049490860494908804449086044490870052601202A
:20E9800040490870062E68D2DFE806F06733574B03683B48007800F0010078B905F00F0380
:20E9A000BDF81A20364800780146029003A8FEF71DFA039820600498606016E03048007885
:20E9C00000F0010088B105F00F000090BDF81830BDF81A202A4800780146029003A8FEF72A
:20E9E00019FD039820600498606000202549087041E02A480078012807D12948B0F902005C
:20EA000040012649486000200870394603A8FFF7B7FD0398206004986060002019490870C1
:20EA200029E0294603A8FEF7C7F903982060049860600020134908701DE01A480389BDF8F3
:20EA400018102A4603A8FFF7A7F8039820600498606000200B4908700DE000BF124801F084
:20EA6000FEFB1248F7F706F8052020700020A0716080A08000BF00BF09B0BDE8F083000022
:20EA8000B90100208A010020400100204401002008010020200100203C010020F80000204C
:20EAA000DC080020BC030020000100208C01002010B502464FF480608A4208DD01FB01F4D3
:20EAC000A302B3FBF2F4B4FBF2F4A0B201E04FF4806010BDF0B503460E4615460021002463
:20EAE0004FF48060182E04D0242E12D0302E34D121E0E721FC2401EBC10707EB0117B3EBBD
:20EB0000870F02DD4FF4806701E0B3FBF1F73A4625E04FF4A5714FF4B47401EBC10707EBF0
:20EB20000117B3EB870F02DD4FF4806701E0B3FBF1F73A4613E040F2AD114FF4EA7401EB19
:20EB4000C10707EB0117B3EB870F02DD4FF4806701E0B3FBF1F73A4601E0642200BF00BFCA
:20EB600002FB02F74FF0640CB7FBFCF75743B7FBFCF75743BF0242F2107CB7FBFCF2B2F5AA
:20EB80004D7F02D24FF44D7700E017463A46AA4201D290B200E0284604EBC40707EB0417FB
:20EBA000B3EB870F01DD4FF48060F0BD2DE9F04105460E4617461C46002F7DD1552D66D198
:20EBC0004748007820BBFBF71FFE45494968401AB0F57A7F15D9012041490870002020704C
:20EBE00040480078C043404908703E484078C04348703E48007820F00200801C3B49087070
:20EC000018E03A48007820F002003849087011E00020207033480078C043334908703148F3
:20EC20004078C04348703148007820F00200801C2E490870AA2E06D12C48007820F0040024
:20EC40002A49087023E02A480078C8B9FBF7DCFD27494968401AB0F57A7F0AD90120244906
:20EC600008702248007820F00400001D1F4908700DE01E48007820F004001C49087006E087
:20EC80001A48007820F00400001D1849087019480078E0B9FBF7B8FD16494968401A41F2DA
:20ECA000883188420CD90120124908700F48007820F00100401C00E010E00C4908700DE032
:20ECC0000A48007820F001000849087006E00748007820F00100401C04490870BDE8F0819B
:20ECE000DC010020DA000020DC000020B0010020E4010020EC010020012013490870002029
:20ED00004860012011490870002048808880C8800F4908600F4908600F4908600F49086020
:20ED20000F4908600F4908600F4908600F4908620F4908620F4908620F4908620F490862C9
:20ED40000F49086270470000F8000020F000002004000020080000200C000020100000206A
:20ED600014000020180000201C00002068060020440600208C060020F8060020D406002029
:20ED8000B006002070B504461546661A32B2002A06DDAA4202DB4E19B0B20CE020460AE094
:20EDA000002A07DA56429E4202DBCE1AB0B202E0204600E0204670BD10B5FBF725FD2E499E
:20EDC0000968401A642855D3FBF71EFD2A4908602A4800782A4908702A4800784870002035
:20EDE0008870C8702848008800B288802748008800B2C880264840880881254800884881C3
:20EE000024480088888123484088C88122480089088222480068801200B24882204800684C
:20EE2000801200B2888215480078022803D113484088C8821EE011480078012804D10F4820
:20EE400080880F49C88215E00C48007804280ED11448007800F0010020B9084880880849F5
:20EE6000C88207E0054840880549C88202E000200349C88210BD000084000020DE000020AD
:20EE8000FC0800203000002004000020080000202C00002022050020BC0300201000002010
:20EEA0000C000020B901002070B505460E46144608216748FBF796FC664908704FF4004127
:20EEC0006548FBF78FFC6549087062480078644909784840634908705E48007860490870A7
:20EEE0005E480078604909784840604908705B4800785D4908705748007858490978484027
:20EF00005B490870FBF780FCB0F57A7F0CD2FBF77BFC58490860FBF777FC57490860FBF71A
:20EF200073FC5649086070BD2088C0F38030002878D1B5F5966F7CDD462E7ADD49480078D6
:20EF400000BBFBF761FC4B490968401A42F2107188421BD9206820F4804000F58040206044
:20EF60000120474948800846F8F7B2FA00204549087045484088401C434948800220434956
:20EF80000870D0E7FBF740FC3A4908603748007800BBFBF739FC38490968401A41F2883118
:20EFA00088421BD9206820F4804000F5804020600220334948800846F8F78AFA0020314941
:20EFC000087031484088401C2F49488002202F490870A8E7FBF718FC274908602448007879
:20EFE00010BBFBF711FC25490968401A41F2883188422AD9206820F4804000F580402060C4
:20F0000003201F4948800846F8F762FA00201D4908701D484088401C1B49488002201B49CB
:20F02000087080E711E004E0FBF7EEFB134908600BE0FBF7E9FB0F490860FBF7E5FB0E49D3
:20F040000860FBF7E1FB0D49086000BF6BE70000000C0140D402002000080140D502002028
:20F06000BD020020BC020020C5020020C4020020CC020020C0020020C8020020D00200205A
:20F08000880700209D030020300B0020BE0100201FB53848007890B93748807E55280ED1D9
:20F0A000364A374800783749498889B2CDE9010200913549887835490EC900F0A5FE2F4925
:20F0C0002F480078CDE9010130488068304A00901178304A10892D4A0CCA00F02DFF2748AB
:20F0E00001902D488088ADF80000264B5B889AB2244B1989224B9879274B1C6802949B887F
:20F10000ADF80C30234600F09FFD1E4A917D507D1A4A00F01BFD1F498889184900F074FA32
:20F120001D48016802918088ADF80C00134ADDE9020100F0D1FB114800F03CF80F48134AA2
:20F14000009011780F4A528890B2144A12680392134A1388039A00F093FC08481149009066
:20F160004A8911490878114B1149098800F00EFB1FBD0000D8000020B00A00208C01002047
:20F18000DE000020DC080020EC030020BC030020DA000020501D002032050020220500205A
:20F1A000FE010020621D0020D4010020D3070020D001002010B50446FBF726FB41F28831A3
:20F1C00088420CD2FBF720FBEE490860FBF71CFBED490860FBF718FBEC49086010BD20683D
:20F1E000C0F3804000286FD14FF40041E848FBF7F9FA00BBFBF708FBE3490968401A41F2C1
:20F20000883188421BD9206820F4802000F5802020600120DF4948800846F8F759F9002066
:20F22000DD490870DD484089401CDC4948810220DB49087003E0FBF7E7FAD3490860D948DF
:20F240000088002847D1D8480078012843D1D748007805283FD0D548807901283BD1D348D8
:20F26000B0F90400C82804DCD048B0F90200C82831DDCF48807A40BBCE480089C82825DAB6
:20F28000FBF7C2FAC1490968401A41F28831884225D9206820F4802000F5802020600220C4
:20F2A000BC494880BF48008888800846F8F710F90020B9490870B9484089401CB74948811B
:20F2C0000220B74908700AE08DE0FFE7FBF79CFAAE49086003E0FBF797FAAC490860FBF7BB
:20F2E00093FAA8490968401A14287CD3FBF78CFAA4490860B048C088B04909680844AF497F
:20F300000860AF480088AF4909680844AD490860AB484088AC4909680844AB490860A8483A
:20F320008088AA4909680844A8490860A8480078401CA74908700846007820287EDB002009
:20F3400008709E4800684FF4FA71B1EB501F2FD89A480068C900B1EB501F29D399480068C4
:20F3600041F28831B1EB501F22D8964800684EF66021B1EB501F1BD39348006841F2883169
:20F38000B1EB501F14D8904800684EF66021B1EB501F0DD38D48006841F28831B1EB501F52
:20F3A00006D88A4800684EF66021B1EB501F16D2206820F4802000F580202060032075494B
:20F3C00048800846F8F784F800207349087073484089401C714948810220714908707D48DC
:20F3E0000068C82100E0C2E0B1EBA02F36DA7A48008872490968C0EB511019282AD2774841
:20F400000078401C75490870084600780A2828DD206820F4802000F58020206004205D49CA
:20F42000488066480068C0F34F1088800846F8F74FF8002058490870584800E01AE04089D4
:20F44000401C5649488102205549087000206349087006E000206149087002E000205F499A
:20F4600008700020554908605649086056490860564908604F48407B00287AD14D484088B7
:20F48000002876D1FBF7C0F955490968401A41F28831884274D94848C0885249524A12784D
:20F4A00021F812004648008850494F4A127821F81200434841884E484B4A127820F81210E1
:20F4C0003F4881884B48484A127820F8121046480078401C444908700846007832284FDB02
:20F4E0000020087032213F48F8F79AFF4249086032213E48F8F794FF4049086032213C48FC
:20F50000F8F78EFF3E49086032213A48F8F788FF3C49086038480068B0F5FA7F0DD83748DE
:20F52000006842F6E061884207D835480068884203D834480068884222D9206820F48020D2
:20F5400000F5802020600520124948802A48008888800846F7F7BCFF00200F4908700F480E
:20F560004089401C0D49488102200D49087007E0FFE700201C490870FBF746F91849086093
:20F5800000BF2BE660020020640200206802002000100140880700209D030020300B0020EE
:20F5A000BE010020C801002030000020DE000020C8070020DC080020621D00207002002011
:20F5C0001A05002074020020780200207C0200206C0200200C000020380500206D02002078
:20F5E00094020020C6120020800200202A1300208E130020F2130020840200208802002028
:20F600008C020020900200207047000013B50C465448007860B9FBF7F7F8534908609DF812
:20F62000012006215148F4F74CFA01204D4908702078C0F3C01000287ED19DF8000018B199
:20F640009DF80000072821D1FBF7DEF846490968401AB0F57A7F1DD9206820F08000803076
:20F6600020600120424948809DF8000088800846F7F72EFF00203F4908703F48C08A401C43
:20F680003D49C88201203D4908701CBDFBF7BCF8354908609DF800009DF8011088425FD0E2
:20F6A0009DF80010364802780078401C344B18702E48815418460078062851DB00201946D8
:20F6C000087006212948F5F755FF28B92D480068401C2C49086006E000202A490860FBF710
:20F6E00093F82949086027480068322838D9FBF78BF82549096801F5FA71884230D9206853
:20F7000020F08000803020600220194948801748007800021549497800EB0110134989788C
:20F720000844134988801148C07800020F49097900EB01100D4900E012E0497908440C4925
:20F74000C8800846F7F7C4FE00200A4908700A48C08A401C0849C88201200849087094E780
:20F7600000BF92E7A6020020A8020020B0020020880700209D030020000B0020BE01002074
:20F78000B6020020B8020020AC0200202DE9F04105460E4614469846069FFBF735F8B0F562
:20F7A0007A6F01D2BDE8F081FBF72EF842F21071884220D23868C0F3804000287CD1FBF774
:20F7C00023F83E490968401A142875D3FBF71CF83A49086098F80000A8BB0DB1C82E0BDDB8
:20F7E00040F2C270844207DD40F63E00844203DA0020334908705FE031480078401C3049CB
:20F80000087008460078FA2856DB00200870386820F4802000F580203860082029494880DC
:20F8200005EB860088800846C480F7F751FE00202549087025484089401C2449488102208B
:20F840002349087038E0FFE70DB1C82E03DD002088F8000030E040F68B60844202DCB4F514
:20F86000BA7F26DA1B480078401C1A49087008460078FA2820DB00200870386820F480206E
:20F8800000F58020386009200E49488005EB860088800846C480F7F71BFE00200A490870F1
:20F8A0000A484089401C0949488102200849087002E000200749087000BF73E7A002002026
:20F8C000A4020020880700209D030020300B0020BE010020A502002037B51446604800788C
:20F8E00001280CD0FAF790FF5E490860FAF78CFF5D490860FAF788FF5C4908603EBD2068E2
:20F90000C0F30040002875D1BDF90000002801DB014600E0414244F62062914228DDFAF79D
:20F9200073FF50490968401AB0F57A7F24D9206820F4803000F58030206001204C49488067
:20F94000BDF90000002801DB014600E04142484A91801046F7F7BCFD0020464908704648EE
:20F96000C088401C4449C880022044490870C5E7FAF74AFF3B490860BDF90200002801DB59
:20F98000014600E0414244F62062914228DDFAF73BFF35490968401AB0F57A7F24D9206892
:20F9A00020F4803000F580302060022030494880BDF90200002801DB014600E041422C4A1F
:20F9C00091801046F7F784FD00202A4908702A48C088401C2849C8800220284908708DE7F8
:20F9E000FAF712FF20490860BDF90400002802DB014601E031E0414244F62062914228DD25
:20FA0000FAF702FF19490968401AB0F57A7F24D9206820F4803000F580302060032014493B
:20FA20004880BDF90400002801DB014600E041420F4A91801046F7F74BFD00200D490870B2
:20FA40000D48C088401C0C49C88002200B49087054E7FAF7D9FE0549086000BF4EE7000075
:20FA600030000020480200204C02002050020020880700209D030020300B0020BE01002043
:20FA80002DE9FF4105460E461F460A9C2068C0F3805000284BD1FAF7B7FE26490968401A37
:20FAA000142844D3FAF7B0FE22490860B5F5FA7F3ADD0F2E38DBBDF80800C82834DDBDF884
:20FAC0000A00322830DA40F2DC50874228DD1A480088401C1849088008460088FA2826DB64
:20FAE00000200880206820F4800000F580002060002012494880BDF808008880BDF80A0086
:20FB0000C8800846F7F7E4FC00200D4908700D480089401C0B49088102200B49087006E0A8
:20FB200000200549088002E0002003490880BDE8FF810000980200209C02002088070020AD
:20FB40009D030020300B0020BE01002070B504460E461546FAF758FE41F28831884201D3BC
:20FB60005A2C08DDFAF750FE31490860FAF74CFE2F49086070BD2888C0F34020002855D1A0
:20FB8000052C01DBBE2C22DDFAF73EFE28490968401A41F2883188421DD9286820F4007046
:20FBA00000F50070286001202249488008468480C680F7F78DFC00201F4908701F48408BC3
:20FBC000401C1E49488301201D490870D2E7FAF71BFE17490860052E01DBBE2E22DDFAF722
:20FBE00013FE18490968401A41F2883188421DD9286820F4007000F50070286002200D49A3
:20FC0000488008468480C680F7F762FC00200A4908700A48408B401C084948830120084946
:20FC20000870A7E7FAF7F0FD0649086000BFA1E740020020880700209D030020000B0020E6
:20FC4000BE010020440200200FB42DE9F04105460E4617460B9C2088C0F30020002877D1C7
:20FC6000012D76D141F28830864272DDB7F5FA7FFBDDBDF92400002801DB014600E0414288
:20FC8000B1F5967F2CDAFAF7BFFD58490968401A41F28831884227D9206820F4807000F553
:20FCA00080702060012052494880BDF92400002801DB014600E041424D4A91801046F7F7DC
:20FCC00007FC00204B4908704B48008B401C4A490883012049490870BDE8F0015DF814FB38
:20FCE000FAF792FD41490860BDF92600002801DB014600E04142B1F5967F2BDAFAF784FDD6
:20FD00003F490968401A41F28831884226D9206820F4807000F58070206002203449488083
:20FD2000BDF92600002801DB014600E04142304A91801046F7F7CCFB00202E4908702E481E
:20FD4000008B401C2C49088301202C490870C3E73CE03CE0FAF758FD29490860BDF92800CE
:20FD6000002801DB014600E04142B1F5967F29DAFAF74AFD23490968401A41F288318842F2
:20FD800031D9206820F4807000F580702060032017494880BDF92800002801DB014600E014
:20FDA0004142134A91801046F7F792FB0020114908701148008B401C0F49088301200F49F3
:20FDC000087089E7FAF720FD0E4908600BE0FAF71BFD06490860FAF717FD09490860FAF713
:20FDE00013FD0849086000BF76E7000034020020880700209D030020000B0020BE0100204F
:20FE0000380200203C0200202DE9FF410646DDE90A870C9C00252078C0F34010002878D158
:20FE2000052F08D1FAF7F0FC3B490860FAF7ECFC3A4908606DE0012F01D0042F32D1B8F1FB
:20FE4000320F2ADD4EBB364890FBF8F085B242F21070854200DA00E028460546FAF7D4FC7A
:20FE60002D490968401AA84253D9206820F020002030206001202B4948800846F7F728FBE7
:20FE80000020294908702948408A401C27494882012027490870BDE8FF81FAF7B5FC1E4950
:20FEA000086036E09DF8040005282EDB9DF8050058BB56BB9DF804001E4991FBF0F085B294
:20FEC00042F21070854200DA00E028460546FAF79BFC12490968401AA8421AD9206820F011
:20FEE00020002030206002200E4948800846F7F7EFFA00200C4908700C48408A401C0B49F1
:20FF0000488201200A490870C5E7FAF77DFC0349086000BFBFE700001C020020200200207C
:20FF200048F13E00880700209D030020000B0020BE010020D8B805000FB42DE9F0410446E8
:20FF40000F46DDE90B85FAF75FFC41F28831884207D350480078012803D04E4800780228D6
:20FF600007D1FAF751FC4C490860FAF74DFC4B490860FAF749FC4A490968401A14287DD318
:20FF8000FAF742FC46490860002607E04549701C31F8100021F81600701C86B2182EF5D3DA
:20FFA000404804862878C0F3801000286FD119213C48F8F735FA3C490860222F37D007F0CC
:20FFC0000F0098B39DF820001E2830DD9DF8210060BBB8F1020F2AD1084600680A2826D259
:20FFE000FAF712FC2C490968401A43F69821884221D9286820F040004030286001202B499F
:020000040801F1
:2000000048802948008888800846F7F761FA0020274908702748808A401C26498882012009
:2000200025490870BDE8F0015DF814FBFFE7FAF7EBFB19490860322C03DB40F6D2708442DF
:2000400021DDFAF7E1FB15490968401AB0F57A7F1DD9286820F040004030286002201349C2
:20006000488008468480F7F733FA0020104908701048808A401C0F49888200E007E0012052
:200080000D490870CEE7FAF7BFFB0449086000BFC8E70000D8000020240200202802002087
:2000A00030020020941200202C020020880700209D030020000B0020BE01002010B50C4947
:2000C000487B01F0D1FC0A49487B05F0C9FA094803F060FC0748F5F7CDFC07480189074805
:2000E00004F0D4FD01F0C0FE012001F0E9FE10BDB00A00208C010020501D0020621500201B
:200100002DE9FF410E4615461F461D48006850BB25B3012F22D1FAF777FB40F6B831884256
:200120001CD9C82E0BDD9DF80000552807D09DF80000F82801D1012411E004240FE0642EBD
:200140000DDA222D01D1012409E005F0F00018B1332D01D0032402E0022400E00524012051
:2001600001F0AEFE08E0052400200649087008460078C04304490870204604B0BDE8F0812C
:200180008C010020DA000020DC00002010B502464FF480630AB9184610BD022902DC4FF44F
:2001A00080731FE0062906DC881E4FF4807404EB801083B216E0162908DC881F00EB4000C0
:2001C0004FF4007404EBC00083B20BE01E2907DCA1F116004FF4607404EB001083B201E09B
:2001E0004FF480631846D7E710B502464FF480630AB9184610BD022902DC4FF400731FE0DE
:20020000062906DC881E4FF4007404EB401083B216E0162908DC881F00EB80004FF42074FA
:2002200004EB800083B20BE01E2907DCA1F116004FF4707404EBC00083B201E04FF480634B
:200240001846D7E710B50446207838B9F7F7DEF8FCF73EF8F7F772FA0120207010BD10B560
:20026000044601F021FFF7F757FAFEF745FD0020207010BD2DE9F04107460D46144605EBFF
:200280004500C0F34F06207800F0010050BBB74203DAFAF7B9FA1C490860FAF7B5FA1A4933
:2002A0000968401A41F2883188422AD9206820F00100401C206002201449488008468680AA
:2002C000F7F706F900201249087012480089401C10490881012010490870FAF795FA0F4953
:2002E00008600EE0FAF790FA0C490968401A41F28831884205D90A48006820F0010008495D
:200300000860BDE8F081000008030020880700209D030020000B0020BE0100200C0300208C
:200320008C0100201CB52C492C48808BC0F30B0010B940F6B83001E02848808B284CCDE920
:200340000001237B274C247814B9274C248801E0264CE4882246254CE17B224C207800F019
:20036000FFF92248008941F2883188420DDA1C4A117B2246127812B91B4A128801E01B4A01
:20038000D2881046144A00F0FFF8194A917A174A1089114A00F060F90F48104C0090A37AFC
:2003A000124CA27D617DE07D00F04EF822461189D088094A00F0ACFA084A127A02EB4203FC
:2003C000C3EBC2124FF6FF7303EAC20122461089014AFFF74FFF1CBD8C010020B00A002044
:2003E000F00A0020EC0100207C090020DC080020C807002070B504460D46207868B90020A3
:200400000F4908700F480078C0B90E480078401C0C490870F6F7E0FF10E000200949087027
:2004200007480078012802DB0020207001E0F6F725FD03480078401C0149087070BD000041
:2004400010030020110300202DE9F04180460E4617461C46069DFAF7D7F940F6B8318842C8
:2004600007D2FAF7D1F940490860FAF7CDF93F4908602878C0F3001000283DD13C48C07AF9
:2004800058B9A4F11900B04215DD2330874212DAFAF7BAF9344908600DE0A4F11900B0429B
:2004A00009DD2330874206DA1E38404503DDFAF7ABF92D490860FAF7A7F92B490968401A5C
:2004C00041F2883188424CD9FAF79EF927490860286820F01000103028602648F6F7F8FF17
:2004E0000020254908702548008A401C2349088201202349087034E01D48C07AB8B9A4F1EF
:200500002300B0422DDD0F30B8422ADDFAF77CF916490968401A1B49884222D9286820F023
:2005200010002860FAF770F90F49086019E0A4F12D00B04215DD1930B84212DD0A38404571
:200540000FDDFAF761F909490968401A0D49884207D9286820F010002860FAF755F9024985
:200560000860BDE8F0810000F8020020FC020020C8070020880700209D030020000B00203C
:20058000BE010020E09304002DE9F04105460E4614460027182E04D0242E05D0302E09D125
:2005A00005E047F60C3707E04AF6C87704E04EF2844701E02F4600BF00BF2078C0F38000E2
:2005C00030BBBD4203DCFAF71FF91D490860FAF71BF91B490968401A41F28831884212D9A6
:2005E000206820F00400001D20601648F6F770FF00201549087015488089401C13498881EB
:20060000012013490870FAF7FFF81249086014E0A7F5FA70A84203DAFAF7F6F80D490860DC
:20062000FAF7F2F80B490968401A41F28831884203D9206820F004002060BDE8F0810000FC
:20064000E4020020880700209D030020000B0020BE010020E802002070B505460E461446F3
:200660002078C0F3C000002849D1012E08D1FAF7CBF831490860FAF7C7F83049086014E00A
:2006800040F6C410854208DAFAF7BEF82A490860FAF7BAF82949086007E041F64C50854227
:2006A00003DAFAF7B1F825490860FAF7ADF822490968401A41F28831884208D8FAF7A4F8FE
:2006C0001E490968401A40F6B831884232D9206820F00800083020601948F6F7F9FE002037
:2006E000184908701848C089401C1749C881012016490870FAF788F8154908601AE0FAF759
:2007000083F813490968401A41F28831884211D91048007870B9104800880A280ADA0E4852
:2007200040880A2806DA0D48807818B9206820F00800206070BD0000EC020020F002002054
:20074000880700209D030020000B0020BE010020F4020020DA00002022050020BC030020EA
:200760002DE9F0478046894615469A46DDE9086400270120B0EBE63F4ED12078C0F3400078
:20078000A0BBB9F1010F03DBFAF73EF85A490860FAF73AF858490968401AC6F3023101EBCD
:2007A0008101052202EB410101EB4102C2EBC111B0EBC10F15D9206820F00200801C2060A4
:2007C0004E484580A0F80480F6F782FE00204C4908704C484089401C4A49488101204A493F
:2007E0000870FAF711F84949086082E0FFE7B9F1050F03DAFAF708F844490860FAF704F8D7
:2008000042490968401A41F28831884271D9206820F0020020606CE0BAF1180F06D0BAF1C9
:20082000240F08D0BAF1300F12D10AE0C6F30B00C0EBC0070EE0C6F30B0000EB800047005C
:2008400008E0C6F30B0000EB800101EBC00701E02F4600BF00BF2078C0F3400098BBBD421C
:2008600003DBF9F7D1FF24490860F9F7CDFF22490968401AC6F3023101EB8101052202EBA5
:20088000410101EB4102C2EBC111B0EBC10F15D9206820F00200801C206018484580A0F89C
:2008A0000480F6F715FE00201549087015484089401C14494881012013490870F9F7A4FF8E
:2008C0001249086015E0FFE707F57A70854203DAF9F79AFF0D490860F9F796FF0B4909685F
:2008E000401A41F28831884203D9206820F002002060BDE8F0870000DC0200208807002029
:200900009D030020000B0020BE010020E00200202DE9F0410746884614460026F9F774FFC6
:200920002B490968401A642850D3002507E02949681C31F8100021F81500681C85B2092D6F
:20094000F5D3244847820A21F7F76AFD06462068C0F3404090BBB8F1320F2BDAB6F57A7F35
:2009600028D91D480078322830DD206820F4003000F500302060C6F30F20184948800A2185
:200980001448F7F7C1FC154988800A211148F7F7CCFC1249C8800846F6F79AFD00201049C2
:2009A000087010480089401C0E49088102200E4908700BE000200849087007E0FFE7B6F565
:2009C0007A7F03D8206820F400302060BDE8F0810003002040070020040300208807002081
:2009E0009D030020300B0020BE01002010B5F9F70BFFA2490968401AC8287DD3F9F704FF55
:200A00009E4908609E480088C01268B99D480089FA2148439C49097A4FF47A725143B0FB3C
:200A2000F1F09849888016E095480088C0F30A0093490988012202EBE1214843401191499F
:200A4000098948439049097A4FF47A725143B0FBF1F08C4988808B488088142801DA0020DF
:200A600001E08848808887498880884840780873874800881C2190FBF1F08249C872854810
:200A8000007848738348407888738348007800F0010040B17A48037B0846C27B7F49804825
:200AA000F3F7C4FE01E07F48407A7649C8737A48007800F0010010B14EF6EE6001E07A480D
:200AC000C08A704908827048807EEE2815D177488078012823D1754880684FF44821B1FB06
:200AE000F0F07349096808447149086008460068000B6E49C86012E0BFE06348807EAA28CF
:200B00000DD1624840686049897948435E49C979B0FBF1F03221B0FBF1F06449C8605A48A4
:200B2000007B594991F91B10084442F2107191FBF0F15E48C0685F4A1268801A814206D849
:200B400001205D4908705948C0685A4908605A48007801283ED100205749087057480068F1
:200B6000401C564908605648406A401C5449486252488068401C51498860084680685149F7
:200B8000884203D900204D498860C8603D48008B401C3C490883494800680A21B0FBF1F0BD
:200BA0003849488248480078401C47490870084600781E280EDB424B30224C21434803F0BF
:200BC0007CF83E4B1022D621404803F076F800203D4908702B4800881E281ADB3C480078B6
:200BE000401C3B49087008460078052814DB0020087038480088401C364908802148408B84
:200C0000401C2049488334480078401C3249087002E000202E4908702F4800783C2811DBD1
:200C200000202D49087025484068401C234948602348C06A401C2249C8622048C068401CAF
:200C40001E49C86023480088B0F5167F0EDB0020204908801A4B30224C211C4803F02DF83E
:200C6000164B1022D621194803F027F80E48808A0A2190FBF1F00349087510BD6C0000205E
:200C8000F00A0020DC080020B00A0020BC03002022050020DA000020B0010020B40900208E
:200CA000340300207C09002014030020EC0300207C0000207000002074000020200C0020E6
:200CC000000B00209F860100800000202C04002075000020780000207600002010B5044601
:200CE000F9F792FD10490968401A4EF66021884218D3F9F789FD0C4908602068401C206040
:200D00000A480078401C09490870084600780A2808DB074B30224C21064802F0CEFF0020CA
:200D20000249087010BD0000C0000020C4000020000B00202C04002010B50446022C1BD1BB
:200D4000F9F762FD0F490968401AC82818D30E4B4FF481520C214FF4E26003F04DF80B4B97
:200D60004BF620220C2140F2157003F045F8F9F74BFD0449086003E0F9F746FD0149086027
:200D800010BD000090000020DC080020FC08002001B511480078022800D108BD0098A0B17E
:200DA000F9F732FD0D490968401AB0F5FA7F10D9F9F72AFD094908606B4641F204120C21F4
:200DC0004FF4E26003F018F803E0F9F71DFD0349086000BFE1E700005D000020880000203E
:200DE00010B50446012C13D1F9F70EFD0B490968401AC82810D30A4B4FF481520C214FF40B
:200E0000E26002F0F9FFF9F7FFFC0449086003E0F9F7FAFC0149086010BD00008C00002012
:200E2000DC08002010B5FBF765FAFBF751FAF4F7DDF903F06DF9FBF737FD054801890548F7
:200E400003F06CFF024881890348F6F7D9FE10BD501D002062150020740400201CB504462D
:200E6000F9F7D2FC40490968401AB0F5FA7F7AD33E480088401C3D4908800846008814286B
:200E800037DB3B48007800F0010010B900203949487437480088C0F3002010B900203549EC
:200EA000087433480078C0F3801010B90020314908812F480078C0F3C01010B900202D49C3
:200EC00048812B480078C0F3001010B900202949888127480078C0F3401010B900202549F6
:200EE000C8814FF480512448F9F784FC00201F4908802248007868B900204FF408430C22CA
:200F000040F2FF7100901E4802F0C2FF01201B49087024E019480078012820D100200190E1
:200F2000184801780078401C164A107005290CDC01A841F20133162240F2FF71009010483C
:200F400002F0A6FF0A20F9F779F941F214030C2240F2FF710A48009402F09AFF00BFF9F734
:200F600053FC014908601CBD9C000020A0000020C8010020D00B0020001001405D00002069
:200F8000F0050020A200002070B504464D48007880BB08214C48F9F725FC4C4908704FF4A5
:200FA00000414B48F9F71EFC4A49087080214A48F9F718FC494908704FF480714648F9F755
:200FC00011FC474908704FF400514348F9F70AFC4449087004214448F9F704FC434908703D
:200FE000002020816081A081E081207460740120344908703E48C08860803D488088A080F4
:201000004FF40060E0803A480089208008212E48F9F7E8FB05462D480078A84202D0208913
:20102000401C2081294805704FF400412848F9F7D9FB054627480078A84202D06089401CE2
:2010400060812448057080212348F9F7CBFB054622480078A84202D0A089401CA0811F4816
:2010600005704FF480711C48F9F7BCFB05461C480078A84202D0E089401CE08118480570DE
:201080004FF400511448F9F7ADFB054615480078A84202D0207C401C20741248057004216C
:2010A0001148F9F79FFB054610480078A84202D0607C401C60740D4805704FF47A70608291
:2010C00070BD00009A000020000C0140940000200008014095000020001001409600002023
:2010E00097000020980000200014014099000020621D002010B5F9F787FB42F2107188421E
:2011000004D2F9F781FB4149086010BDF9F77CFB3E490968401A41F28831884274D3F9F728
:2011200073FB3A4908603A48407D3A4991F82310884207DA3648407D364981F823000020B7
:20114000354908703248407D324991F82210884207DD2F48407D2F4981F8220000202E49A0
:2011600008702B48807D2B4991F82910884207DA2748807D274981F8290000202649087021
:201180002348807D234991F82810884207DD2048807D204981F8280000201F4908701C4839
:2011A000C07D1C4991F82B10884207DA1848C07D184981F82B000020174908701448C07DEB
:2011C000144991F82A10884207DD1148C07D114981F82A0000201049087010480088401C81
:2011E0000E490880084600880C280DDD0A48007850B900200880012007490870054B302216
:201200004C21074802F059FD00BF7EE7C8000020DC080020000B0020CE000020CC000020B5
:201220002C04002010B50748007850B9F9F7ECFA04494968401AB0F5FA6F02D90120014947
:20124000087010BDD401002000B587B0012003900320049003A90E48F9F736F90D4800681F
:20126000806820F001000B490968886000200090082001900720029069460648F7F786FB3A
:2012800020B140F29D2104A004F024FF07B000BD00080140741D00202E2E5C436F72655CC7
:2012A0005372635C6164632E630000000EB550485049086081154F4881600021C1604161A3
:2012C0004FF46021C16100204A494860092149480161F7F771FE18B1592147A004F0FAFE3D
:2012E0000A200090012001900720029069464148F7F74CFB18B163213FA004F0EBFE0B2028
:201300000090022001900720029069463948F7F73DFB18B16D2138A004F0DCFE0C200090C2
:20132000032001900720029069463248F7F72EFB18B1772130A004F0CDFE0D20009004202F
:2013400001900120029069462A48F7F71FFB18B1812129A004F0BEFE0520009001900120D5
:20136000029069462348F7F711FB18B18B2122A004F0B0FE072000900620019007200290C7
:2013800069461C48F7F702FB18B195211AA004F0A1FE0E20009007200190012002906946AB
:2013A0001448F7F7F3FA18B19F2113A004F092FE10200090082001900220029069460D4805
:2013C000F7F7E4FA18B1A9210BA004F083FE11200090092001900720029069460548F7F770
:2013E000D5FA18B1B32104A004F074FE0EBD000000240140741D00202E2E5C436F72655CF9
:201400005372635C6164632E6300000000B589B02348244908608115224881600021C1603E
:201420004161C16100201F49486001211D480161F7F7C2FD18B1C7211BA004F04BFE012058
:201440000190029003200590002003904FF480500890002007900690049001A91148F7F781
:201460008BF818B1D62110A004F034FE02200190029001A90B48F7F77FF818B1DF210AA039
:2014800004F028FE03200190029001A90548F7F773F818B1E82104A004F01CFE09B000BDA2
:2014A00000280140A41D00202E2E5C436F72655C5372635C6164632E6300000010B50F48EC
:2014C0000F4908601220486000210D488160C1604FF4A02101610021416181610121C161AB
:2014E0000021016241628162C162F8F7ABF918B15C2104A004F0EEFD10BD000000640040F2
:20150000A82200202E2E5C436F72655C5372635C63616E2E6300000008B500BF0A48406986
:2015200040F00100084948610846406900F00100009000BF00BF022211460B20F9F733FAC7
:201540000B20F9F723FA08BD0010024000B585B000BF3A48806940F0100038498861084630
:20156000806900F01000009000BF00BF00BF0846806940F0200088610846806900F02000FE
:20158000009000BF00BF00BF0846806940F0040088610846806900F00400009000BF00BFF1
:2015A00000BF0846806940F0080088610846806900F00800009000BF00BF002289142048B0
:2015C000F9F71CF94EF2203001900320029001A91B48F8F779FF40F61870019003200290B8
:2015E00001A91848F8F770FF4EF6024001900320029001A91448F8F767FF4FF480500190B8
:20160000124802900020039001A90F48F8F75CFF4FF480500190012002900220049001A929
:201620000748F8F751FF002211462820F9F7BBF92820F9F7ABF905B000BD00000010024017
:201640000010014000080140000C01400000211010B50848084908600320486040F2E24184
:2016600005488160F9F7D6F818B13A2103A004F031FD10BD00300040F00700202E2E5C4346
:201680006F72655C5372635C697764672E63000000B595B031483249086000204860202189
:2016A0002F4881604FF41661C1600021016101214161FAF753F84FF48050119011A9284896
:2016C000FAF7F4F82648FAF725FB70200F90802010900FA92248F9F7CAFF4FF40060089029
:2016E0004010099000200A9039200B9000200C900D900E9008A91A48F9F77AFF6FF0800001
:20170000174909680861602001904FF496600290002003900490059006900790002201A9DE
:201720000F48FAF773FA042201A90D48FAF76EFA082201A90A48FAF769FA6020019040F6B5
:201740005F10029000200390082004900C2201A90348FAF75BFA15B000BD0000002C0140C1
:20176000901C002000B587B000200390049005900690019002904FF0804019490860002033
:2017800048600021164881604FF6FF71C1600021016141618161F9F7E1FF18B17E2111A07B
:2017A00004F098FC4FF400500390002004900590069003A90A48FAF779F818B1862109A023
:2017C00004F088FC00200190029001A90448F9F74EFF18B18C2103A004F07CFC07B000BD22
:2017E000D01C00202E2E5C557365725C5372635C74696D2E6300000000B589B01C481D4913
:2018000008600020486000211A4881604721C1600021016180218161FAF77CFA20B14FF42A
:201820008F7115A004F056FC00200790089007A91048F9F71CFF20B140F225110EA004F070
:2018400049FC6020009024200190002002900490002269460748FAF7D9F920B14FF4977119
:2018600005A004F037FC0348FAF786F909B000BD00040040101D00202E2E5C557365725C27
:201880005372635C74696D2E6300000010B50C480C4908604FF4165048600021094881606F
:2018A000C16001610C21416100218161C161FAF76FFC18B1462104A004F00CFC10BD0000B8
:2018C00000480040EC2400202E2E5C436F72655C5372635C75736172742E630000BFFEE7CB
:2018E00030B504460A460021002329480078401C274D2870284600780F2841DB00202870E3
:2019000024480089244D2D88411B002907DA214800894FF6FF7528441F4D2D88411B44F678
:201920002060814200DD00211A4800891A4D28804FF47A70414319480068081A174D2D68D7
:2019400005EB2020154D2860284600680314C3EB031040F35C0000B2114D28800D4880891A
:20196000104D2D68C5EB80200E4D2D6805EB60100C4D286028460068C0F38F20054DE88101
:2019800012B90020064D28800548B0F9000030BDAA030020C8070020AC030020B003002020
:2019A000B8030020B40300202DE9F04107460C46154629462046F6F71DFC8046002606E087
:2019C000701C34F8100024F81600701C86B2681EB042F5DC24F810704046BDE8F081704711
:2019E00002480068C0F30220704700000CED00E010B5002807DA0A07140E054A00F00F037E
:201A00001B1FD45403E00A07130E024A135410BD18ED00E000E400E010B5F8F7F5FE40F649
:201A2000B831884216D90C480078012812D10020094908700948C07AAA280BD13320084965
:201A4000087008460078C0430649087004484078C043487010BD0000CF000020B00A002029
:201A6000DA000020DC00002010B50446012C06D0022C23D0032C40D0042C7DD15CE02422FE
:201A80004E494F48F2F70BF824224E494E48F2F706F824224D494E48F2F701F824224D49A2
:201AA0004D48F1F7FCFF24224C494D48F1F7F7FF24224C494C48F1F7F2FF7CE024224B49E2
:201AC0003F48F1F7ECFF242249493F48F1F7E7FF242248493E48F1F7E2FF242246493E48FE
:201AE000F1F7DDFF242245493D48F1F7D8FF242243493D48F1F7D3FF5DE024224149304874
:201B0000F1F7CDFF242240492F48F1F7C8FF24223E492F48F1F7C3FF24223D492E48F1F704
:201B2000BEFF24223B492E48F1F7B9FF24223A492D48F1F7B4FF3EE0242238492048F1F7FA
:201B4000AEFF242236492048F1F7A9FF242235491F48F1F7A4FF242233491F48F1F79FFFB6
:201B6000242232491E48F1F79AFF242230491E48F1F795FF1FE0FFE7242210491048F1F758
:201B80008EFF24220F491048F1F789FF24220F490F48F1F784FF24220E490F48F1F77FFF98
:201BA00024220E490E48F1F77AFF24220D490E48F1F775FF00BF00BF10BD00004C6B010878
:201BC00044060020706B010868060020946B01088C060020B86B0108B0060020DC6B01081D
:201BE000D4060020006C0108F8060020246C0108486C01086C6C0108906C0108B46C0108F3
:201C0000D86C0108FC6C0108206D0108446D0108686D01088C6D0108B06D0108D46D010866
:201C2000F86D01081C6E0108406E0108646E0108886E01082DE9F04304460D46601B06B2F9
:201C4000B2F9000000FB06FC908810B90020106212E0B2F9040000FB06F7106AC319D06941
:201C6000984202DAD069106206E09069984202DD9069106200E0136250889CFBF0F0B2F8B2
:201C80000690D2F8208098FBF9F800EB0801002906DA1069884203DD108A00B2BDE8F0833C
:201CA000002905DD5069884202DC908A00B2F5E708B2F3E72DE9F34F83B00C46204603F046
:201CC00069F800901D4800990160BDF90C001B49B1F9001000FB01F7FF13BDF90E001749AB
:201CE000B1F9021000FB01F84FEAE8380FFA87FB0FFA88F001900198ABEB000000B2ADF8B8
:201D00000800BDF90C000D49B1F9021000FB01F5ED13BDF90E000949B1F9001000FB01F634
:201D2000F6130FFA85F90FFA86FA09EB0A0000B2ADF80A00029805B0BDE8F08F4C0000204C
:201D40007047000030B50246B2F900303F4CB4F90040A34202DD13883C4C2380B2F90230E5
:201D60003B4CB4F90040A34202DD5388384C2380B2F90430374CB4F90040A34202DD9388FB
:201D8000344C2380344B1B885B1C1BB2324C23802346B3F90030B3F5FA7F56DB2B4BB3F9E0
:201DA00000000023294C2380031E01DB1C4600E05C42B5256C43294D2D68C5EB8404274DCB
:201DC0002D6805EB6414254D2C602B461B689B121BB20B801E4BB3F9000000231C4C2380CC
:201DE000031E01DB1C4600E05C42B5256C431C4D2D68C5EB84041A4D2D6805EB6414184D7E
:201E00002C602B461B689B121BB24B80114BB3F9000000230F4C2380031E01DB1C4600E095
:201E20005C42B5256C430F4D2D68C5EB84040D4D2D6805EB64140B4D2C602B461B689B1276
:201E40001BB28B800023044C238030BD6C0500206E050020700500207205002074050020BE
:201E6000780500207C05002000B585B000BF1148806940F004000F4988610846806900F09D
:201E80000400009000BF00BF002289140A48F8F7B5FC4FF480500190012002900220049072
:201EA00001A90548F8F710FB00200449087005B000BD0000001002400008014072040020A9
:201EC00010B50446012C0BD10C480078A8B9012211030B48F8F792FC0120084908700CE0E0
:201EE0005CB906480078012807D1002201030448F8F784FC00200149087010BD72040020E0
:201F00000008014010B5044619480078012816D1B4F5D16F0FDB17480088401C80B21549DA
:201F2000088047F23051884220DD0020114908800F4908701AE000200E49088016E0B4F52E
:201F4000BC6F10DA0C480088401C80B20A4908803C280BDDF4F792FF012005490870002058
:201F60000649087002E000200349088010BD000084050020800500208205002003020020DD
:201F800038B50446002034490870F020487008460078C043314908702F484078C043487088
:201FA0002D4840782E4B0090DA79997958792D4B1B78FAF7B5FD2C48007810BB2B48006875
:201FC0002B4908602948406848602848806888602648C068C8602748406808612548406ACF
:201FE00048612448C06A88612822234801F002FE042222A12048083801F0FCFD01201A4914
:20200000087020A341F205320C214FF4E26001F0F3FE04B938BDF8F7F7FB1C490860002007
:202020001B49087012E0F8F7EFFB18490968401A64280BD9F8F7E8FB1449086014480078F2
:20204000401C134908701348F8F70CFC104800780A28E8DB00BFDDE7DA000020DC000020C0
:20206000D00A00203C040020B6000020200C0020900B0020000B002008E80108464C4147EB
:20208000000000005245414459000000B8000020BC000020F007002010B50248F9F7F7FB0F
:2020A00010BD0000901C002010B500210B48F9F785FE04210948F9F781FE08210748F9F78E
:2020C0007DFE00210548F9F719FB04210348F9F715FB08210148F9F711FB10BD901C00209C
:2020E00008B508490968C9084FF47A72B1FBF2F14143009100BF00BF00994A1E0092002983
:20210000F9D108BD000000202DE9F04705460E4617469846F8F778FB84490968401A0528C2
:2021200001D2BDE8F087F8F76FFB804908600FFA88F07F4948807F480088281AC8810846ED
:20214000007801287ED1F8F75FFB7949C969401AB0F5FA6F06D9F8F757FB7549C8610120C2
:20216000887601E0744886607148407E01281BD100206F494876002405E000206F4921F8C2
:202180001400601CC4B2192CF7DB00206C4908806C4908606C4908706548408A20B1644887
:2021A000408A0002694908606148C0890A2849DB604805605E48807E00286FD15E4886604C
:2021C0000774C068002869D05B4880895A490989401A00B25E4908800846B0F900000028C0
:2021E00003DD0846B0F9000000E00020584908800846B0F900001E2803DA0846B0F90000CE
:2022000000E01E20524908800846008818B94A48007C642842D049484949098830F811003D
:2022200048490968081A47490860084600684849B1F900100844434908604548008881B2F9
:202240003F4800E06FE002880088401C3C4B18803A4820F8121018460088192807DB002056
:2022600019460880012038490870314908763548006840B334480078012810D131480068AE
:202280004FF47A7148436421484329498989FA225143B0FBF1F02649088217E03FE0284836
:2022A000008800EB80004100214880894143254800684FF47A72504364225043B0FBF1F0B8
:2022C0001B49088202E00020194908821C480088A0B91748B0F810901C480068C0EB092096
:2022E0001E2190FBF1F01949096808441749086008460068C0F30F200D4948820C48408A76
:20230000002808DD0C4880680949898AB0FBF1F00749C88203E04FF6FF700549C88206486C
:2023200080680549C86000BFFBE6000078030020140300207C03002034030020540700205C
:20234000680300206C0300207003002074030020720300202DE9F04104460D461746984685
:20236000069E00201349086088601348008848600020C8600DB90846866000200F49087030
:2023800048800520888000208860084684810020C881088248824FF6FF70C8820020087694
:2023A000487601208876F8F72FFA0449C861BDE8F081000034030020B40900201403002031
:2023C0002DE9F04106460F4606F00F0000287DD0052FFCD001206F4908700846007E012855
:2023E00064D1002008760846408A6B49098888425CD06848408A002854D06648408A6749C9
:202400000988401A642100FB01F56448008895FBF0F004B214F11E0F44DBB4F5E47F41DA89
:2024200004F164005D4909884843642190FBF1F0584988825A48058804F16400684364212D
:2024400090FBF1F0574908805548458804F164006843642190FBF1F0524948805048858881
:2024600004F164006843642190FBF1F04D4988804B48C58804F164006843642190FBF1F0F4
:202480004849C8804648058904F164006843642190FBF1F0434908810B461022A22142486D
:2024A00001F00BFC3B48408A3B4908803F480078864203D13E480078874265D0032E1DD016
:2024C00005DC012E08D0022E33D10EE054E0042E1DD0332E2DD123E0324800882D494882FB
:2024E0002F4800882D49088029E02E484088294948822B4840882949088020E029488088AE
:2025000024494882264880882449088017E02548C088204948822248C088204908800EE0A9
:20252000204800891B4948821D4800891B49088005E00020174948821849088000BF00BF0C
:202540001448408A144908801248408A114988820846408A002807DD16488068898AB0FBC0
:20256000F1F00C49C88203E04FF6FF700949C88201200849487607E00020064908704882E0
:2025800088824FF6FF70C8820848067008480770BDE8F0811403002082030020840300200D
:2025A000DC720108300C00202C0400208003002081030020340300202DE9F0470746894611
:2025C0001546AD10002414E057F82460300E144A02F82400C6F30741A000401C1154C6F323
:2025E0000721A000801C1154A000C01C1654601CC4B2AC42E8DB57F825A0A1000848F2F79B
:20260000D9FD8046BAEB080007D1AA0004494846F1F745FA0020BDE8F0874FF0FF30FAE762
:20262000F015002010B5B0F900205243B0F9023003FB03210C4A914214D909163939CBB231
:202640000A4C34F81320B0F9003003FB02F1CB131BB20380B0F9023003FB02F1CB131BB256
:20266000438000BF10BD0000400AC139AC6E01082DE9F14181B0BDF90400DFF86880B8F901
:20268000008000FB08F1C913BDF90600DFF85480B8F9028000FB08F2D2130EB217B2F019E4
:2026A00000B2ADF80000BDF90400DFF83880B8F9028000FB08F3DB13BDF90600DFF824802C
:2026C000B8F9008000FB08F4E4130FFA83FC25B2CCF10000284400B2ADF802000098BDE8BD
:2026E000FC8100004C00002010B504462078012808D10B4B30224C210A4801F0DEFA0020F8
:2027000020700AE02078022807D1074B1022EC21044801F0D2FA00202070002010BD00006E
:20272000000B00202C040020300B00204FF055301F4A106040001F4A10601D480168B1F19D
:20274000553F01D0002070471A480168B1F1AA3F01D00020F7E74FF0AA30154A10604008E8
:20276000144A106012480168B1F1AA3F01D00020E9E710480168B1F1553F01D00020E2E7CB
:202780004FF055300A4A106040000A4A106008480168B1F1553F01D00020D4E7054801685C
:2027A000B1F1AA3F01D00020CDE70120CBE70000000800201008002001200C490968B1F12D
:2027C000EE3F00D0002009494968B1F1CC3F00D0002006498968B1F1BB3F00D00020034924
:2027E000C968B1F1DD3F00D0002070477829002010B5214800780D282FD2DFE800F0070ADE
:202800000D101316191C1F2225282B00F0F7D6FC24E0F0F707FD21E0F0F743FD1EE0F0F7CF
:2028200085FD1BE0F0F7C8FD18E0F0F70CFE15E0F0F750FE12E0F0F794FE0FE0F0F7D9FE44
:202840000CE0F0F71FFF09E0F0F760FF06E0F0F7A1FF03E0F0F7E2FF00E000BF00BF064894
:202860000078401C04490870084600780C2801DD0020087010BD00000006002010B5F0F7B0
:202880009DFCF0F7CFFCF0F70CFDF0F74FFDF0F793FDF0F7D8FDF0F71DFEF0F762FEF0F767
:2028A000A8FEF0F7EFFEF0F731FFF0F773FFF0F7B5FF10BD10B53B480068B0F1AA3F70D14B
:2028C00038480068384909684840401C002866D136490860C0433649086034480068801C8A
:2028E00032490860FFF784FF31480068801E304908602E4800680D302C490860FFF75CFFD3
:2029000008B9F5F73BF82A4800680D3828490860264800680B302549086000F0C5FC0446FD
:2029200034B1012C0AD0032C04D0042C05D100E007E006E0F5F722F803E000BFF5F71EF84B
:2029400000BF00BF1A4800680B381949086017480068C01C1549086000F044F808B9F5F7E0
:202960000DF813480068C01E114908600F480068401D0E490860FFF7D9FE08B9F4F7FEFF9E
:202980000B480068401F0A490860222003F042FD08B9F4F7F3FF00200249086001E0F4F7B1
:2029A000EDFF10BD3C250020602500202C2500205025002010B500F047FC00F055FC00F009
:2029C00001F810BD4FF0EE30054908604FF0CC3048604FF0BB3088604010C86070470000FA
:2029E00078290020F0B55527552F01D00020F0BDAA27AA2F01D00020F9E74FF05531B1F1F1
:202A0000553F01D00020F2E74FF0AA31B1F1AA3F01D00020EBE74FF47A714A008C1840F69E
:202A2000B830844201D00020E1E74FF0FF3102228C18012C01D00020D9E74FF47A73F94DA4
:202A40005E1916F57A7F01D00020D0E76FF0004301255E19B6F1004F01D00020C7E76FF020
:202A6000004302255E19981C864201D00020BEE76FF0004303255E19D81C864201D0002075
:202A8000B5E74FF4FA614A108C1AB4F57A7F01D00020ACE74FF4FA614A1C8C1A601C08B1F7
:202AA0000020A4E7002101228C1A601C08B100209DE74FF47A735D005E1B16F57A7F01D0CD
:202AC000002094E7002301255E1B701C08B100208DE74FF0004301255E1B581E864201D090
:202AE000002084E74FF47A71491C0846814201D000207CE74FF0FF31491C09B1002076E748
:202B00000021491C012901D0002070E74FF47A735B1C1846834201D0002068E700235B1C19
:202B2000012B01D0002062E76FF000435B1CB3F1004F01D000205AE74FF000435B1C18469A
:202B4000834201D0002052E74FF47A71491E0846814201D000204AE70021491E481C00B121
:202B600045E74FF0FF31491E881C00B13FE74FF47A735B1E1846834201D0002037E74FF0BE
:202B800000435B1E1846834201D000202FE76FF000435B1E1846834201D0002027E70023EF
:202BA0005B1E581C00B122E764210A2201FB02F4B4F57A7F01D0002019E76FF070411122F5
:202BC00001FB02F49848844201D000200FE74FF0FF31012201FB02F4601C08B1002006E7B0
:202BE0006421002201FB02F40CB10020FFE64FF47A710A22B1FBF2F4642C01D00020F6E631
:202C000001210A22B1FBF2F40CB10020EFE600210A22B1FBF2F40CB10020E8E64FF47A716A
:202C20000022B1FBF2F40CB10020E0E64FF0FF310122B1FBF2F4601C08B10020D7E60221E4
:202C40004C00042C01D00020D1E602210C02B4F5007F01D00020CAE60221CC070CB1002083
:202C6000C5E64FF6FF714C084810844201D00020BDE64FF6FF710C0AFF2C01D00020B6E66B
:202C80004FF6FF71CC0F0CB10020B0E6012109B90020ACE6002109B10020A8E6FF2109B930
:202CA0000020A4E664210A22914201D800209EE664216422914201D9002098E60A21642262
:202CC000914201D9002092E64FF0FF310022914201D800208BE66FF00043DD07AB4201DC91
:202CE000002084E60A216422914201D300207EE664216422914201D2002078E664210A228E
:202D0000914201D2002072E600214A1E914201D300206CE64FF000435D1EAB4201DB00200D
:202D200065E664210A22914201D200205FE664216422914201D2002059E60A2164229142F8
:202D400001D3002053E64FF0FF310022914201D200204CE66FF00043DD07AB4201DA00204F
:202D600045E60A216422914201D900203FE664216422914201D9002039E664210A2291420A
:202D800001D8002033E600214A1E914201D900202DE64FF000435D1EAB4201DD002026E6C4
:202DA00064216422914201D0002020E64FF0FF310A46914201D0002019E6002100229142A6
:202DC00001D0002013E64FF000431D46AB4201D000200CE600230025AB4201D0002006E642
:202DE0006FF000431D46AB4201D00020FFE564216422914201D00020F9E54FF0FF310A46A0
:202E0000914201D00020F2E500210022914201D00020ECE54FF000431D46AB4206D0002077
:202E2000E5E5000030F8FFFFEFFFFF0F00230025AB4201D00020DAE56FF000431D46AB42CF
:202E400001D00020D3E50121002221B9022904D0032906D103E0921C04E0121D02E00832E9
:202E600000E000BF00BF022A01D00020BFE502210022012904D0022904D0032906D103E00B
:202E8000921C04E0121D02E0083200E000BF00BF042A01D00020AAE503210022012904D005
:202EA000022904D0032906D103E0921C04E0121D02E0083200E000BF00BF082A01D00020CF
:202EC00095E504210022012904D0022904D0032906D103E0921C04E0121D02E0083200E091
:202EE00000BF00BF0AB1002081E50021002211B10AB100207BE501B90AB1002077E50021C1
:202F0000012211B10AB1002071E511B90AB900206DE50121012201B10AB9002067E511B9AC
:202F20000AB9002063E50121FF2201B10AB900205DE511B90AB9002059E50021FF2211B15D
:202F40000AB1002053E511B90AB900204FE54FF055310A4681EA02040CB1002047E54FF0AF
:202F600055314A0081EA0204601C08B100203EE50021002281EA02040CB1002037E54FF0AC
:202F8000FF310A4681EA02040CB100202FE500214A1E81EA0204601C08B1002027E54FF0B5
:202FA0005531CC43B4F1AA3F01D000201FE5E443B4F1553F01D0002019E50021CC43601CFE
:202FC00008B1002013E5E4430CB100200FE501200DE5000008B500BF7148806940F00400C3
:202FE0006F4988610846806900F00400009000BF00BF00BF0846806940F008008861084692
:20300000806900F00800009000BF00BF00BF0846806940F0100088610846806900F010006B
:20302000009000BF00BF00BF0846806940F0200088610846806900F02000009000BF00BFFE
:203040005848F4F7EFFC08B9002008BD5648F4F7E9FC08B90020F8E75448F4F7E3FC08B9FF
:203060000020F2E75248F4F7DDFC08B90020ECE74B48806920F00400494988610846806903
:2030800020F0080088610846806920F0100088610846806920F0200088614648F1F734FBFA
:2030A00000BF3F48C06940F000703D49C8610846C06900F00070009000BF00BF3E48F2F7FE
:2030C00033F808B90020C0E73548C06920F000703349C86100BF0846406940F001004861E2
:2030E0000846406900F00100009000BF00BF3348F2F750FD08B90020A7E72948406920F090
:2031000001002749486100BF0846806940F4007088610846806900F40070009000BF00BF69
:2031200000BF0846806940F4806088610846806900F48060009000BF00BF2148F1F7FCF93D
:2031400008B9002081E71F48F1F7F6F908B900207BE71348806920F400701149886108464C
:20316000806920F48060886100BF0846806940F4006088610846806900F40060009000BF3C
:2031800000BF114801F089FB08B900205DE70448806920F4006002498861012055E7000043
:2031A0000010024000080140000C0140001001400014014000000140006400400800024052
:2031C0000024014000280140002C014010B5002419480068194909684840401C48BB1648EA
:2031E00000681749884210D316490846F0F74EFB012801D1042400E0032411484B380E4920
:203200000860C0430D49086014E00E490A480068F0F73CFB01280AD1074800681030064918
:20322000086008460068C0430449086002E0032400E00124204610BD3406002038060020BF
:203240007B0000201406002004480549086008460068C04303490860704700003000002023
:20326000340600203806002010B50A480A490860C0430A4908600A480A4908600846F6F7BE
:2032800008FE08480068806840F0010005490968886010BD00300008482500206C2500206D
:2032A000003002400806002010B502241F4800681F4909684840401C002834D11B480068FF
:2032C0001C49884223D2002006E01849096851F82010194A1160401C18498908174A92095B
:2032E000B1FBF2F18142F0D814498908134A9209B1FBF2F10D4A126802EB81010B4A116039
:2033000011460968C9430A4A116000240CE00A48006808490968884201D1042400E00324BD
:20332000FFF7A2FF00E00124204610BD482500206C25002080890108003002408059010022
:2033400070B50A2050490870F7F7A0FA00F0E2FF00204E490860C0434D4908604B48006899
:20336000801C4A490860FFF789FA49480068801E47490860EFF7D6FE0C2043490870434839
:2033800000680B304149086042484349086008460068806840F00100096888603E48F6F77F
:2033A00078FD002405E03D4951F8240039490860641C3B48B4EB900FF5D33648056839483D
:2033C0000068854201D0F4F7D9FA314800680B382F4908600E202C4908702C480068C01C58
:2033E0002A490860FFF7FEFA08B9F4F7C7FA28480068C01E2649086010202349087023488B
:203400000068401D21490860FFF790F908B9F4F7B5FA1F480068401F1D49086012201A49AA
:2034200008701A480068C01D18490860FFF7D2FD08B9F4F7A3FA142013490870FFF7CAFDD1
:2034400008B9F4F79BFA12480068C01F1049086016200D4908701C2002F0DCFF08B9F4F710
:203460008DFA1820084908704FF400510804F0F786FA08B9F4F782FA00F0B6FFAA200549D8
:203480000871EFF733FE70BD040600202C2500205025002000300240080600200030000867
:2034A000805901008089010810B5124800780A281EDB00200F4908704FF0AA300E49086096
:2034C00040080E49086072B6FFF780FE044662B634B1012C08D0032C05D0042C02D100E016
:2034E00005E004E000BF00BFF4F748FA00BF00BF10BD0000590000203C250020602500206E
:20350000002107E041F64C5100BF0A00A1F1010399B2FAD10200A0F1010398B2F2D17047FF
:20352000002106E0072100BF0A00A1F1010399B2FAD10200A0F1010398B2F3D170477047D4
:203540002DE9F143BDF9000044F2F30100FB01F9BDF902004FF416514843C0F1000844461C
:2035600008EB09004710A8EB09004610002F0FDA002E03DA0520F749088018E0002C03DCF3
:203580000420F449088012E00320F24908800EE0002E03DB0220EF49088008E0002C03DC9B
:2035A0000620EC49088002E00120EA4908800020E9490870E748008807287BD2DFE800F0B6
:2035C0007A044D97E0FCFB0004F51650801B4FF4966101EBA040E14908800846008800EB3F
:2035E0006640488008464088A0EB6440888008460088C0F5166080B2E22803DD40F65F104E
:20360000C88029E0D5480088D4494988401A85B2B5F58B7F05DBD14800883338CF49C88035
:203620001AE0CE480088C0F5166080B28A2813DDCA480088E230C949C8800846C088B0F5B2
:20364000166F09DB0120C4490870C448C088C0F59650401EC149C88074E107F51650801B6A
:203660004FF4966101EBA040BC4908800846008800EB6640488008460088A0EB6740888078
:2036800008464088C0F5166080B2E22803DD40F65F10C8802AE0B1484088B0490988401A31
:2036A00085B2B5F58B7F06DBAC4840883338AB49C8801BE045E1A9484088C0F5166080B2A4
:2036C0008A2813DDA5484088E230A449C8800846C088B0F5166F09DB01209F4908709F4840
:2036E000C088C0F59650401E9C49C8802AE1C4F5165038444FF4966101EBA0409749088048
:2037000008460088A0EB674088800846808800EB6440488008464088C0F5166080B2E2286F
:2037200003DD40F65F10C88029E08C4840888B498988401A85B2B5F58B7F05DB8748408876
:2037400033388649C8801AE084484088C0F5166080B28A2813DD81484088E2307F49C880A7
:203760000846C088B0F5166F09DB01207A4908707A48C088C0F59650401E7849C880E1E07C
:2037800004F51650801B4FF4966101EBA040734908800846008800EB6640488008464088A0
:2037A000A0EB6440888008468088C0F5166080B2E22806DD01E078E02EE040F65F10C880FE
:2037C00029E06648808865494988401A85B2B5F58B7F05DB6148808833386049C8801AE07F
:2037E0005E488088C0F5166080B28A2813DD5B488088E2305949C8800846C088B0F5166FB5
:2038000009DB0120544908705448C088C0F59650401E5249C88095E007F51650801B4FF419
:20382000966101EBA0404D4908800846008800EB6640488008460088A0EB6740888008461A
:203840008088C0F5166080B2E22803DD40F65F10C88029E04148808840490988401A85B2E7
:20386000B5F58B7F05DB3D48808833383B49C8801AE03A488088C0F5166080B28A2813DD6D
:2038800036488088E2303549C8800846C088B0F5166F09DB0120304908703048C088C0F59F
:2038A0009650401E2D49C8804CE0C4F5165038444FF4966101EBA04028490880084600886A
:2038C000A0EB674088800846808800EB6440488040F65F10C88008460088C0F5166080B2E1
:2038E000E22803DD40F65F10C88029E01B4800881A498988401A85B2B5F58B7F05DB174805
:20390000008833381549C8801AE014480088C0F5166080B28A2813DD10480088E2300F49E7
:20392000C8800846C088B0F5166F09DB01200A4908700A48C088C0F59650401E0749C88084
:2039400000E000BF00BF0448007848B9002000F003FB08E03400002036000020380000204C
:20396000022000F0F9FA40F64C100949C880088800F0DAFA0649488800F0DCFA0449888880
:2039800000F0DEFA0249C88800F0E0FABDE8F883380000202DE9F04104460025002600277F
:2039A000F3F7ACFAA84618E000BF334800780128FBD10020304908703048008805442F4819
:2039C000408806442D48808807440C212C48F8F7D5F908F101001FFA80F8B8F10A0FE3DBA4
:2039E0000A20B5FBF0F0274908800A20B6FBF0F048800A20B7FBF0F088800846008846F2C0
:203A0000A81188421DDB1F48008849F64041884217DC1C48408846F2A811884211DB19488B
:203A2000408849F6404188420BDC1648808846F2A811884205DB1348808849F6404188425F
:203A400016DD206820F4802000F58020206006200D4948800846F3F73BFD00200B49087082
:203A60000B484089401C0A494881022009490870F3F744FABDE8F08120050020140500200A
:203A8000901C002026050020880700209D030020300B0020BE01002008B50020009053485E
:203AA0000088072870D2DFE800F0933362630405320000BF4E480088404201B211F5004F29
:203AC00004DA4FF40040ADF8000009E0B1F5004F04DB47F6FF70ADF8000001E0ADF800103C
:203AE00043484088404201B211F5004F04DA4FF40040ADF8020009E0B1F5004F04DB47F6E7
:203B0000FF70ADF8020001E0ADF8021061E000BF37484088404201B211F5004F04DA4FF405
:203B20000040ADF8020009E0B1F5004F04DB47F6FF70ADF8020001E0ADF802102C4880887A
:203B4000BDF80220801A01B2B1F5004F04DB47F6FF70ADF8000009E011F5004F04DA4FF4BD
:203B60000040ADF8000001E0ADF8001031E000BF1F480088404201B2B1F5004F05DB47F6C4
:203B8000FF70ADF800000AE022E011F5004F04DA4FF40040ADF8000001E0ADF800101448D8
:203BA0008088BDF80020801A01B211F5004F04DA4FF40040ADF8020009E0B1F5004F04DBC1
:203BC00047F6FF70ADF8020001E0ADF8021000E000BF00BFBDF900000011ADF80000BDF97A
:203BE00002000011ADF80200009808BD340000202C0500202DE9F04781460D4616463046D0
:203C0000F11706EB9171C1F38707002415E015F824000106A000401C285C01EB0041A000C9
:203C2000801C285C01EB0021A000C01C285C08440A4941F82400601CC4B2BC42E7DB314632
:203C40002846F1F7B7FA8046044840F827807A1C01464846F3F73AFDBDE8F087F01600209E
:203C60002DE9F04190B080460D4616463046F11706EB9171C1F38707002414E0A000C01C01
:203C8000285C0106A000801C285C01EB0041A000401C285C01EB002015F8241008444DF84E
:203CA0002400601CC4B2BC42E8DB3A4669464046F3F70CFD10B0BDE8F0812DE9F843814697
:203CC0000D4616461F46002000908046002420E02819C1B26A464846F3F746FA401C18B9ED
:203CE0004FF0FF30BDE8F883385D9DF8001088420DD0385D00902819C1B29DF80020484639
:203D0000F3F788FA401C10B94FF0FF30EAE7601CC4B2B442DCDB31463846F1F733FA804664
:203D20004FEA28200090A819C1B29DF800204846F3F770FA401C10B94FF0FF30D2E708F063
:203D4000FF000090A819401CC1B29DF800204846F3F760FA401C10B94FF0FF30C2E7002061
:203D6000C0E7000070B505460C46002C33D11E4800691E4948600B4630224C212846FFF758
:203D80009CFF401C28B9194B30224C212846FFF794FF1548006816490860134840684860FA
:203DA0001148806888601048C068C8600E4840690E4948620C488069C8620D4B1022D6214A
:203DC0002846FFF77AFF401C28B9094B1022D6212846FFF772FF064800680A21B0FBF1F00A
:203DE00004494882002070BD900B0020000B0020200C0020DC0800202DE9F04706468846C2
:203E0000174699460025FCB255201F490870AA204870084680F80280A01CC870380A0871C5
:203E20000846447122464946801DEFF738FE552016490870AA20487030128870CE70221D4A
:203E40001149891C1148001DEFF729FE04F108010E48F1F7AFF90546280EA11D0A4A5054C5
:203E6000C5F30741E01D1154C5F30721401C1154401C1554F021401C1154421C0249304689
:203E8000F1F7B4F8BDE8F0873E0E00203D0F00202DE9F04781460E4690461F46DDF820A062
:203EA0000025FCB255201E490870AA204870300A8870CE70084680F80480A01C4871380AE8
:203EC00088710846C471224651460830EFF7E7FD04F1080212491348EFF7E1FD04F10801EE
:203EE0001048F1F767F90546280E04F108010C4A5054C5F3074104F109001154C5F3072166
:203F0000401C1154401C1554F021401C1154401CC2B20349484601F008F9BDE8F087000091
:203F20003C100020D21000200149096848637047901C00200149096888637047901C002001
:203F400001490968C8637047901C00200149096808647047901C002008490968096A21F404
:203F60000051064A1268116204490968096A41EA0031024A1268116270470000901C00206A
:203F800010B51048007801281BD10F4A32210F4800F048F90446EFF781FF0D490860084687
:203FA0000068EFF79EFF0B490860002005490870084800681E2804DA0348008800B20649C4
:203FC000088010BD100100201C0100201408002014010020180100200C0100202DE9F047FA
:203FE00005460C4616461F46DDE90889F6F70CFC19490968401A32282BD3F6F705FC164945
:20400000086005FB06F090FBF7F000FB08F000EBC000000142F2107190FBF1F020802088C8
:204020000E49096808440D4908600D480078401C0B4908700846007808280ADB0020087046
:2040400006480068C0F3CF00A9F80000002003490860BDE8F0870000040400200C0400203F
:204060000804002070B504460D461646F6F7CCFB24490968401A322841D3E07828B9F6F776
:20408000C3FB214908600120E070F6F7BDFB1E490968401AB0F57A6F04D90020A0704FF668
:2040A000FF70A060208980B24FF6FF71884202D10020A07001E00120A070A078012812D1FE
:2040C000A06810B94FF0FF30A0604FF4B4707043A168B0FBF1F0208020880A220B49FDF736
:2040E00063FC288007E00020208028800A210748F0F791FB70BDF6F787FB0249086000BF6F
:20410000F8E7000010040020140400204E15002000B585B000BF1048806940F020000E4940
:2041200088610846806900F02000009000BF00BF04200190094802900120039001A90848FB
:20414000F6F7C2F9002202210820F6F72CFC0820F6F71CFC05B000BD001002400000111023
:20416000001401402DE9F04104460D4617461E46F6F74AFB28490968401A32284AD3E07808
:2041800028B9F6F741FB254908600120E070F6F73BFB22490968401A4FF47A6191FBF6F1E4
:2041A000884201D90020A070A078012822D1A06810B94FF0FF30A0604FF4B4707843B0FBEB
:2041C000F6F0A168B0FBF1F0208020880A221449FDF7EAFB2880F6F717FB6168411AA068E7
:2041E000B1EB400F12D940F20E41A0684843800AA0600BE00020208028800A210848F0F796
:204200000AFB4FF0FF30A060BDE8F081F6F7FCFA0149086000BFF7E7FC03002000040020A0
:204220003A1500202DE9F74F88B0044689464FF0000BDA460020069000210F4688460D46AB
:204240000E4600BF0FE034F81B00EFF73DFE3A464346CDE90401EFF70BFD074688460BF12B
:20426000010000F0FF0BCB45EDDB4846EFF72CFE02460B46CDE9020138464146EFF79FFDF4
:20428000CDE90401EFF7A5FE06900698EFF742FE81B20A9801804FF0000A23E034F81A0098
:2042A000EFF7FCFD00900699EFF7AAFC029034F81A00EFF7F3FD00900699EFF7A1FC019073
:2042C0000299EFF7A3FC0390EFF770FE2A463346CDE90401EFF7CCFC05460E460AF10100EA
:2042E00000F0FF0ACA45D9DB2846314602F056FBCDE90201EFF741FE80B20590EFF7E4FD6E
:2043000005460E4628463146EFF737FE80B20BB0BDE8F08F10B594B009200A904FF480302E
:204320000B9000200C9001200E90109002201190C10312914FF4E01113910AA8F6F712FE16
:2043400018B1CD211AA001F0C5FE0F20059002200690002007904FF4806008900020099091
:20436000022105A8F6F7BCFC18B1DB2110A001F0B1FE022001908003039001A8F6F718FC40
:2043800018B1E2210AA001F0A5FEF6F77BFD4FF47A71B0FBF1F42046F7F70AF90420F7F787
:2043A00001F800221146501EF6F7FDFA14B010BD2E2E5C53656C6654657374557365725CCB
:2043C0007372635F6D6964646C6577617265735C73746D33326678785F5354557374617225
:2043E0007475702E6300000010B590B00220069001200A9010200B9000200D9006A8F6F738
:20440000B1FD20B140F2031114A001F063FE0F2001900020029003904FF4806004900020F5
:204420000590002101A8F6F75BFC20B140F211110AA001F04FFEF6F725FD4FF47A71B0FBE4
:20444000F1F42046F7F7B4F80420F6F7ABFF00221146501EF6F7A7FA10B010BD2E2E5C53AF
:20446000656C6654657374557365725C7372635F6D6964646C6577617265735C73746D334F
:20448000326678785F535455737461727475702E63000000034618044843B0FBF2F0704761
:2044A00010B5F6F7E7F9F7F79DF803480078401C0149087010BD00005900002010B594B0B7
:2044C00009200A904FF480300B9000200C9001200E90109002201190C10312914FF4E01112
:2044E00013910AA8F6F73EFD20B140F295111CA001F0F0FD0F2005900220069000200790C8
:204500004FF48060089000200990022105A8F6F7E7FB20B140F2A31111A001F0DBFD022035
:2045200001908003039001A8F6F742FB20B14FF4D5710BA001F0CEFDF6F7A4FC4FF47A7185
:20454000B0FBF1F42046F7F733F80420F6F72AFF00221146501EF6F726FA14B010BD00008D
:204560002E2E2F436F72652F5372632F6D61696E2E6300001148006840F001000F490860B9
:20458000084640680E4908400C494860084600680C490840094908600846006820F4802012
:2045A00008600846406820F4FE0048604FF41F008860C80304490860704700000010024010
:2045C0000000FFF8FFFFF6FE08ED00E010B50248F7F706FA10BD0000901C002000220268FB
:2045E000184B984208D0B0F1804F05D0164B984202D0164B984203D122F070024B681A43B1
:20460000104B984208D0B0F1804F05D00E4B984202D00E4B984203D122F44072CB681A43E4
:2046200022F080024B691A4302608B68C3620B688362044B984201D10B6903630123436166
:2046400070470000002C0140000400400008004030B50023012404FA01F3046A9C430462D8
:20466000046A02FA01F52C43046230BD30B50023042404FA01F3046A9C430462046A02FAD9
:2046800001F52C43046230BD30B50C460021816821F47F4142EA032525432943816030BD56
:2046A0000A460021816821F0700142F0070319438160704730B5002400220023056A25F01C
:2046C00001050562026A4368846924F0700424F003040D682C4322F002028D682A430D4D10
:2046E000A84206D100BF22F00802CD682A4322F00402084DA84207D123F4807323F40073B9
:204700004D692B438D692B43436084614D684563026230BD002C014030B500240022002320
:20472000056A25F010050562026A4368846924F4E04424F440740D6844EA052422F020026D
:204740008D6842EA05120F4DA84207D100BF22F08002CD6842EA051222F04002094DA842A4
:2047600009D123F4806323F400634D6943EA85038D6943EA8503436084614D68856302624C
:2047800030BD0000002C014030B5002400220023056A25F480750562026A4368C46924F035
:2047A000700424F003040D682C4322F400728D6842EA05220E4DA84207D100BF22F4006262
:2047C000CD6842EA052222F48062094DA84209D123F4805323F400534D6943EA05138D69FA
:2047E00043EA05134360C4614D68C563026230BD002C014030B5002200230024056A25F43B
:2048000080550562036A4468C26922F4E04222F440720D6842EA052223F400538D6843EAC4
:204820000533074DA84204D124F480444D6944EA85144460C2614D680564036230BD00009D
:20484000002C014030B50B46144600210022026A056A25F001050562816921F0F00141EAA4
:20486000041122F00A021A438161026230BD30B50B46144600210022056A25F010050562A2
:204880008169026A21F4704141EA043122F0A00242EA03128161026230BD0146002240F2D9
:2048A00005100860086882B240F20510824201D00020704740F28A200860086882B240F20A
:2048C0008A20824201D00020F3E70020086045F255504860486882B245F25550824201D03E
:2048E0000020E6E742F6A8204860486882B242F6A820824201D00020DBE70020486045F2C9
:2049000055508860886882B245F25550824201D00020CEE74AF6A2208860886882B24AF652
:20492000A220824201D00020C3E70020886045F25550C860C86882B245F25550824201D075
:204940000020B6E742F6AA20C860C86882B242F6AA20824201D00020ABE70020C86045F244
:2049600055508861886982B245F25550824201D000209EE74AF6AA208861886982B24AF616
:20498000AA20824201D0002093E70020886145F25550C861C86982B245F25550824201D03A
:2049A000002086E74AF6AA20C861C86982B24AF6AA20824201D000207BE70020C86141F235
:2049C00055500862086A82B241F25550824201D000206EE742F6AA200862086A82B242F6F6
:2049E000AA20824201D0002063E70020086245F255504862486A82B245F25550824201D087
:204A0000002056E74AF6AA204862486A82B24AF6AA20824201D000204BE70020486245F2AD
:204A200055508862886A82B245F25550824201D000203EE74AF6AA208862886A82B24AF6B1
:204A4000AA20824201D0002033E70020886245F25550C862C86A82B245F25550824201D0D6
:204A6000002026E74AF6AA20C862C86A82B24AF6AA20824201D000201BE70020C8625520EF
:204A80000863086B82B2552A01D0002011E7AA200863086B82B2AA2A01D0002009E70020EB
:204AA000086345F255504863486B82B245F25550824201D00020FCE64AF6AA204863486B42
:204AC00082B24AF6AA20824201D00020F1E60020486345F255508863886B82B245F2555077
:204AE000824201D00020E4E64AF6AA208863886B82B24AF6AA20824201D00020D9E600207D
:204B0000886345F25550C863C86B82B245F25550824201D00020CCE64AF6AA20C863C86B91
:204B200082B24AF6AA20824201D00020C1E60020C86345F255500864086C82B245F25550C4
:204B4000824201D00020B4E64AF6AA200864086C82B24AF6AA20824201D00020A9E600207A
:204B6000086441F215508864886C82B241F21550824201D000209CE640F60A208864886C0E
:204B800082B240F60A20824201D0002091E600208864086101208CE62DE9F04104460E4668
:204BA00090461F4630480078012812D12F4801780078401C2D4A10702D4820F811601046AF
:204BC000007832281CDB0020274908701146087016E0322226493046FCF7E6FE054620883C
:204BE000A84209DDF5F710FE22490968401AB0F57A7F05D9258003E0F5F706FE1D490860F3
:204C000040F6340008FB00F0642190FBF1F0C0F580502188884203DBF5F7F6FD16490860CA
:204C2000F5F7F2FD14490968401A42F21071884217D9386820F040004030386003200F498F
:204C40004880208888800846F2F742FC00200C4908700C48808A401C0A49888201200A49EF
:204C60000870BDE8F0810000190400201A0400207A150020200400201C0400208807002049
:204C80009D030020000B0020BE0100202DE9F04704460F46E7824FF0090841462046F3F7CE
:204CA000A9FAC01B0FFA80F919F1780F2ADDB9F1780F27DA002606E0701C34F8100024F83A
:204CC0001600701CC6B2A8F10100B042F4DC24F8107041462046F3F717FB05B2608AA8424E
:204CE00000DA658241462046F3F71FFB05B2A08AA84200DDA582064B18227E210548FEF7C7
:204D0000DCFF02E0002004490870BDE8F0870000621500202C0400201804002003B50246B2
:204D2000002006E002EB4001BDF804300B80411CC8B20C28F6D30CBDF0B504460D46671B6A
:204D400039B2178892F802C007FB0CF74FF0640C97FBFCF7BBB29778C7EBC70707EB470609
:204D6000002901DA002014E0994206DA4FF4B6774F4397FBF3F7B8B20BE0CF1A4FF4D96C1C
:204D800007FB0CF7A6EB030C97FBFCF707F5B677B8B2F0BD08B5024602F5004081B20846EC
:204DA000CB1701EB936399114FF6FE70014001F4407038B3B0F5807F36D0B0F5007F03D060
:204DC000B0F5407F40D10DE0C8B2214B33F81000ADF80200C8B2C0F1FF0033F81000ADF89F
:204DE000000032E0C8B2C0F1FF00194B33F81000ADF80200C8B233F81000404200B2ADF8A3
:204E0000000022E0C8B2124B33F81000404200B2ADF80200C8B2C0F1FF0033F810004042BC
:204E200000B2ADF8000010E0C8B2C0F1FF00084B33F81000404200B2ADF80200C8B233F8F3
:204E40001000ADF8000000E000BF00BF009808BD3A6F010870B505466C6A0020E085E08401
:204E60002046F7F7EEF870BD2DE9F04106460D461446002025490870F5F7C6FC23494860C3
:204E800005F0FF08A5F50040083830B1A0F6FA70B8B1B0F5545F2DD108E0424621461C4821
:204EA000EEF7FDFD00201B4908702BE023462A46314640F21560FEF79FFF0120164908708A
:204EC00020E02178627801EB02218FB2002007E0124931F81010B94200DD03E0411CC8B2D2
:204EE0000B28F5D300BF00F14901CAB20C4981F8252007E023462A46314640F21560FEF75B
:204F00007BFF00BF00BFBDE8F0810000D4010020C8010020D20100205D00002004730108B5
:204F20001C09002010B50A46C37893421EDBC3681B68DB6823F02003C4682468E360C378B1
:204F40009B1AC370C3681B68DB6843F02003C4682468E360114683780B4499B203788B42F3
:204F600002DC0378CB1A99B281701BE0C3681B68DB6823F02003C4682468E360C17800233E
:204F8000C370C3681B68DB6843F02003C4682468E3608378194403788B4202DC0378CB1ABE
:204FA00099B2817010BD0168C96821F490710268D1600168496921F0010102685161202112
:204FC00080F83A10704710B504462068C06820F040002168C860202084F839002046F7F74F
:204FE00076F9002010BD00BFC27803789A42FBD0C2681268D26822F08002C3681B68DA60E0
:20500000C2788AB9C26812681268C2F3C0125AB1C26812685160C2681268D26842F080027C
:20502000C3681B68DA60704743788268D1544278521CD2B2427003789A4201D100224270AC
:20504000C278521CC270C2681268D26842F08002C3681B68DA6000BFE5E710B502460B4613
:205060001946D4789C4209DB94780C44A1B214788C4204DC14780C1BA1B200E000219468D7
:20508000605C10BD70B5044694F83A0022284AD1A068B0F5805F13D1A56A206940B9206864
:2050A0004068C0F308002880A06A801CA06219E020684068C0B22880A06A401CA06211E0A1
:2050C000206938B920684068C1B2A26A501CA062117007E02068406800F07F01A26A501CB9
:2050E000A0621170E08D401E80B2E085C8B92068C06820F020002168C8602068C06820F4F5
:2051000080702168C8602068406920F0010021684861202084F83A002046F7F7D7F8002041
:2051200070BD0020FCE70220FAE7F0B507460D461646002405E0295D3846FFF754FF601CC9
:20514000C4B2B442F7DBF0BD2DE9F041044600252068006920F44050E16808432168086193
:205160002169A06808436169084305432068C06841F20C61884328432168C860206840698D
:2051800020F44070A1690843216848615F49206888425CD1F5F78CFE00EBC00101EB00107F
:2051A00061688900B0FBF1F6F5F782FE00EBC00101EB001061688900B0FBF1F06421B0FBE9
:2051C000F1F000EBC00101EB0010A6EB8000322101EB00106421B0FBF1F000F0F006F5F703
:2051E00067FE00EBC00101EB001061688900B0FBF1F06421B0FBF1F006EB0016F5F758FE6A
:2052000000EBC00101EB001061688900B0FBF1F7F5F74EFE00EBC00101EB001061688900CF
:20522000B0FBF1F06421B0FBF1F000EBC00101EB0010A7EB8000322101EB00106421B0FB98
:20524000F1F000F00F003044216888605BE0F5F71FFE00EBC00101EB001061688900B0FBA0
:20526000F1F6F5F715FE00EBC00101EB001061688900B0FBF1F06421B0FBF1F000EBC00105
:2052800001EB0010A6EB8000322101EB00106421B0FBF1F000F0F006F5F7FAFD00EBC0012C
:2052A00001EB001061688900B0FBF1F06421B0FBF1F006EB0016F5F7EBFD00EBC00101EB90
:2052C000001061688900B0FBF1F7F5F7E1FD00EBC00101EB001061688900B0FBF1F0642104
:2052E000B0FBF1F000EBC00101EB0010A7EB8000322101EB00106421B0FBF1F000F00F0009
:20530000304421688860BDE8F081000000380140014691F8390021282CD18868B0F5805F56
:205320000FD10A6A1088C0F308000B685860086918B9086A801C086209E0086A401C0862C0
:2053400005E00B6A581C086218780B685860C88C401E80B2C88458B90868C06820F08000F1
:205360000B68D8600868C06840F040000B68D860002070470220FCE710B5054800F00EF8EB
:20538000044800F040F80448F6F75CFE10BD0000E0050020F0050020EC24002008B5C26808
:2053A00012681268C2F3401262B3C26812685268D1B2C268126812680022B2B943788268AC
:2053C000D1544278521CD2B2427003789A4201DB00224270C278521CD2B2C27003789A428E
:2053E00003DD0278C2700122027100BF00220092C268126812680092C26812685268009278
:2054000000BF00BF08BDC16809680968C1F3C01139B3C1680968C96801F0800109B36FF075
:205420008001C26812681160C17891B1C178491EC17082788168895CC26812685160817874
:20544000491CC9B28170027891420ADB0021817007E0C1680968C96821F08001C26812684F
:20546000D160704710B50248F4F7C2F810BD0000A822002010B54FF4FA71024800F004F830
:2054800010BD0000E00500202DE9F34F83B00398C0780D2873DB00210398FFF7DEFD01903B
:2054A0006B490198087001210398FFF7D6FD8146674981F80190019855287DD1B9F1AA0F59
:2054C000FBD102210398FFF7C8FD6149887003210398FFF7C2FD5E49C87004210398FFF7DC
:2054E000BCFD06465A490E71112E03D0162E01D00C2E7DD105210398FFF7AFFD074654488A
:20550000477107210398FFF7A8FD834606210398FFF7A3FD0BEB00201FFA80F84FEA18203C
:205520004B49887181F8078007210398FFF795FD0446381B02287AD10398C17807F10B00AA
:2055400081421DDA43480078012806D1F5F75CF94149086000203F490870F5F755F93E497A
:205560000968411A0498814206D9F5F74DF93A49086001203749087005B0BDE8F08F64E0CE
:2055800001203449087000250FE005F10800C1B20398FFF762FD314948550846415D05F187
:2055A00008002B4A1154681C85B2A542EDDB04F10800C1B2039800E043E0FFF74EFD4FEA17
:2055C000006B04F10900C1B20398FFF746FD0BEB004B04F10A00C1B20398FFF73EFD0BEBA6
:2055E000002B04F10B00C1B20398FFF736FD00E022E05844029004F108011548EFF7DAFD21
:2056000082460298B0EB0A000CD1144A41463046FFF72AFC07F10B00C1B20398FFF782FCAA
:20562000AAE704E001210398FFF77CFC0DE001210398FFF777FC08E001210398FFF772FCAE
:2056400003E001210398FFF76DFC00BF94E70000FE110020180200201402002068110020D9
:20566000012806D0022845D003287DD004287CD1AAE0FE49FE4A13680B6053684B6092689C
:205680008A600A46FB490B68D3604B681361896851611146F84A13688B615368CB6192683B
:2056A0000A62F64A13684B6253688B629268CA62F34A13680B6353684B6392688A63F14998
:2056C000C978AA2915D140F27321E84A118040F2FD31918140F2226111834FF40C72E3499F
:2056E0004A8340F63411E14A91844FF40C72DF49CA8492E0DD4AE4490B6813604B685360D9
:20570000896891601146E14A1368CB6053680B6192684A61DE4A13688B615368CB61926843
:205720000A62DC4A13684B6253688B629268CA620A46D9490B6813634B6853638968916338
:20574000D049C978AA2917D140F2CA21118040F27641918140F2747111834FF40C72C34913
:205760004A8340F62E3101E007E055E0BF4A91844FF40C72BD49CA844FE0BC49C74A1368D7
:205780000B6053684B6092688A60C54A1368CB6053680B6192684A61C24A13688B615368A5
:2057A000CB6192680A620A46BF490B6853624B6893628968D1621146BC4A13680B6353680A
:2057C0004B6392688A6328E0A84AB9490B6813604B685360896891601146B64A1368CB600D
:2057E00053680B6192684A610A46B3490B6893614B68D361896811621146B04A13684B6266
:2058000053688B629268CA62AD4A13680B6353684B6392688A6300E000BF00BFA949897B36
:2058200078290DDCA749897B502909DB8F490988A44A927B5143642291FBF2F18B4A11803A
:20584000A049097C78290DDC9E49097C502909DB864989899B4A127C5143642291FBF2F1AA
:20586000824A91819749897C78290DDC9549897C502909DB7D49098B924A927C514364223D
:2058800091FBF2F1794A11838E49097D78290DDC8C49097D502909DB7449898C894A127D6F
:2058A0005143642291FBF2F1704A91848549897D78290EDC8349897D50290ADB6B49498E76
:2058C000804A927D5143642291FBF2F18AB267494A867C49C97B5A2905DC6449097A491EA6
:2058E000624A117208E07749C97B6E2904DB5F49097A491C5D4A11727249497C5A2906DC78
:205900005A49097D491ECAB258490A7509E06D49497C6E2905DB5549097D491CCAB25349DF
:205920000A756849C97C5A2908DC504991F82010491ECAB24D4981F820200BE06149C97C2D
:205940006E2907DB494991F82010491CCAB2474981F820205B49497D5A2908DC434991F873
:205960002C10491ECAB2414981F82C200BE05549497D6E2907DB3D4991F82C10491CCAB2C5
:205980003A4981F82C204F49C97D5A2908DC374991F83810491ECAB2344981F838200BE00D
:2059A0004849C97D6E2907DB304991F83810491CCAB22E4981F838204349C97C78290DDCC9
:2059C0004149C97C502909DB2849C9883E4AD27C5143642291FBF2F1244AD1803A49497D72
:2059E00078290EDC3849497D50290ADB1F49498A354A527D5143642291FBF2F18AB21B49C5
:205A00004A823149C97D78290EDC2F49C97D50290ADB1649C98B2C4AD27D5143642291FB35
:205A2000F2F18AB21149CA832749497E78290EDC2549497E50290ADB0C49498D224A527EE4
:205A40005143642291FBF2F18AB208494A851E49C97E78293FDC1C49C97E50293BDB034970
:205A6000C98E194AD27E514364222FE0E40B00201A73010826730108327301083E73010844
:205A80004A730108BA01002056730108627301086E7301087A7301088673010892730108C5
:205AA0009E730108AA730108B6730108C2730108CE730108DA730108E6730108F2730108C6
:205AC000FE730108B00A0020D00A002091FBF2F18AB23049CA863049897C78290DDC2E4985
:205AE000897C502909DB2B4949892B4A927C5143642291FBF2F1274A51812749097D782918
:205B00000EDC2549097D50290ADB2249C98A224A127D5143642291FBF2F18AB21D49CA8219
:205B20001D49897D78290EDC1B49897D50290ADB1849498C184A927D5143642291FBF2F176
:205B40008AB214494A841449097E78290EDC1249097E50290ADB0F49C98D0F4A127E514304
:205B6000642291FBF2F18AB20A49CA850A49897E78290EDC0849897E50290ADB0549498F91
:205B8000054A927E5143642291FBF2F18AB201494A877047E40B0020D00A002000BFFEE762
:205BA00000B587B00020C7490860C74908800720C64908701821C648EDF78AFF1821C54821
:205BC000EDF786FF1821C448EDF782FF1022C349C348EDF764FFC348C3490A680260496886
:205BE00041601022C1A1C648EDF77DFF1022C5A1C3481030EDF777FF2E21C148203880F89D
:205C00003F102022C4A1CD48EDF76DFF00BFCCA2D2E900109268CDE905020491CBA207CAA7
:205C200001AB07C39DF81A0030389DF81910303901EB810100EB4100C04988760322C6A183
:205C400004A8EDF772FF18B90120BC49C87670E00322C2A104A8EDF768FF18B90220B7494C
:205C6000C87666E00322BEA104A8EDF75EFF18B90320B249C8765CE00322BAA104A8EDF7B6
:205C800054FF18B90420AD49C87652E00322B6A104A8EDF74AFF18B90520A849C87648E0B4
:205CA0000322B2A104A8EDF740FF18B90620A349C8763EE00322AEA104A8EDF736FF18B954
:205CC00007209E49C87634E00322AAA104A8EDF72CFF18B908209949C8762AE00322A6A1AA
:205CE00004A8EDF722FF18B909209449C87620E00322A2A104A8EDF718FF18B90A208F49FC
:205D0000C87616E003229EA104A8EDF70EFF18B90B208A49C8760CE003229AA104A8EDF765
:205D200004FF18B90C208549C87602E000208349C8769DF8151030399DF81400202801D165
:205D4000002002E09DF81400303800EB800001EB40007A4908779DF8051030399DF80400AB
:205D6000202801D1002002E09DF80400303800EB800001EB4000714948779DF808103039E0
:205D80009DF80700202801D1002002E09DF80700303800EB800001EB4000684988779DF86B
:205DA0000B1030399DF80A00202801D1002002E09DF80A00303800EB800001EB40005F495E
:205DC000C87700BF7048007828B930214C48203880F82A1036E06C480078012805D1312132
:205DE0004748203880F82A102CE067480078022805D132214248203880F82A1022E0624844
:205E00000078052805D132213D48203880F82A1018E05D480078032805D1332138482038E3
:205E200080F82A100EE058480078042805D134213348203880F82A1004E0302130482038C9
:205E400080F82A10102251A12D482038EDF74BFE102253A12A481038EDF745FE082255A14B
:205E60005748EDF740FE082256A155480830EDF73AFE082256A152481030EDF734FE57489F
:205E8000574B0ECB0EC000F0D7F800F0AFF85548007B544991F91B10084452498979484385
:205EA000C0EB001001034F48C07941F2C6125043B1FBF0F04C49888108468089C88107B034
:205EC00000BD00008C010020C8010020B00100208C090020980A0020800A0020647101089F
:205EE000A4090020B10100204072010820202020202020203336202020202020000000001F
:205F00003C0900205636723272325F32303235303733314300000000544330313130303059
:205F20002D4D53303030302D563072312E2020202020202020202020000000005C0900206B
:205F40004A756C20333120323032350031303A32303A3139000000004A616E0046656200E2
:205F60004D617200417072004D6179004A756E004A756C0041756700536570004F637400F4
:205F80004E6F760044656300FC010020564C363530302026205653373530302E000000002F
:205FA00030303030303030303030303030303030000000004D4F54494E4F56410000000074
:205FC000400B0020575548414E2E202000000000323032313039303100000000B80B0020F3
:205FE000E8F7FF1FB00A00200402002010B5302209490A48EDF753FD102209490948EDF7FC
:206000004EFD0948094C1ECC1EC0102208490948EDF745FD10BD00009C720108000B0020BE
:20602000CC720108300B0020200C0020EC720108DC720108300C002010B50C2213A1174852
:20604000EDF751FD164817490A680260496841601548164909680160202215491548EDF7BB
:206060001EFD1448007814490870202213491448EDF715FD102213491348EDF710FDCC22A4
:2060800012491348EDF70BFD10BD000030303030303030303030303000000000C40B002062
:2060A000BF010020FC720108BA0100208872010848720108B00A0020B90100206872010851
:2060C000D00A00208C720108F00A002074710108B409002088B004460D4631E01948FAF7A2
:2060E000BEF80020FBF7ECFEF0F7C8FE20216846EDF7EEFC2046EDF702FD06463246214610
:206100006846EDF7CCFC2046EDF7F9FC694608440DA10A880280897881702046EDF7EFFC02
:2061200069460844C0F803506B464FF620720C214FF4E260FDF760FEC820F4F77FF800BFC4
:20614000CCE7000000010020202C200008B52B4988420DD100BF2A49896941F00401284A5A
:2061600091611146896901F00401009100BF43E0244988420DD100BF2149896941F0080111
:206180001F4A91611146896901F00801009100BF32E01D4988420DD100BF1949896941F0AD
:2061A0001001174A91611146896901F01001009100BF21E0154988420DD100BF10498969CF
:2061C00041F020010E4A91611146896901F02001009100BF10E00E4988420DD100BF084979
:2061E000896941F04001064A91611146896901F04001009100BF00BF08BD00000008014061
:2062000000100240000C014000100140001401400018014070B504460E46A1882068F4F781
:20622000E1FA28B9A07908B9012506E0002504E0A07908B9002500E00125012E04D1207A10
:2062400068402840E07102E0207A6840E071257270BD10B50446A18801222068F4F7CEFA0E
:2062600010BD00BF704702E008C8121F08C1002AFAD170477047002001E001C1121F002AAE
:20628000FBD1704700F0010181F3138870470000014908607047000010060020F0B5044635
:2062A0000E4619681F683D14A54206DA31440814A04212DD204601040FE0A5420CDD02EBF1
:2062C00004473DB2A94202DA2046010405E0891A081410B9002100E020461960F0BD000058
:2062E00010B50A46437993421EDB1E4B1B685B6923F002031B4C2468636143799B1A43715B
:20630000184B1B685B6943F00203164C24686361114603790B4499B283788B4202DC8378DB
:20632000CB1A99B201711BE00E4B1B685B6923F002030C4C24686361417900234371094B7B
:206340001B685B6943F00203064C246863610379194483788B4202DC8378CB1A99B2017100
:2063600010BD0000A822002010B502460B46194654799C4209DB14790C44A1B294788C4210
:2063800004DC94780C1BA1B200E000219468605C10BD00007FB50646002404E0305D18499B
:2063A0000855601CC4B2082CF8DB3823154A02A9304600F08DFB00241EE0002504E002A85F
:2063C00000F0AEFA681CC5B20F48005DA842F6DC40230E4A694602A800F07AFB002507E035
:2063E0001DF805000A4901EBC4014855681CC5B2082DF5DB601CC4B2102CDEDB7FBD0000BF
:2064000095030020CC7A0108A47D0108047B01085614002001460120064A12688A4206D164
:20642000044A1268044B1B685A40521C02B10020704700002C250020502500202DE9F04FD5
:2064400087B082460F469046994600250AE0785D3A49495D884203D03846FFF79BFF07254F
:20646000681CC5B2082DF2DB4023354A05A9504600F02EFB012536E0002405E005A8005D91
:2064800003A90855601CC4B2082CF7DBB8F1000F04D1681E2B4901EBC00B04E0C5F1100013
:2064A000284901EBC00B002406E003A9201D085C05A90855601CC4B2042CF6DB01AA05A906
:2064C000584600F043F8002409E003A8005D01A9095D484005AA211D5054601CC4B2042C93
:2064E000F3DB681CC5B2112DC6DB9DF814609DF818008DF814008DF818609DF815609DF809
:2065000019008DF815008DF819609DF816609DF81A008DF816008DF81A609DF817609DF8D5
:206520001B008DF817008DF81B604023064A494605A800F0CDFA07B0BDE8F08F950300206B
:206540000C7A0108561400204C7A0108F0B587B005460E4617464023104A05A9304600F0AA
:20656000B7FA002410E005A8005D295D484000F03F0003A908550A4800EB8410095D405C33
:2065800001A90855601CC4B2082CECDB2023054A394601A800F09CFA07B0F0BD447B01089B
:2065A000A47B0108847B01081CB5F6F719F9F6F71FF9B7490870F4F769F9FDF77FFFF6F7B2
:2065C00051FAFAF7C3FFFBF763F8FBF7CBF8FBF713F9FAF7A1FFFAF769FEFAF717FFFAF7DC
:2065E0006DFFFBF753F9FCF7E5F9EDF771FF1420F3F724FEA748F5F73BF9FFF7D1FAFBF7CA
:2066000027F8FAF70FFCA448F0F7E0FCF0F762FEA148F0F793FCF0F7A9FEA04908700846CD
:2066200001789D48FDF79EFB9D499E48F0F77CFEF9F744FDF1F76CFB00209B49087026E13F
:206640009A480078401C9949087008460078C82801DD0020087096480088F1F7DBFDFBF7E6
:20666000DBF9EEF72BFFFEF705FF924A5178924AD07A924B924A1278F8F798FAFAF7D2FDEF
:20668000F0F7C6FB8C48807EAA2841D18D48007BC0B18C48B0F902000B2190FBF1F084B28E
:2066A00088498548007B844A92F91B20104480B2CDE900018048C379827983492046FDF7CB
:2066C0008DFC46E07F48B0F902000B2190FBF1F07C49897A884206DD7A48B0F902000B21F3
:2066E00090FBF1F001E07748807A84B275497248007B714A92F91B20104480B2CDE90001AD
:206700006D48C379827970492046FDF767FC20E06948807EEE280AD16748007B6649C97E57
:206720000844C2B267496848FDF79CFC11E06248007B6149C97E0844C2B25F48007E08B900
:20674000012001E05C48007E03465E495E48FDF709FD5E48F1F740FD5D48EEF7C9F900BFAF
:206760005C48007818BB5C48007828B1F4F74CF842F21071884229D95248C0880A2190FBED
:20678000F1F084B2554880884B4A0090127B4A4D95F91B502A4490B2514A137B4E4A117801
:2067A0002246FBF7D7FD01204A4908700EE0454C23894A4C627AA188434CE068FBF7A4FC50
:2067C000484A11783D4A1078FBF7FAFD00BFFAF70DF9F8F7F1FA4448FAF780FAFAF78AFCA8
:2067E000384B9A7D1989987AF8F700F83F4908703C48807910B93E48F0F78CFD39488079AE
:2068000030B93C493C48F0F727FE3C48FBF76CFF3B480078E8B93B4800683B4908603948A5
:20682000406848603748806888603648C068C8602D48001F4068086128221A480830FDF76E
:20684000D9F9042231A11748FDF7D4F901202C490870F8F71DFCF9F765FD2E480068FAF717
:2068600097FA17480078FAF7BBFA15480078FAF763FA2948FAF7F2FAFDF782FBF1F7A8FA9E
:20688000FCF712FEFCF716F82448F3F7EBFFD7E6FC010020D01C00202C0400202404002036
:2068A000FFEF010800E801085C0000205A00002000020020B1010020B00A0020DA00002032
:2068C000D8000020DC080020EC0300203D0400203C0400205B000020EC0100207C090020BF
:2068E000F00A0020DE000020040B0020EE000020250400209D03002088070020BE010020AC
:2069000003020020200C0020900B0020464C4147000000008C010020D00B0020F007002072
:206920000CB5002104E0425C0DF801204A1CD1B20829F8DB002112E0425C5206120E425421
:2069400006290ADA4A1C1DF8022002F08002802A03D1425C42F0010242544A1CD1B2072913
:20696000EADB9DF8002002F0800222B1C27842F01002C27003E0C27822F01002C2709DF89E
:20698000032002F0080222B1827942F00102827103E0827922F0010282710CBD2DE9F041EC
:2069A00006460F46EDF7ECFB04000D4618BF0120284320F00040C0F17F6000F1E040C00FF1
:2069C0000ED0301C18BF0120384320F00040C0F17F6000F1E040C00F04BF0120FFF758FC2C
:2069E00020462946BDE8F08130B502460023002952D03348007890B13248334C247830F820
:206A00001400324C2468201A304C206020460068104420602B482C4C247820F814202A483B
:206A20000078401C284C2070204600781E280FDB002020702248007818B90120204C2070F0
:206A400006E01F480078012802D102201C4C20701B480078022806D11C4800681E24B0FBC6
:206A6000F4F083B211E01648007801280CD11648007808B9134608E014480068124C24789A
:206A8000B0FBF4F083B200E01346052093FBF0F0904212DD134610E0002005E00024094DDD
:206AA00025F81040441CE0B21E28F7DB0020064C2070064C2060024C2070184630BD000062
:206AC000E8030020EA140020E0030020E40300202DE9F04104461D46154E002000BF4FF00E
:206AE00000080746401C01F807800828F7DB002000BF12F8013B04EBE3073F7803F0070CA8
:206B000016F80CC007EA0C0767B101EBE0073F7800F0070C16F80CC047EA0C0701EBE00CFC
:206B20008CF80070471C3846AF42E2DBBDE8F081B47D010800000000000000000102030478
:206B4000060708090000000001020304204E00040300000400000004000000009CFFFFFFF7
:206B6000FF7F0000000000FE00FCFF0100000000204E000403000004000000040000000020
:206B80000080FFFFFF7F0000000000FE00FCFF0100000000400000040300000400000004B0
:206BA000000000000000FCFF00000000000000F00000000000000000307500012C01000413
:206BC0000000000400000000CCF7FFFF000000000030DFFF000000000000000000100004CE
:206BE0000100000400000004000000009CFFFFFF1A0400000070FEFF0068100000000000F0
:206C0000307500042C0100040000000400000000E6FBFFFF000000000098EFFF0000000031
:206C200000000000204E00040300000400000004000000009CFFFFFFFF7F0000000000FEC2
:206C400000FCFF0100000000204E00040300000400000004000000000080FFFFFF7F0000BF
:206C6000000000FE00FCFF0100000000400000040300000400000004000000000000FCFFD0
:206C800000000000000000F00000000000000000307500012C010004000000040000000029
:206CA000CCF7FFFF000000000030DFFF0000000000000000001000040100000400000004E8
:206CC000000000009CFFFFFF1A0400000070FEFF0068100000000000307500042C0100043E
:206CE0000000000400000000E6FBFFFF000000000098EFFF0000000000000000204E0004B9
:206D00000300000400000004000000009CFFFFFFFF7F0000000000FE00FCFF010000000057
:206D2000204E00040300000400000004000000000080FFFFFF7F0000000000FE00FCFF01E0
:206D400000000000400000040300000400000004000000000000FCFF00000000000000F0F9
:206D60000000000000000000307500012C0100040000000400000000CCF7FFFF0000000077
:206D80000030DFFF0000000000000000001000040100000400000004000000009CFFFFFF2F
:206DA0001A0400000070FEFF0068100000000000307500042C0100040000000400000000F2
:206DC000E6FBFFFF000000000098EFFF0000000000000000204E00040300000400000004D1
:206DE000000000009CFFFFFFFF7F0000000000FE00FCFF0100000000204E00040300000409
:206E000000000004000000000080FFFFFF7F0000000000FE00FCFF01000000004000000434
:206E20000300000400000004000000000000FCFF00000000000000F000000000000000005C
:206E4000307500012C0100040000000400000000CCF7FFFF000000000030DFFF0000000088
:206E600000000000001000040100000400000004000000009CFFFFFF1A0400000070FEFFD1
:206E80000068100000000000307500042C0100040000000400000000E6FBFFFF00000000BD
:206EA0000098EFFF0000000000000000657F367E107D807C657B527A467940784177C47616
:206EC000CE75DF74F47310739F72C271EA701770486F7D6E1A6E566D966CDA6B216B6D6A76
:206EE000136A6469B8680F68696718677666D8653D65A4640E64C4633263A26215628A610B
:206F00004561BE603960B55F345FB55E765EFA5D805D085D915C1C5CE25B705BFF5A905A3D
:206F2000235AED5981591859AF584858E357B1574D57EB568A562B56CC550000C900920197
:206F40005B022403ED03B6047F0548061107D907A2086A09330AFB0AC40B8C0C540D1C0EE8
:206F6000E30EAB0F72103A110112C8128F1355141C15E215A8166E173318F918BE19821A67
:206F8000471B0B1CCF1C931D571E1A1FDD1F9F2061212322E522A62367242825E825A8261A
:206FA00067272628E528A329612A1F2BDC2B992C552D112ECC2E872F4130FB30B5316E32E8
:206FC0002633DF3396344D350436BA366F372438D9388C39403AF23AA53B563C073DB83DA7
:206FE000683E173FC53F73402141CE417A422543D0437A442445CD4575461C47C347694824
:207000000F49B449584AFB4A9D4B3F4CE04C814D204EBF4E5D4FFB4F97503351CE51685212
:2070200002539B533254C9546055F5558A561D57B0574258D3586459F359825A0F5B9C5B05
:20704000285CB35C3E5DC75D4F5ED75E5D5FE35F6860EB606E61F0617162F1627063EE6381
:207060006C64E8646365DD655666CF664667BC673268A66819698B69FD696D6ADC6A4A6BD3
:20708000B76B236C8E6CF86C616DC96D306E966EFB6E5E6FC16F22708370E27040719D713F
:2070A000F9715472AE7207735E73B5730A745F74B27404755575A575F37541768D76D876C9
:2070C00022776B77B377FA773F788478C77809794A798979C879057A417A7C7AB67AEE7A58
:2070E000267B5C7B917BC57BF87B297C597C887CB67CE37C0E7D397D627D897DB07DD57DA5
:20710000FA7D1D7E3E7E5F7E7E7E9C7EB97ED57EEF7E097F217F377F4D7F617F747F867F35
:20712000977FA67FB47FC17FCD7FD87FE17FE97FF07FF57FF97FFD7FFE7F000005000000DD
:2071400000000000050000000000000005000000000000000500000000000000050000001B
:2071600000000000A0282400000000000000000000000000983A38100810F90FEE0FE60FF7
:20718000E00FDB0FD70FD30FCF0FCB0FC70FC20FBC0FB50FAD0FA40F9B0F900F850F7A0F8B
:2071A0006F0F640F5A0F4F0F460F3D0F340F2B0F230F1B0F120F0A0F030FFA0EF20EE90E52
:2071C000E10ED70ECE0EC40EB90EAF0EA40E990E8F0E840E7A0E700E670E5D0E550E4C0E7E
:2071E000440E3D0E350E2E0E270E210E1B0E150E0F0E090E030EFE0DF80DF40DEE0DE90D7C
:20720000E40DDF0DDA0DD40DCE0DC80DC30DBC0DB60DAF0DA70D9F0D970D8E0D850D7B0D48
:20722000700D640D570D490D3B0D2E0D250D1C0D120D080DFD0CF10CE00CC70C930C1C0C08
:20724000045500000000000055026400190310100F87A555DB026464646464646464646489
:2072600001025500B80B3C870000000055020C0C96004B00960000000000646464646464F2
:20728000646464640000000090016400FA00B004C8000A000A00A08C240800000100000086
:2072A00000000000000000000000000000000000000000000000000000000000000041414C
:2072C000000000004141414100000000000000000000000000000000000000006400A000A6
:2072E000BE000E01B4000000000000000000000000000000000000000000000041564F4ED9
:2073000049544F4D7401E8025C04D1054507B9082D0AA20B160D8A0EFF0F880100006400F8
:20732000200302010002120300006400E8030201AE021D05BC026400140503016603AC0791
:20734000480364003408050100040000CC016400340804010004C40100006400480302014B
:207360000002BA0300006400B0040201AE02E005BC026400360603016603320948036400E9
:207380003408050100040000CC016400340804010004DC0130020000A903020152017604A6
:2073A000BC020000E2040302E9016F0748030000B3050402AE02290BD403000034080503BC
:2073C00000040000B00400003408040200040B023002640067030101EB00AE04BC026400E1
:2073E0001F0402014B01B00648036400B805030100022D0BD4036400340805020004000039
:207400003A076400340804010004000000002110422063308440A550C660E77008812991E3
:207420004AA16BB18CC1ADD1CEE1EFF13112100273325222B5529442F772D6623993188398
:207440007BB35AA3BDD39CC3FFF3DEE36224433420040114E664C774A44485546AA54BB5D4
:2074600028850995EEE5CFF5ACC58DD55336722611163006D776F6669556B4465BB77AA718
:2074800019973887DFF7FEE79DD7BCC7C448E5588668A7784008611802282338CCC9EDD9D4
:2074A0008EE9AFF9488969990AA92BB9F55AD44AB77A966A711A500A333A122AFDDBDCCB98
:2074C000BFFB9EEB799B588B3BBB1AABA66C877CE44CC55C222C033C600C411CAEED8FFDD4
:2074E000ECCDCDDD2AAD0BBD688D499D977EB66ED55EF44E133E322E511E700E9FFFBEEF18
:20750000DDDFFCCF1BBF3AAF599F788F8891A981CAB1EBA10CD12DC14EF16FE18010A1004D
:20752000C230E3200450254046706760B9839893FBA3DAB33DC31CD37FE35EF3B102901297
:20754000F322D2323542145277625672EAB5CBA5A89589856EF54FE52CD50DC5E234C324D3
:20756000A01481046674476424540544DBA7FAB79987B8975FE77EF71DC73CD7D326F23617
:207580009106B01657667676154634564CD96DC90EF92FE9C899E9898AB9ABA944586548D3
:2075A00006782768C018E1088238A3287DCB5CDB3FEB1EFBF98BD89BBBAB9ABB754A545A97
:2075C000376A167AF10AD01AB32A923A2EFD0FED6CDD4DCDAABD8BADE89DC98D267C076CD3
:2075E000645C454CA23C832CE01CC10C1FEF3EFF5DCF7CDF9BAFBABFD98FF89F176E367E17
:20760000554E745E932EB23ED10EF01E00000000B71DC1046E3B8209D926430DDC760413D2
:207620006B6BC517B24D861A0550471EB8ED08260FF0C922D6D68A2F61CB4B2B649B0C353B
:20764000D386CD310AA08E3CBDBD4F3870DB114CC7C6D0481EE09345A9FD5241ACAD155F35
:207660001BB0D45BC2969756758B5652C836196A7F2BD86EA60D9B6311105A6714401D7935
:20768000A35DDC7D7A7B9F70CD665E74E0B6239857ABE29C8E8DA191399060953CC0278BFE
:2076A0008BDDE68F52FBA582E5E66486585B2BBEEF46EABA3660A9B7817D68B3842D2FADB3
:2076C0003330EEA9EA16ADA45D0B6CA0906D32D42770F3D0FE56B0DD494B71D94C1B36C76B
:2076E000FB06F7C32220B4CE953D75CA28803AF29F9DFBF646BBB8FBF1A679FFF4F63EE12D
:2077000043EBFFE59ACDBCE82DD07DEC77708634C06D4730194B043DAE56C539AB068227A0
:207720001C1B4323C53D002E7220C12ACF9D8E1278804F16A1A60C1B16BBCD1F13EB8A01E2
:20774000A4F64B057DD00808CACDC90C07AB9778B0B6567C69901571DE8DD475DBDD936B94
:207760006CC0526FB5E6116202FBD066BF469F5E085B5E5AD17D1D576660DC5363309B4D8C
:20778000D42D5A490D0B1944BA16D84097C6A5AC20DB64A8F9FD27A54EE0E6A14BB0A1BF61
:2077A000FCAD60BB258B23B69296E2B22F2BAD8A98366C8E41102F83F60DEE87F35DA9995A
:2077C0004440689D9D662B902A7BEA94E71DB4E0500075E4892636E93E3BF7ED3B6BB0F38A
:2077E0008C7671F7555032FAE24DF3FE5FF0BCC6E8ED7DC231CB3ECF86D6FFCB8386B8D584
:20780000349B79D1EDBD3ADC5AA0FBD8EEE00C6959FDCD6D80DB8E6037C64F643296087AAC
:20782000858BC97E5CAD8A73EBB04B77560D044FE110C54B383686468F2B47428A7B005CF9
:207840003D66C158E4408255535D43519E3B1D252926DC21F0009F2C471D5E28424D193643
:20786000F550D8322C769B3F9B6B5A3B26D6150391CBD40748ED970AFFF0560EFAA0111073
:207880004DBDD014949B93192386521D0E562FF1B94BEEF5606DADF8D7706CFCD2202BE27C
:2078A000653DEAE6BC1BA9EB0B0668EFB6BB27D701A6E6D3D880A5DE6F9D64DA6ACD23C471
:2078C000DDD0E2C004F6A1CDB3EB60C97E8D3EBDC990FFB910B6BCB4A7AB7DB0A2FB3AAED9
